:020000040800F2
:100000000000012025230608A9230608055202083E
:10001000A9230608A9230608A92306080000000052
:10002000000000000000000000000000A9230608F6
:10003000A923060800000000A9230608056B010893
:10004000A9230608A9230608A9230608A923060848
:10005000A9230608A92306084532010849320108E8
:100060004D3201085132010855320108EDB4000843
:1000700001B5000815B5000829B500083DB5000810
:1000800051B5000865B50008A9230608A92306088C
:10009000A9230608A9230608A9230608593201083E
:1000A000C5BD0008E9BC0008D9BD0008D5BC0008E2
:1000B00011BD000825BD000839BD0008EDAA0008E3
:1000C000E1AA000805AB0008F9AA0008A923060860
:1000D000A9230608A1C00008ADC00008B9C00008E7
:1000E0005D320108A9230608A9230608EDBD000812
:1000F00075BD00089DBD000861BD000879B5000808
:10010000A9230608A92306084DBD0008A92306084F
:10011000C5C00008A9230608A9230608B5CE000813
:100120008DB50008A1B50008B5B50008C9B500082F
:10013000DDB5000800000000000000000000000025
:100140000000000000000000000000004BC200089A
:10015000F1B5000805B6000819B60008D1C00008BE
:100160001DAB000811AB0008A9230608A923060847
:10017000A9230608A92306080000000000000000CB
:10018000A9230608A9230608A9230608A923060807
:10019000A9230608A923060800000000A9230608D1
:1001A000000000000000000000000000A923060875
:1001B000A9230608A923060800000000000000008B
:1001C000000000000000000000000000000000002F
:1001D000000000000000000000000000A923060845
:0801E000701E06000100000082
:1001E800182F02200201000007002200382F0220E9
:1001F8000202000102003F00582F0220010B0000FC
:1002080000007600782F0220010F00000000760021
:10021800982F0220010C010000007700B82F02205F
:100228000111000000007600D82F02200113000001
:1002380000001E00F82F02200119000000000D0028
:10024800183002200115000000000C003830022090
:10025800011A000000000E0058300220011B0000A7
:1002680000001E00783002200116000000000C007B
:10027800983002200117000000000E00B83002205C
:100288000118000000000C00D830022001270100EE
:1002980000001800F8300220011F0000000048008C
:1002A80018310220012000000000490038310220E6
:1002B8000121000000004A005831022001220000FC
:1002C80000004B00783102200123000000004C00A0
:1002D800983102200124000000004D00B8310220AE
:1002E8000125000000004E00D83102200126000040
:1002F80000004F00F8310220012A00000000290008
:1003080018320220012B0100000029003832022097
:10031800012C01000000700058320220012D01005C
:100328000000520078320220012E0100000028004F
:10033800983202200228010000012C00B832022065
:100348000232060000024200D832022001310000C9
:1003580000003C00F83202200134000000002000B8
:10800000836B1A6C12F0500F21D11A6C42F400727B
:108010001A641A68916811F0405F1BD19969C9B957
:10802000D16A11F4700F02D09168490512D45168D9
:1080300021F0200151601A6C22F480721A641A6CCB
:10804000D20407D41A6C42F001021A6470479B6B89
:10805000DB6C184770477047836B40221A645A6C78
:1080600042F004025A64704790F83530022B03D076
:1080700080234365012070470268052380F835306E
:108080000020136823F00103136070470268436BFC
:108090009169126803B118477047836B19684A6881
:1080A00042F400424A600022996B0A65D96B0A6566
:1080B00093F84120602A02D1202283F841207047A2
:1080C000F0B5059D06680C4FB46931EA04040CBF95
:1080D00001240024944201D000200CE03C68641B81
:1080E0009C42F1D9202380F84130002380F84230AF
:1080F00080F840300320F0BD5022012030B50468E4
:10810000039D60682B4320F07F700B4320F45930AF
:1081100043EA024320F47F7020F0030003436360CE
:1081200030BD836B0022A3F85A20A3F85220704779
:10813000436ADA0710B506D50168846A4A6822F4F2
:10814000003222434A609C0706D50168C46A4A6827
:1081500022F4803222434A60590706D50168046B35
:108160004A6822F4802222434A601A0706D5016831
:10817000446B4A6822F4004222434A60DC0606D57A
:108180000168846B8A6822F4805222438A609906CF
:1081900006D50168C46B8A6822F4005222438A60C3
:1081A0005A0610D50168046C4A68B4F5801F22F4A1
:1081B000801242EA04024A6005D14A68446C22F403
:1081C000C00222434A601B0606D50268816C5368D0
:1081D00023F400230B43536010BD0F4B984215D07E
:1081E000A3F57843984213D003F58063984211D0E9
:1081F00003F57843984208D10323084A142101FB70
:108200000322138A01339BB2138270470023F4E7E1
:108210000123F2E70223F0E70030014000000120D3
:10822000036920221F2B70B544682DD9A3F12005C6
:108230006168AA400A4226D08069027C022A01D1E4
:108240000022027445681F2B134A2969C1F30321D8
:1082500002EB81018968565CC1684868815921F048
:108260000101815128686D79C16802EB4502128DC8
:1082700002F4F05221EA0202C2604FF0200206D955
:10828000203B9A40E26070BD21689A40D2E702FA32
:1082900003F3A360F7E700BFD87E0608D0E9072301
:1082A0009A422FBFD01AC0688018C01A7047D0E910
:1082B000092300699A4238BF12180138D31AC01A2C
:1082C0007047D0E90902131A5842584170470246D4
:1082D000036A4169C85C0133D1688B4228BF00231F
:1082E00013627047436A8269D154436A0269013359
:1082F000934228BF0023426B4362136843F080031C
:1083000013607047436BD86910F0100002D0102240
:1083100001201A6270477047704701207047014B77
:108320005868704750220120034B93F80402C31E83
:1083300058425841704700BF50220120012380F865
:108340004930704708B5D0F814320BB9022008BD87
:108350001B6898470028FAD0F8E7D0F818321BB10C
:108360000020C3F81402704702207047D0F8302272
:1083700001F00F01D0F8183210B51C2404FB0122C3
:1083800003F50371B2F81022C3F80C22D0F81C22B6
:10839000D3F80402D2689047002010BDD0F81C32F8
:1083A00010B56BB1D0F8184294F80002FF2807D03E
:1083B0009B68214694F801229847FF2384F80032F5
:1083C000002010BD43230380004870475000012067
:1083D0004323038000487047940001204323038017
:1083E00000487047D80001200A23038000487047E6
:1083F0001C01012020230380004870472801012030
:108400002023038000487047480101202023038077
:1084100000487047680101200A2303800048704724
:1084200088010120042301480B807047940101203A
:10843000002370B54D1C1E46040FB0F1204F4FEACB
:10844000001034BF3034373401F8134005F813609E
:108450000133DCB2A242EFD870BD1A2310B50B80F5
:10846000094BD3F8100AD3F8182A80180AD0D3F889
:10847000144A08220549FFF7DBFF04221031204689
:10848000FFF7D6FF024810BD0070F01F9A010120CF
:108490009801012000207047212808B51CD022280F
:1084A0002CD0202816D1A9B1072A13D11A4B08794C
:1084B0000A6883F8B80148798979C3F8B42183F848
:1084C000B90183F8BA11154BD3F83C3213B11146F8
:1084D00000209847002008BD0029FBD0072AF9D1C9
:1084E0000D4BD3F8B4210A6093F8B8210A7193F8C0
:1084F000B92193F8BA314A718B71EBE70029E9D0C1
:10850000022AE7D1054BD3F84032002BE2D009888C
:1085100000209847DEE700BF000001205022012024
:10852000064AD2E99132934203F1FF338CBF002017
:1085300001209B1A03EB0030704700BF502201203E
:10854000EEE7034B93F87002003818BF0120704724
:1085500050220120034B93F87002032894BF00209F
:10856000012070475022012000487047C424012098
:10857000837B042B0DD0074BD3F898200132C3F82E
:108580009820426004228273D3F89C200132C3F801
:108590009C2070471C3F01200020704738B5002503
:1085A000044680F8425090F84130292B0AD1282304
:1085B000012180F841302123036358F0FFFD84F846
:1085C000405038BD90F841302A2BFAD1282302219F
:1085D00080F8413022230363EFE7154B202210B5CA
:1085E000C362002304460363436380F8412080F89C
:1085F00042304B0711D503685A6A436A591C4162DD
:108600001A70038D4BB1013B0385438D013B9BB237
:108610004385436C43F0040343640721204658F02C
:10862000CDFD23681022DA61002384F8403010BDAC
:108630000000FFFF0022304B10B580F842200446B6
:10864000C3624285436C1943416490F84130282B42
:1086500007D090F84130292B03D090F841302A2BD5
:1086600021D10321204658F0A9FD282384F8413068
:1086700000232363214B6363236819681A6811F48C
:1086800080411DD022F48042A06B1A601C4B036510
:10869000002384F84030FFF7E7FC58B3A06B036D6C
:1086A000BDE810401847072158F088FD94F8413084
:1086B000602B02D0202384F8413000232363DAE7C3
:1086C00012F400420DD01A68E06B22F400421A60E6
:1086D0000B4B036584F84010FFF7C6FC50B1E06B0C
:1086E000DDE794F84130602B02D1202384F841303B
:1086F00084F8402010BD00BF0000FFFF2DA000083F
:108700009B800008036899691A6810B4CC0508D5E5
:10871000140606D5446C44F0010444644FF480749C
:10872000DC614C0508D5140606D5446C44F00804F9
:1087300044644FF48064DC61890508D5120606D5CF
:10874000426C42F0020242644FF40072DA61436C00
:1087500013F00B0F03D0416C5DF8044B6AE75DF832
:10876000044B704703682DE9F04F13F0010885B002
:1087700000F0C881AC4A916821F400019160C16A9F
:1087800094680C43B1FA81F14909946013F400260E
:1087900000F0BA81A44D426BD5F88C40B2F5801F31
:1087A00024F4401444EA0204C5F88C4000F0AE8181
:1087B000B2FA82F2520913F48014019411D0DFF856
:1087C00068C2856BDCF88C40B5F5800F24F440045A
:1087D00044EA0504CCF88C4000F09B81002D08BFD2
:1087E00001229F0638D5904CDFF844C2256C45F035
:1087F00080552564246C04F080540394039C8B4CB6
:10880000256845F480752560DCF800E02568ED05F5
:1088100040F18181844C856AD4F870E005F4407998
:108820001EF4407E40F08281B9F5407F7E4C40F0DE
:10883000A981D4F808C025F0704E2CF4F81C2EF451
:10884000407E4CEA0E0CC4F808C0C5F30B05D4F802
:1088500070C045EA0C052567DC060CD5724DD5F8CD
:108860008C4024F08074C5F88C40D5F88C40076BA0
:108870003C43C5F88C405F0409D5DFF8ACC1C46D3A
:10888000DCF8905025F440352C43CCF890401D0482
:1088900009D5DFF894C1046EDCF8905025F440252A
:1088A0002C43CCF89040DC0309D5DFF87CC1446E42
:1088B000DCF8905025F440152C43CCF890405F062E
:1088C00009D5DFF864C1C46BDCF8905025F00305CE
:1088D0002C43CCF890401D0609D5DFF84CC1046C40
:1088E000DCF8905025F00C052C43CCF89040DC05CA
:1088F00009D5DFF834C1446CDCF8905025F0300520
:108900002C43CCF890409F0509D5DFF81CC1846C3E
:10891000DCF8905025F0C0052C43CCF890405D0564
:1089200009D5DFF804C1C46CDCF8905025F440751B
:108930002C43CCF890401C0509D5DFF8ECC0046D41
:10894000DCF8905025F440652C43CCF89040DF04CF
:1089500009D5DFF8D4C0446DDCF8905025F44055BB
:108960002C43CCF890409D0409D5DFF8BCC0846D41
:10897000DCF8905025F440452C43CCF8904013F49B
:1089800000150FD0DFF8A0E0D0F874C0DEF89040FA
:10899000BCF1006F24F0006408BF012244EA0C041B
:1089A000CEF890405C030AD5DFF87CE0DEF890401A
:1089B00024F0407CC46E4CEA0404CEF890401F02C0
:1089C0000AD5DFF864E0DEF8904024F0805C846F24
:1089D0004CEA0404CEF890405C0140F1D880DFF806
:1089E00048E0DEF8904024F0005CC46F4CEA0404D8
:1089F000CEF89040002940F0CF80012A40F08080DE
:108A0000094B0B491A6822F080521A600C681A68E8
:108A1000970000F178810EB1426B5AB1019A002A99
:108A200038D0826BB2BB05E00038024000700040D5
:108A300050220120D3F888404FF4403696FAA6FE23
:108A400047F6C072BEFA8EFE92FAA2F2B2FA82F72E
:108A500096FAA6F64FF0706CB6FA86F69CFAACFC65
:108A60000269BCFA8CFC04F44034BA40476924FA29
:108A70000EF407FA0CF7B4403A432243C3F88820B7
:108A8000D3F88C20046A22F4F852013C42EA042212
:108A9000C3F88C2055B3436FB3F1006F26D1A04DBE
:108AA0004FF0706CD5F888209CFAACF747F6C0738D
:108AB000B7FA87F793FAA3F34FF44034B3FA83F687
:108AC00094FAA4F4B4FA84F49CFAACFC036902F0BE
:108AD00070628069BCFA8CFCB340FA4000FA04F47E
:108AE00002FA0CF223431343C5F888308C4B1A6802
:108AF00042F080521A6008681A68920040F10981B9
:108B0000002010E0414641E6324654E600220121B1
:108B100051E6012165E6DCF80050A5EB0E05642D59
:108B20007FF674AE032005B0BDE8F08FF1453FF449
:108B30007BAED4F870E0D4F870A02EF4407E4AF4F6
:108B4000803AC4F870A0D4F870A02AF4803AC4F82F
:108B500070A0C4F870E0D4F870E01EF0010F3FF48C
:108B600063AEDCF800A041F2883BD4F870E01EF060
:108B7000020F7FF459AEDCF800E0AEEB0A0EDE45E2
:108B8000F3D9CFE7D4F808C02CF4F81C5BE619B988
:108B9000B3F1007F7FF431AFDFF884E1DFF884C107
:108BA000DEF8001021F08061CEF80010DCF8004003
:108BB000DEF800100F0100F19F80B8F1000F2AD0FD
:108BC000C16A41BBDEF884404FF0706898FAA8F99A
:108BD00047F6C07BB9FA89F99BFAABFBBBFA8BFB72
:108BE00098FAA8F84FF0E04AB8FA88F89AFAAAFA80
:108BF0004168BAFA8AFA04F0706401FA0BFB8168E2
:108C000024FA09F401FA0AF104FA08F44BEA010122
:108C10002143CEF884101EB1416BB1F5801F05D001
:108C20000199B9B3816BB1F5800F33D1DFF8F0E072
:108C30004FF0E048DEF8844098FAA8F947F6C07B88
:108C4000B9FA89F99BFAABFB4FF0706ABBFA8BFB60
:108C50009AFAAAFABAFA8AFA98FAA8F8416804F0D5
:108C6000E044B8FA88F801FA0BFBC16824FA09F469
:108C700001FA0AF104FA08F44BEA01012143CEF8A3
:108C80008410DEF88C40C16924F01F0401392143AF
:108C9000CEF88C109C011ED547F6C07393FAA3F34F
:108CA0004FF07061B3FA83F491FAA1F14FF0E04E06
:108CB000B1FA81F19EFAAEFE4368BEFA8EFEA34081
:108CC000C46804FA01F10B43816801FA0EF10B4309
:108CD0001349C1F88430124B196841F08061196062
:108CE000DCF80040196809013FF587AEDCF8001098
:108CF000091B6429F6D915E7DCF80010091B642963
:108D00007FF656AF0EE70A68121B642A7FF67FAE25
:108D100008E70A68121A642A7FF6EEAE02E700BF7F
:108D200000380240502201202DE9F347066905462C
:108D3000C3680C464FF0004901F150071E4001F195
:108D4000380816B902B0BDE8F087B6FA86F329FAFA
:108D500003F21B3BD24316402A61002C42D0042B65
:108D6000EFD8DFE803F03B36302903002369D5F85C
:108D70002CA033B19B6823B11FFA8AF104F10800DB
:108D80009847A36A33B19B6823B11FFA8AF104F1B3
:108D900020009847236C2BB19B681BB11FFA8AF106
:108DA00040469847A36D002BCBD09B68002BC8D0C2
:108DB0001FFA8AF1384604E0236904F10800696B60
:108DC0005B689847BDE7A36A04F12000A96B5B6864
:108DD000F7E7236C4046E96B5B68F2E7A36D296C0B
:108DE0005B68E7E7042B06D8DFE803F00D0B090703
:108DF0000300EB6A0193019BA3E76B6BFAE7AB6B94
:108E0000F8E7EB6BF6E72B6CF4E737B5224B002560
:108E1000224C234AC4F8A43242F20F7304F529709D
:108E2000C4F8B452C4F8B0321E4BC4F8AC52D3F8F4
:108E3000BC31B3FBF2F3013BC4F8A83258F02EF971
:108E4000194B062137201A6C42F020021A641B6C61
:108E500003F020030193019B55F0B0FA134B4FF43C
:108E6000000228465A60D4F8A432DA6842F00102BF
:108E7000DA601A6842F001021A60D4F820320C4A13
:108E8000C3F81052C3F808220A4AC4E98F55C3F840
:108E9000042203B030BD00BF001400405022012066
:108EA00080841E00000001200038024000E100E044
:108EB000405101204041012010B501200C460CF02A
:108EC000ADFC054B122103F11402218002280CBFD6
:108ED0001846104610BD00BFC0010120436BDA697F
:108EE000910670B5044613D5586AE36AC0B2002BE8
:108EF0004AD0216B9847636B1A6822F480721A601B
:108F00009A6822F001029A609A6942F008029A6116
:108F1000636BDA69D20701D501221A62DA69960712
:108F200001D502221A62DA69550701D504221A62B4
:108F3000DA69100701D508221A62DA6911060ED51E
:108F400094F89D20212A0AD0D4E909128A4227D117
:108F50000022A4F886201A6822F080021A60DA69DA
:108F6000520640F19380DA6904F13400196816075B
:108F70009D6821D1960640F18A808D0640F1878058
:108F8000BDE8704057F0CCBEE3696269D054E36934
:108F9000E2680133B3FBF2F102FB1133E361AAE7AC
:108FA000A169895C0132C9B299622169B2FBF1F011
:108FB00001FB1022A262D2E705F0010501F49076D0
:108FC0002E4364D0D60709D5CE0507D501261E62EB
:108FD000D4F8A06046F00106C4F8A060960708D552
:108FE0003DB102261E62D4F8A06046F00406C4F823
:108FF000A060560708D53DB104261E62D4F8A060D3
:1090000046F00206C4F8A06016070AD501F0200653
:10901000354306D008251D62D4F8A0302B43C4F890
:10902000A030D4F8A030002B30D0960603D58D06A2
:1090300001D557F075FED4F8A020636B110703D457
:109040009A6812F040021FD01A6822F490721A60D7
:109050009A6822F001029A60202284F89E209A6881
:10906000520613D59A68D4F8980022F040029A600C
:1090700060B1254B0365FEF7F7FF38B1D4F89800CF
:10908000BDE87040036D1847C4F8A02070BD1606F7
:109090002ED50D062CD594F89D20212AF6D1B4F8B2
:1090A000862092B242B91A6822F080021A601A68C9
:1090B00042F040021A60E9E7E16BD4F88020B1F594
:1090C000805F0FD1616C69B932F8021BC1F30801EE
:1090D0009962C4F88020B4F88630013B9BB2A4F8B2
:1090E0008630D3E7511CC4F8801012789A62F2E7F8
:1090F0005006CBD54A06C9D51A6822F040021A603C
:10910000202384F89D30C1E72381000870B5002634
:109110000E4CD4F8E4329BB9FEE712F8016B013B28
:109120004FF00105C4F8E422636007D157F076FAE6
:109130006368D4F8E4222BB1002DEED0304670BD28
:109140000025F5E7002DE3D0F8E700BF502201200D
:1091500008B5054A0B68C2F8E40253600BB957F032
:109160005DFA002008BD00BF5022012090F8482081
:10917000531C0244DBB280F8483082F8341090F877
:1091800049200AB1132B01D957F028BB70470022A0
:1091900080F8492057F022BBF8B50446D0F83002D9
:1091A000237C93BB4FF400730222812157F0ACFA69
:1091B0004FF4007302220121D4F8300257F0A4FAD0
:1091C000082303228221D4F8300257F09DFA4FF48D
:1091D00007705EF0A3FC0546C4F8180230B3D4F85B
:1091E0001C3200271B689847267CC5F81472C5F806
:1091F00018728EB94FF40073D5F804220121D4F807
:10920000300257F0E9F93046F8BD402302228121AF
:1092100057F07AFA4023CDE74023D5F80422012104
:10922000D4F830023E4657F0D7F9ECE70126EAE7DA
:1092300010B504468121D0F8300257F022FA0121FE
:10924000D4F8300257F01DFA8221D4F8300257F0DA
:1092500018FAD4F8183253B1D4F81C325B68984726
:10926000D4F818025EF062FC0023C4F81832002023
:1092700010BD10B504460121D0F8300257F001FAB4
:109280008121D4F8300257F0FCF9D4F828025EF0BE
:109290004DFC0020C4F8280210BD37B50B780446F9
:1092A0000D4613F060022BD0202A21D1CA884878BD
:1092B0000AB31B06D4F818120AD5D4F81C3201914F
:1092C0009B689847EA880199204657F07CFA0FE09E
:1092D000032381F8012281F80002C4F8F431134617
:1092E000D4F83002C4E942220A46002157F074F94A
:1092F000002003B030BDD4F81C329B689847F7E7D4
:109300004B780A2BF4D101220049DEE738250120F1
:1093100070B50446D0F83002237C93BB4FF4007341
:109320000222012157F0F0F94FF40073022281214B
:10933000D4F8300257F0E8F94FF41B705EF0EEFB02
:109340000646C4F8280218B30025D4F82C3205814B
:10935000A0F85C5228461B6898470121D4F83002D7
:1093600057F091FC8121D4F8300257F08CFCD4F8EE
:1093700030021F2306F50372012157F02DF928460C
:1093800070BD40230222012157F0BEF94023CDE7F2
:109390000120F5E770B5D0F82852044695F8183248
:1093A0004BB9D5F8143233B16B7A23B90121D0F817
:1093B000300257F064FA8121D4F8300257F05FFA96
:1093C0006B7A022B09D105F50372D4F830021F2302
:1093D0000121BDE8704057F0FFB870BD70B50E4B6D
:1093E0000446D0F82852C5F82C32002385F83812EC
:1093F00005F50B722B7281210D23D0F8300257F046
:1094000021F905F50372D4F830021F230121BDE8CC
:10941000704057F0E1B800BF555342532DE9F04179
:109420000B7804460D46D0F8287213F0600635D04C
:10943000202E7ED14A78FE2A07D0FF2A18D0D4F8F1
:109440003002022657F05AFA25E04E88002EF6D157
:10945000CD88012DF3D11A06F1D5D0F82C329B69B5
:1094600098472A4638603946204657F0ACF912E052
:109470004A88002AE3D1CE88002EE0D11B06DED434
:109480004FF4807307F5037201213B811F23D0F84D
:10949000300257F0A1F83046BDE8F08191F8018024
:1094A000B8F10A0F2AD0B8F10B0F2AD0B8F1010F8A
:1094B000F1D10979D0F8300257F0E5FBD4F8300249
:1094C000297957F0DEF895F90430D4F83002002BF2
:1094D000237C1BDAC3B94FF400730222812157F0B9
:1094E00013F9D4F828727B7A022B17D18121D4F892
:1094F000300257F0C4F900237B72CCE70122391DFA
:10950000B3E78B787B60C6E74023E6E723B94FF4E7
:10951000007302224146E2E74023FAE795F904206E
:10952000002AB8DA012BB6D001212046FFF756FFFA
:10953000B1E70026AFE72DE9F743137806460D465D
:1095400017462F2BD0F828423CD8192B08D8032BCC
:109550005ED0122B00F08680002B3ED02022F0E15E
:109560001A3B152BFAD801A252F823F0A396000853
:109570009D9600085D9500085D9500089D96000881
:109580005D9500085D9500085D9500085D950008F3
:10959000B79600085D950008059700085D950008DE
:1095A0005D9500083F9700085D9500081998000830
:1095B0005D9500085D9500085D9500085D950008C3
:1095C000399900085A2BC9D10823B94A6381D2F8C6
:1095D0003F30E360D2F843306BE0D4F81432002B14
:1095E000BCD1D0F82C3208469B689847054650B14C
:1095F0003A220221D6F8280255F05AF805232372A0
:109600004FF0FF3500E06081284603B0BDE8F083ED
:109610001222002104F10C005EF0BAFA702394F8D3
:109620005D2223730C23E37494F85C329A4211D0C8
:1096300004EBC302013392F83C12DBB2A173042B9A
:1096400092F8411208BF0023217692F8402284F854
:109650005C326276122363813B79122B98BF63815F
:109660000025D1E75378DB0715D4D0F82C3201EB75
:10967000C1051279DB6903EB85052B79053393422C
:1096800028BF13466381002BEAD0013B9BB2E95C03
:10969000E2181173F7E70723864DF3E70020608196
:1096A000DEE70823824A6381D2F83730E360D2F8DC
:1096B0003B302361D4E700230DF1020201A9E360EE
:1096C00023616361D0F82C3228465B6898470546D1
:1096D00020B13A220221D6F82802CAE00823E37317
:1096E000019B013B1A0EE37422741A0C62741A0A6D
:1096F000BDF80230A27402225BBAA282E3820C237C
:10970000638181E7D0F82C3204F25E22284604F50A
:1097100018715B68984705460028DAD1D4F86032A2
:109720002082013B1A0EE37322731A0C62731A0A29
:10973000B4F85E32A2735BBA63820823E0E7237A4F
:109740006BBB94F91832002BBFF608AFD0F82C325F
:1097500008469B6898470028BBD1D7F80220D6F866
:10976000280212BAD0F86012C4F86422B7F80730A1
:109770005BBA9BB29F18C4F868328F4277D8022137
:109780002172B4F85E124A434B43C4F86422D4F801
:109790001422C4F86832934201D0202268E04FF4CA
:1097A0000073D6F82C026381D6F82842D0F81090C6
:1097B0002846D4F8687204F10C08B4F85E229F427F
:1097C000D4F8641228BF1F46B7FBF2F3B1FBF2F2E4
:1097D0009BB24146C847002802DA112204217AE7E9
:1097E000BBB2D6F830024246812156F02BFFD4F8A6
:1097F0006432D4F868023B44C51BC4F86432D4F820
:109800003432C4F86852DB1BC4F83432002D7FF4C4
:1098100027AF03232372F7E6237A002B4CD194F968
:109820001832002BFFF69AAED0F82C3208469B680F
:10983000984700287FF44DAFD6F82C322846DB68D5
:109840009847054608B1272244E7D7F80220D6F802
:10985000280212BAD0F86012C4F86422B7F80730B0
:109860005BBA9BB2D718C4F868328F4204D9212260
:10987000052154F01DFFC3E6B4F85E124A434B4382
:10988000C4F86422D4F81422C4F86832934284D114
:10989000B3F5007F4FF0010104F10C0228BF4FF433
:1098A00000732172D6F830029BB256F095FEABE6FB
:1098B000D87E0608087F0608D4F8687204F10C0800
:1098C000B4F85E22B7F5007FD4F86412D0F82C0209
:1098D00028BF4FF40077D0F814902846B7FBF2F376
:1098E000B1FBF2F29BB24146C847002801DA0322DD
:1098F00074E7D4F86432D4F868523B44ED1BC4F8E2
:109900006432D4F83432C4F86852DB1BC4F8343201
:1099100025B929463046FFF761FD75E6B5F5007FAC
:1099200042464FF00101D6F8300228BF4FF40075CF
:10993000ABB256F051FE93E6787810F0020003D0F7
:1099400024220521204694E7D4F86422B4F8683232
:109950001344D4F8602293427FF6A1AE2122F0E7AF
:10996000D0F8281210B50B7A0446022B07D0033B1F
:10997000012B02D80021FFF731FD002010BD01F2BC
:109980001B2291F81912FFF7D6FD0028F5DA012104
:109990002046F0E770B5D0F828420546267A1EB179
:1099A000012E55D0002070BDD4F81032C4F83032EA
:1099B000D4F81432C4F83432D0F83032B3F82C3240
:1099C0001F2B0DD1D4F80C22264B9A4208D194F8C3
:1099D0001912012904D894F81A32013B0F2B0AD925
:1099E00020220521204654F063FE0223637228469C
:1099F000FFF7D0FCD6E704F21B22FFF79CFD0028FE
:109A0000237A06DA052BF2D101212846FFF7E6FC7E
:109A1000C8E7013B022BC5D961890029F5D0D5F8EB
:109A20002832D3F8142283F83862914228BF1146B5
:109A3000D3F83422521AC3F8342204221A728BB299
:109A400004F10C028121D5F8300256F0FBFDA9E7A4
:109A500004F21B2294F81912FFF76DFD0028A1DA19
:109A6000D2E700BF5553424308B520B9034854F02C
:109A70006BF9034808BD0348F9E700BF440F070826
:109A80003C250120650F0708024808B554F05CF931
:109A9000014808BD860F07083C250120024808B58B
:109AA00054F052F9014808BD8B0F07083C250120EE
:109AB000024808B554F048F9014808BD960F070858
:109AC0003C250120064BD3F8A0321A79022A05D191
:109AD0009A68920702D5586956F060BA704700BF7D
:109AE0005022012030B40E4A14240E49D2F8A002AC
:109AF0000379022B0DD190F910306343CB589D6848
:109B000015F4C05F07D19B681D0604D483689B07CA
:109B100003D430BC704700BFE8E730BC08F0F6B9AA
:109B2000502201200000012073B5441C0025094E7D
:109B3000D6F8A002012300220DF1070156F036FAF3
:109B40009DF80700FF2802D10135A542F0D102B0EF
:109B500070BD00BF5022012037B504460820019196
:109B6000FFF7E2FFFF2813D0FE2813D10A4D002291
:109B7000019B2146D5F8A00256F018FA0022D5F82C
:109B8000A0020223114656F011FA002003B030BDA6
:109B90000120FBE70220F9E75022012037B54FF6FC
:109BA000FF53104D002401AAD5F8A0022146ADF8BC
:109BB00004300223C5F86C4256F0F8F90120FFF793
:109BC000B3FFFF2805D10423022085F8703203B0CB
:109BD00030BD0923204685F87032D5F8EC33C5F83E
:109BE0006032F4E75022012040F0400313B58DF8B5
:109BF00000300B0E04468DF804108DF801300B0C6C
:109C00008DF802300B0A8DF8033095238DF805305E
:109C100056F0F2F900B964B9074806236A460021F4
:109C2000D0F8A00256F0C2F90820FFF77DFF02B07D
:109C300010BDFF20FBE700BF502201202DE9F041BD
:109C4000174C1E460546884694F870321746042B7A
:109C500017D1FFF737FF94F86632DBB9690211209C
:109C6000FFF7C2FFC0B90523012084F87032D4F891
:109C7000EC33C4E99385C4E99676C4F86032BDE854
:109C8000F081082B01D00020F9E7FFF787FF0228B9
:109C9000F9D1DEE72946E2E7FFF724FFF3E700BF4B
:109CA0005022012070B5274C0C23002232210220C3
:109CB00007F031FFC4F8A00210B984F8700270BD3B
:109CC000002108F0A7F84FF47A700CF0BCFFD4F82C
:109CD000A0020379022B04D183689A0701D508F00A
:109CE00015F900220A23D4F8A0021146164D56F0A9
:109CF0005DF9D4F8A002154A14210379022B0AD188
:109D000090F910304B43D3589E6816F4C05F0BD1C6
:109D10009B681B0608D4D4F8EC33C4F860320123E6
:109D200084F8703200230AE0013DE9D107F0E6FE35
:109D300094F86432C4F8A052013384F8705284F865
:109D40006432BCE750220120A186010000000120FE
:109D500038B5134C0023A07BE0B125688D4219D1A2
:109D6000104C03F581751AB904EB0514A27138BDC6
:109D700004F1180101EB43239A4209D1831E584292
:109D8000584156F035FB012304EB0514A371EEE7AF
:109D90000020F6E701331034082BDCD1E7E700BFE1
:109DA000343F01201C2F0120164838B5002300F154
:109DB000180480F8A03025688D421ED1A57B032DA4
:109DC0001BD1114C03F581754AB9042304EB05142A
:109DD000A371D0F89C300133C0F89C3038BD04F139
:109DE000180004EB051400EB4320131A58425841A5
:109DF00056F0FEFA0123A371F0E701331034082B6B
:109E0000D9D1EBE71C3F01201C2F012082B0054A6D
:109E100001901068136801991B1A8B42FAD302B0A3
:109E2000704700BF50220120002808DB42090123AF
:109E300000F01F0003FA00F0014B43F822007047C6
:109E400000E100E02DE9F04F002385B0DFF8B88194
:109E50006B4ADFF8B89101270C689F4007EA0405B8
:109E600037EA040440F0B6804C6824F0100ABAF1D6
:109E7000020F16D14FEAD30E03F0070B4FF00F0C71
:109E800000EB8E0E4FEA8B0BDEF820600CFA0BFC19
:109E900026EA0C0C0E6906FA0BF646EA0C06CEF81A
:109EA00020604FEA430E4FF0030CD0F800B00AF1E7
:109EB000FF3A0CFA0EFCBAF1010F6FEA0C062BEA1E
:109EC0000C0B04F0030C01960CFA0EFC4CEA0B0C84
:109ED000C0F800C015D8D0F808C006EA0C0CCE684F
:109EE00006FA0EFA4AEA0C0CC0F808C0D0F804C012
:109EF0002CEA0707C4F3001C0CFA03FC4CEA070722
:109F00004760C768019E37408E6806FA0EF63E43EA
:109F1000C660E6005ED5D8F8446023F0030703F07E
:109F2000030C4FF00F0E46F4804607F180474FEACE
:109F30008C0CC8F8446007F59C37D8F8446006F4E8
:109F400080460396039E0EFA0CF6D7F808A02AEA7C
:109F5000060E2C4EB04244D006F58066B04242D088
:109F600006F58066B04240D006F58066B0423ED02D
:109F700006F58066B0423CD048453CD006F5006608
:109F8000B0423AD006F58066B0420CBF07260826DC
:109F900006FA0CF614F4803F46EA0E06BE606FEA3D
:109FA000050716680CBF3E402E4314F4003F1660B0
:109FB00056680CBF3E402E4314F4801F56609668CE
:109FC0000CBF3E402E43A4029660D66854BF3E406C
:109FD0002E43D6600133102B7FF43DAF05B0BDE8B2
:109FE000F08F0026D4E70126D2E70226D0E7032629
:109FF000CEE70426CCE70526CAE70626C8E700BF59
:10A00000003C0140000002400038024000140240C1
:10A0100003689A69910701D500229A629A69D2076A
:10A0200003D49A6942F001029A61704770B590F8C2
:10A03000403004460D461646012B00F018810123DE
:10A0400080F84030CB0640F19780D00640F19480F4
:10A05000638D9BB2002B40F08780E36AB3F1007FF1
:10A0600003D0E36AB3F1007F6AD194F84130282B22
:10A0700066D129462046FEF7B0FAAB065CD5B60697
:10A080005AD52368202207212046DA610822DA61A6
:10A0900057F094F8236820465A6842F400425A6008
:10A0A0005A6822F0FF7222F48B3222F4FF7222F0FF
:10A0B00001025A60FFF7ACFF22681368580402D40B
:10A0C0001368190409D594F84130212B0CBFA36BF8
:10A0D000E36B1B685B689BB26385638D9BB21BB1AE
:10A0E000636C43F0040363646B0710D5636A526AC0
:10A0F000591C61621A70238D4BB1013B2385638D1E
:10A10000013B9BB26385636C43F0040363640023EB
:10A110002363636384F84230636C002B00F09A8001
:10A12000616C2046FEF786FA94F84130282B03D163
:10A1300029462046FEF751FA002084F8400070BD01
:10A14000E26A236812F5803F0BD094F84120292A57
:10A1500007D110222046DA61FFF75AFFFEF71EFAF8
:10A160008BE71022DA6188E723681022DA61636CDA
:10A1700043F00403636480E769071DD572071BD5AC
:10A18000638D9BB263B123685A6A636A591C61622A
:10A190001A70238D013B2385638D013B9BB2638540
:10A1A000638D9BB2002B7FF468AFE36A13F5803FA9
:10A1B0003FF463AF2046D1E72B072CD530072AD5D3
:10A1C00094F84130226803F02803282B20D19369AA
:10A1D00091699368D068E068022813D1C3F3C21371
:10A1E00083EA114313F006030CD1A16C0131A16481
:10A1F000A16C02297FF441AF0821A364D16184F8E6
:10A2000040303AE70421204656F0D8FF0023F6E715
:10A210000823D361FAE7A9077FF52FAFB2077FF5CF
:10A220002CAF638D9BB26BB1636A5A1C6262226869
:10A230001B789362638D013B9BB26385238D013B49
:10A2400023851AE7E36AB3F1807FB3D0E36A002B7A
:10A25000B0D012E7E36A13F5803F05D0054BE36207
:10A26000202384F8413067E794F84130F8E7022072
:10A2700065E700BF0000FFFF194B9A6802F00C026F
:10A28000042A28D0082A28D15A68596802F03F02C7
:10A29000586811F4800F47F6C07191FAA1F3B3FA30
:10A2A00083F300EA010020FA03F014BF0D4B0E4BBC
:10A2B000B3FBF2F20A4B50434FF440325B6892FA20
:10A2C000A2F2B2FA82F203F44033D34001335B00CE
:10A2D000B0FBF3F07047034870470348704700BF76
:10A2E0000038024000127A000024F400094B4FF4B9
:10A2F000E0529B6892FAA2F2B2FA82F203F4E053BF
:10A30000D340054A1344054A93F84730D2F8BC01BC
:10A31000D840704700380240D87E0608000001206F
:10A32000094B4FF460429B6892FAA2F2B2FA82F2B1
:10A3300003F46043D340054A1344054A93F8473079
:10A34000D2F8BC01D840704700380240D87E0608D9
:10A350000000012038B5C2690446036881680069BD
:10A360001D68014360690143A14811432840256AE3
:10A370000143E0681960596821F440510143596074
:10A38000A1699868294320F4306001439960994994
:10A390008B421FD101F59431D1F8901001F00301E7
:10A3A0000139022900F205819348014491F84F10C8
:10A3B000B2F5004F40F0AE80082900F2A880DFE837
:10A3C00011F0E600FB000101A6000D01A600A600A9
:10A3D000A600350089498B420AD101F5FA31D1F83E
:10A3E0009000854900F00C00014491F85210DFE71D
:10A3F00083498B421FD101F5F831D1F8901001F05B
:10A400003001202900F0DB800AD8002900F0BC8050
:10A41000102900F0E080B2F5004F78D00120C7E0AD
:10A420003029F8D1B2F5004F40F0A9806268530896
:10A4300003F58033CCE073498B4210D101F5F6313E
:10A44000D1F8901001F0C001802900F0B88004D844
:10A45000002900F099804029DBE7C029E1E76A493B
:10A460008B4213D101F5F431D1F8901001F4407111
:10A47000B1F5007F00F0A38005D8002900F08480AA
:10A48000B1F5807FC5E7B1F5407FCAE75F498B42F0
:10A4900013D101F59231D1F8901001F44061B1F57A
:10A4A000006F00F08C8005D8002900F08280B1F5A3
:10A4B000806FAEE7B1F5406FB3E755498B4211D1DC
:10A4C00001F5E031D1F8901001F44051B1F5005F91
:10A4D00075D004D8002957D0B1F5805F99E7B1F560
:10A4E000405F9EE74B498B4295D101F5DE31D1F8B3
:10A4F000901001F44041B1F5004F60D004D800291C
:10A5000042D0B1F5804F84E7B1F5404F89E7012093
:10A51000002346E0082981D801A252F821F000BFAB
:10A5200045A500085DA5000863A500081DA4000856
:10A5300079A500081DA400081DA400081DA400089A
:10A540007FA50008FFF7D2FED4E9002300EB5300FB
:10A55000B0FBF3F080B2D060002029E0FFF7E0FE0E
:10A56000F2E761684A0802F5740202F51052B2FB84
:10A57000F1F292B2DA60EFE7FFF77EFEE4E761689E
:10A580004A0802F50042F2E7B2F5004FDAD1FFF7D0
:10A59000ADFE63685A0802EB4000B0FBF3F39BB2D8
:10A5A000002023F00F02C3F3420321681343CB6062
:10A5B00038BDB2F5004FD1D1FFF7B2FEE9E7B2F5F1
:10A5C000004FCED16268530803F1F47303F5904352
:10A5D000B3FBF2F3E3E7B2F5004FCDD1FFF74CFE4A
:10A5E00061684A0802EB4003B3FBF1F3D7E700BF11
:10A5F000F369FFEF00100140D87E060800440040D8
:10A6000000480040004C0040005000400014014051
:10A6100000780040007C0040A348A44AA449121AD4
:10A6200070B5A4B05DF06AF8A24A0020D2F8883074
:10A6300043F47003C2F888309F4B196841F0010160
:10A6400019609860196821F0847121F480311960D3
:10A650009A495960196821F4802119609849D86095
:10A660009160BFF34F8FBFF36F8FC2F85002BFF3FB
:10A670004F8FBFF36F8F516941F400315161BFF3C8
:10A680004F8FBFF36F8F1A6C42F080521A641A6CAE
:10A6900002F080520292029A8A4A116841F44041C3
:10A6A0001160126802F440420192019A9A6802F025
:10A6B0000C02042A07D09A6802F00C02082A65D11D
:10A6C0005A68520262D57C4B1B687B4A936803F040
:10A6D0000C03082B68D013687B4C23F08073136045
:10A6E000216813689D0160D447F6C07393FAA3F301
:10A6F000B3FA83F04FF4403393FAA3F34FF0706151
:10A7000091FAA1F14FF4D873B1FA81F18340092095
:10A7100000FA01F10B4343F0015343F00803536087
:10A72000136843F080731360634B21681A689001CB
:10A7300040D51A6C42F080521A641B6C03F08053AF
:10A740000393039B5F4B1A6842F480321A602168BE
:10A750005A68D20333D51A6842F400321A60594A53
:10A76000216853689B0330D54FF400134FF4C07C2D
:10A7700004A804934FF0006321930723CDE908C395
:10A7800003230A93FDF7EEFF28B3FEE71A684A4950
:10A7900042F480321A604C4A10680B689E0394D4CD
:10A7A00013681B1A642BF8D9FEE723685B1A022B87
:10A7B00097D9F9E72268521A022AB7D9F4E7226832
:10A7C000521AB2F57A7FC3D9FEE723685B1AB3F554
:10A7D0007A7FC6D9F8E73D4A136803F00F03062BCA
:10A7E00008D9354B9A6822F0F0029A601A689001F5
:10A7F0000CD4FEE7136823F00F0343F00703136044
:10A80000136803F00F03072BF3D1EAE79A6841F2CC
:10A81000883022F0030242F002029A6021689A68AE
:10A8200002F00C02082A39D1284A1368190755D4B6
:10A83000214CA36823F4E05343F4A053A360A3681E
:10A8400023F4604343F40043A360FFF715FDA368BE
:10A85000F02292FAA2F2B2FA82F203F0F0031C4E56
:10A86000D3401C4D334493F85F30D840C5F8BC0149
:10A8700053F0D0FD184B04A804930023CDE9133303
:10A88000CDE91533CDE91733CDE91933CDE91B33C4
:10A89000CDE91D33FDF766FF60B3FEE72268521A6B
:10A8A0008242BCD9A5E700BF00000000181B0000D1
:10A8B000FC6D070800ED00E0003802401030002475
:10A8C000000000080070004050220120003C0240BF
:10A8D000D87E060800000120C0FF0300136823F0A3
:10A8E0000F0343F007031360136803F00F03072BF4
:10A8F0009ED07EE7D4F88C3023F08073C4F88C307F
:10A90000D4F88C3043F08073C4F88C30A36803F023
:10A910000C03042B14D0082B14D0184BC5F8BC31F1
:10A92000174B9B68C3F303131E44D5F8BC3196F84C
:10A930005F20D340134A9342C5F8BC311BD0FEE7D9
:10A94000114BEBE76368626813F4800F636802F0F1
:10A950003F0218BF0C49C3F3881308BF0749B1FB76
:10A96000F2F25343064A5268C2F3014201325200E6
:10A97000B3FBF2F3D2E724B070BD00BF0024F400B3
:10A980000038024000E6DF0C00127A0003682DE96F
:10A99000F041C3F30D04054688464D4F002C62D1AB
:10A9A0004C4A93421ED302F58042934219D302F5DA
:10A9B000804293421ED3484A93421DD902F5803209
:10A9C00093421BD902F50032934219D902F50032A5
:10A9D000934217D902F50032934215D905200CF0A5
:10A9E0007FF9012497F80434012B0FD14FF0FF3089
:10A9F000BDE8F0810224F5E70324F3E70424F1E73E
:10AA00000524EFE70624EDE70724EBE7012387F8A9
:10AA1000043453F07DFC68BB304E336923F440733B
:10AA20003361336943F400733361336923F0F8030E
:10AA30003361782393FAA3F3B3FA83F332699C402A
:10AA4000144344F002043461336943F480333361C6
:10AA5000BFF34F8F53F05CFC336923F07A0333610B
:10AA600040B987F8040497F80434012B06D16FF03D
:10AA70000100BDE7002387F80434B7E701232E68FF
:10AA8000D8F8008087F8043453F042FCB0B9134C76
:10AA9000236923F440732361236943F40073236122
:10AAA000236943F001032361C6F80080BFF34F8F91
:10AAB00053F02EFC236923F001032361002387F860
:10AAC00004340028D3D12B6804332B6090E700BFF7
:10AAD0005022012000400008FFFF0008003C024017
:10AAE0000148FDF70FBE00BF602601200148FDF7B9
:10AAF000CDBA00BF602601200148FDF703BE00BFAC
:10AB0000B02601200148FDF7C1BA00BFB0260120E0
:10AB10000148FDF7F7BD00BF002701200148FDF700
:10AB2000B5BA00BF002701202DE9F843904F0C264D
:10AB3000054606FB0076D6F8E831002B00F01281BE
:10AB400096F8EE0153F042FB96F8EC0109F038FF5D
:10AB5000044696F8ED0109F033FF6B1C0646DBB2A4
:10AB60001CB140F60B122372E2801EB140F60B229C
:10AB70003372F28020464FF0090909F0D5FE3046C5
:10AB800009F0D2FE1121204609F0D9FE11213046EC
:10AB900009F0D5FE4FF0650803E0052000210CF018
:10ABA00041F8204609F0AFFE10B9B8F10108F4D120
:10ABB000204609F0BEFE002105200CF033F82046A7
:10ABC00009F0B2FE052000210CF02CF8B9F10109C2
:10ABD000E0D120464FF00C0809F0ABFE0021052023
:10ABE00008FB05780CF01EF8304609F0A2FE0021A3
:10ABF00005200CF017F8204609F096FE00210520EC
:10AC00000CF010F8304609F08FFE204698F8F2213B
:10AC10003E2109F0B5FE50243046564E98F8F221F8
:10AC20003E2109F0ADFE04FB0564D8F8E831C4F814
:10AC30001034FFF75BFB98F8EF31022B00F09480A3
:10AC4000032B00F09380012B14BF4FF4C8714FF415
:10AC5000487153F033FA50220021C4F8140402FB67
:10AC600005630120C3F81814C3F82014C3F8241492
:10AC7000C3F82C14C3F8301493F85114C3F81C040F
:10AC800001F0FF0009B983F8500402FB0562242497
:10AC9000D2F8103482F85144196821F0010119608A
:10ACA000D2F8141421F070611961996821F40041FF
:10ACB00099604FF400419960596841F0007141F486
:10ACC00000415960D96821F40041D960D2F82814B4
:10ACD0000902D96000211960186840F0010018606D
:10ACE0002020C2F8541482F85104C2F8401482F8AB
:10ACF000521492F8510420285FFA80FC17D192F880
:10AD00005004012813D082F85144186820F0010043
:10AD10001860186820F48050186018681860186867
:10AD200040F00100186082F851C482F850140C24DD
:10AD3000022104FB057494F9F10153F03FFB94F9EF
:10AD4000F101FFF771F8022194F9F00153F036FB9D
:10AD500094F9F001FFF768F85020012300FB056526
:10AD600085F80C34BDE8F883642172E7C82170E7E8
:10AD700000000120502201202DE9F04F984685B0B7
:10AD8000431C064689469DF83C50039200F0208102
:10AD9000AA4F502303FB007393F80CB4BBF1000FD0
:10ADA0006ED0FF2A03D0B8F1000F40F0BE80002D16
:10ADB00000F0BB805024744307EB040A9AF8513426
:10ADC000202B40F0FC809AF85034012B00F0F780E3
:10ADD0009B4B0122D7F800B04FF400411C448AF885
:10ADE00050241923CDF800B02046FDF769F900285A
:10ADF00040F0E58021231FFA88F809FA02F9CAF821
:10AE000044048AF8513410238AF852340E9BCAF84D
:10AE10005404CAF83434AAF83A84BAF83A349BB2E3
:10AE2000FF2B31D94FF40053FF22AAF838240093A6
:10AE30004FF080734FF050084946204608FB0678D3
:10AE4000FDF75CF9B8F83A34594620469BB23BBB53
:10AE500053F016FA38BBD8F810342021AB46D9612C
:10AE60005A6822F0FF7222F48B3222F4FF7222F031
:10AE700001025A6088F8511488F8500488F8520486
:10AE8000584605B0BDE8F08FBAF83A244FF40053A5
:10AE900092B2AAF83824D2B200934FF00073C9E7F7
:10AEA00053F012FA10B1D8F8543488E0D8F834349A
:10AEB0005A1CC8F83424D8F810241B789362B8F8C8
:10AEC0003824B8F83A34013A013B92B29BB2A8F860
:10AED0003824A8F83A34002AB4D1B8F83A349BB2EE
:10AEE000002BAFD00A2380212046CDF800B0FDF71B
:10AEF000E7F8002863D1B8F83A349BB2FF2B0AD99F
:10AF0000FF224FF08073A8F838240090494620466D
:10AF1000FDF7F4F896E7B8F83A244FF0007392B2D0
:10AF2000A8F83824D2B20090F0E7502474433D19B9
:10AF300095F85134202B42D1B8F1000F3FD095F84D
:10AF40005034012B3BD03E4B0122D7F800A04FF4E8
:10AF500000411C4485F850241923CDF800A0204658
:10AF6000FDF7AEF858BB212309FA02F91FFA88F859
:10AF7000C5F8440485F851344023494685F85234D5
:10AF80000E9BC5F854042046C5F834344FF40053E2
:10AF9000A5F83A8400934FF08073FDF7AFF851465F
:10AFA000204653F091F90246A8B1D5F85434502305
:10AFB00003FB0673D3F85424002283F85024B7F817
:10AFC000FC34304601339BB2A7F8FC34FFF7ACFDEC
:10AFD0004FF0000B54E7D5F81034204603999962DE
:10AFE0000A238021CDF800A0FDF76AF80028DED101
:10AFF000B5F83A349BB2FF2B09D8B5F83A244FF094
:10B00000007392B2A5F83824D2B2009005E0FF2276
:10B010004FF08073A5F8382400904FF0500849464F
:10B02000204608FB0675FDF769F85146204653F0A7
:10B030004BF938B108FB067835E700BF50220120F4
:10B0400060260120D5F834345A1CC5F83424D5F8CC
:10B0500010241B789362B5F83824B5F83A34013AD5
:10B06000013B92B29BB2A5F83824A5F83A34DAB97C
:10B07000B5F83A349BB2BBB10A2380212046CDF803
:10B0800000A0FDF71DF8002899D1B5F83A349BB21D
:10B09000FF2B16D9FF224FF08073A5F838240090BB
:10B0A00049462046FDF72AF8B5F83A349BB2002B02
:10B0B000BBD15146204653F0E3F860B1D5F8543483
:10B0C0007DE7B5F83A244FF0007392B2A5F8382422
:10B0D000D2B20090E4E7D5F810342021D9615A6843
:10B0E00022F0FF7222F48B3222F4FF7222F001026E
:10B0F0005A6085F8511485F8500485F85204BFE66B
:10B100002DE9F04FB0F1FF3F85B0804693469DF8A2
:10B110003C9000F09A805024B74F44433D1995F875
:10B120000CA4BAF1000F00F0FB809BB2FF2A05F5DA
:10B1300082644FEA4106039340F0F680B9F1000FB4
:10B1400000F0F28095F85134202B75D195F85034E9
:10B15000012B71D00122D7F800A019234FF4004130
:10B1600085F850242046CDF800A0FCF7A9FF002860
:10B1700062D12223C5F8440485F85134102385F8A0
:10B1800052340E9BC5F85404C5F83434039BA5F81B
:10B190003A34B5F83A349BB2FF2B1DD94FF4105313
:10B1A000A5F838B45A4600934FF0807350253146C5
:10B1B000204605FB0875FCF7A1FFB5F83A349BB2B1
:10B1C000002B56D15146204653F05AF8002800F083
:10B1D0009280D5F854342FE0B5F83A244FF4105348
:10B1E00092B2A5F83824D2B200934FF00073DDE795
:10B1F0005146204653F00CF8C8B9D5F810349A6976
:10B2000012F0200224D02021D9615A6822F0FF7266
:10B2100022F48B3222F4FF7222F001025A60C5F848
:10B22000540485F8500485F8511485F852045023CD
:10B2300003FB0873D3F85434B7F8FC3440460133A9
:10B240009BB2A7F8FC34FFF76FFC4FF0000A67E0F1
:10B250003B68A3EB0A030A2B0BD9D5F8543485F8C5
:10B26000502443F02003C5F85434202385F851348A
:10B27000DDE7D5F810349A695207B9D55A6AD5F87E
:10B280003434591CC5F834141A70B5F83824B5F89C
:10B290003A34013A013B92B29BB2A5F83824A5F8A2
:10B2A0003A34002A89D1B5F83A349BB2002B84D0C5
:10B2B0000A2380212046CDF800A0FCF701FF0028DA
:10B2C000BAD1B5F83A349BB2FF2B0AD9FF224FF01E
:10B2D0008073A5F83824009031462046FCF70EFF15
:10B2E0006BE7B5F83A244FF0007392B2A5F8382412
:10B2F000D2B20090F0E7D5F810342021CA46D961C7
:10B300005A6822F0FF7222F48B3222F4FF7222F08C
:10B3100001025A6085F8511485F8500485F85204EA
:10B32000504605B0BDE8F08F502505FB087595F82F
:10B330005134202B80D10E9B002B3FF47DAF95F82C
:10B340005034012B3FF478AF0122D7F80090192335
:10B350004FF4004185F850242046CDF80090FCF7CA
:10B36000AFFE00287FF468AF2223C5F844043146BD
:10B3700085F851344FF0400385F852340E9BC5F8E0
:10B380005404C5F83434039BA5F83A344FF4005301
:10B39000009303462046FCF7B1FE4946204652F092
:10B3A00093FF024650B1D5F85434502303FB087381
:10B3B000D3F85424002283F850243DE7D5F8103404
:10B3C00040212046C3F828B00A23CDF80090FCF7AE
:10B3D00077FE0028E9D1B5F83A349BB2FF2B0DD89F
:10B3E000B5F83A244FF4105392B2A5F83824D2B2EB
:10B3F00000934FF0007309E0502201204FF41053E6
:10B40000FF22A5F8382400934FF080735025314671
:10B41000204605FB0875FCF771FE0A230022042173
:10B420002046CDF80090FCF74BFE00287FF404AFD7
:10B43000D5F81034596AD5F83434581CC5F834049A
:10B440001970B5F83834B5F83A14013B01399BB29C
:10B4500089B2A5F83834A5F83A14E3B9B5F83A3406
:10B460009BB2C3B10A2380212046CDF80090FCF79F
:10B4700027FE00287FF4E0AEB5F83A349BB2FF2BEC
:10B480002AD9FF224FF08073A5F838240090314666
:10B490002046FCF733FEB5F83A349BB2002BBCD102
:10B4A0004946204652F0ECFE00287FF492AED5F8D3
:10B4B00010342021D9615A6822F0FF7222F48B32B5
:10B4C00022F4FF7222F001025A6085F8511485F8C7
:10B4D000500485F8520423E7B5F83A244FF000737E
:10B4E00092B2A5F83824D2B20090D0E70348D0F841
:10B4F000183213B100F5037018477047000001209F
:10B500000348D0F8383213B100F50B701847704774
:10B51000000001200348D0F8583213B100F5137031
:10B5200018477047000001200348D0F8783213B163
:10B5300000F51B7018477047000001200348D0F841
:10B54000983213B100F523701847704700000120AE
:10B550000348D0F8B83213B100F52B701847704784
:10B56000000001200348D0F8D83213B100F5337041
:10B5700018477047000001200348D0F8F83213B193
:10B5800000F53B7018477047000001200348D0F8D1
:10B59000183313B100F543701847704700000120BD
:10B5A0000348D0F8383313B100F54B701847704793
:10B5B000000001200348D0F8583313B100F5537050
:10B5C00018477047000001200348D0F8783313B1C2
:10B5D00000F55B7018477047000001200348D0F861
:10B5E000983313B100F563701847704700000120CD
:10B5F0000348D0F8B83313B100F56B7018477047A3
:10B60000000001200348D0F8D83313B100F573705F
:10B6100018477047000001200348D0F8F83313B1F1
:10B6200000F57B70184770470000012038B544686A
:10B6300044F4805444603BB9012004E0013C05D14E
:10B64000FCF7CBFD002038BD40F2E9348568AD073A
:10B65000F4D56AB112F8014B047340F2E9348568FD
:10B66000ED0707D5C46809B101F8014B013BE2E7DA
:10B67000FF24F1E7013CF2D1E2E70023054A52F84A
:10B680003310814201D1D8B2704701330E2BF6D16D
:10B69000FE207047487F06082DE9F04707460068FE
:10B6A000FFF7EBFF0D28054608DD0024274A00219F
:10B6B000052005F0EBFB2046BDE8F087DFF8989009
:10B6C0004FEA800809EB800ADAF800655EBB0721C3
:10B6D000682005F0A9FC0446CAF8000528B901460F
:10B6E0001B4A052005F0D2FBE5E7314668225CF0F5
:10B6F0004FFA18482AB2DAF8004500F1700300EB5F
:10B70000C500A46003EBC203006F24622360A4633E
:10B710002465FFF7B2FF0D289EBF09F5A76600B2AA
:10B7200006EB80166660C844787918210023D8F8A3
:10B73000004501FB0042D760C2E9043300FB01125F
:10B74000A35401FB00440834B5E700BFA40F070869
:10B75000C90F0708D87E06085022012070B50028BE
:10B7600029D04C6854B9036842685B685679022254
:10B770001D68B240EB6823EA0203EB608A6832B9C5
:10B7800003685B681D68EB6823F00103EB60816070
:10B790004CB103685B6819684368CC685D79022323
:10B7A000AB402343CB6032B103685B681A68D3684F
:10B7B00043F00103D36070BD0A4B30B51A46002434
:10B7C0001D79854208D1DD68294203D0142000FB91
:10B7D000042030BD0029F9D0013414330B2CEFD1F3
:10B7E0000020F6E70C040120036807EE902A70B5EC
:10B7F000D3E900340E461D682368AB4279D03D4B37
:10B80000F8EE677A2560013E93ED6F7AB6B2B8EE36
:10B81000477A87EE270ADFED387A30EE270A59F0AB
:10B820009BF800230138E660A36060602046C4E90D
:10B8300004338023A36155F031FC304B9D4216D078
:10B84000B5F1804F13D0A3F57C439D420FD003F593
:10B8500080639D420BD003F580639D4207D003F5C2
:10B8600078439D4203D003F570539D4241D194F833
:10B870003C30012B3DD00223214A84F83D3023681F
:10B8800099680A409A609A6822F4803222F007028E
:10B890009A60012284F83D20002284F83C20174A57
:10B8A000954212D0B5F1804F0FD0A2F57C4295425F
:10B8B0000BD002F58062954207D002F58062954276
:10B8C00003D002F57842954213D10C485A6883425E
:10B8D000996803D000F58060834201D122F47002A0
:10B8E00022F0700221F080015A609960002384F8F0
:10B8F0003C3070BD000001200AD7233C000001400D
:10B900008800FEFF43680068F0B540685C799A796A
:10B91000974B12F00202234490F83C400EBF1546AC
:10B9200002220825012C93F8E03017D001240C2BBB
:10B9300080F83C404FF0020480F83D4000F0C680A3
:10B940000DD8042B65D0082B00F09080002B32D04E
:10B95000012380F83D30002380F83C30F0BD102BEF
:10B9600000F0DB80142BF3D103681C6A24F48014EC
:10B970001C621D6A5E6825F400155C6D45EA025282
:10B9800024F080747B4D24F4E044AB4244F4C04482
:10B9900003D005F58065AB4201D146F480265E6098
:10B9A0005C65D9651A625A6D42F400625A655A6D37
:10B9B00022F48062D7E003681C6A24F001041C6250
:10B9C0001C6A5F6824F002049E69224326F48036D4
:10B9D000684C26F07306A34246F0600603D004F5D7
:10B9E0008064A34206D122F0080247F440772A433C
:10B9F00022F004025F609E6159631A629A6942F004
:10BA000008029A619A6922F004029A619A699A611D
:10BA10009EE703681C6A24F010041C621C6A5F68BD
:10BA200024F020049E6944EA021226F08076514CEC
:10BA300026F4E646A34246F4C04603D004F58064EB
:10BA4000A34207D122F0800247F4406742EA051280
:10BA500022F040025F609E6199631A629A6942F423
:10BA600000629A619A6922F48062CEE703681C6AD8
:10BA700024F480741C621C6A5F6824F40074DE691C
:10BA800044EA022226F480363A4C26F07306A3429A
:10BA900046F0600603D004F58064A34207D122F487
:10BAA000006247F4405742EA052222F480625F6058
:10BAB000DE61D9631A62DA6942F00802DA61DA6992
:10BAC00022F00402DA61DA69DA6141E703681C6A8C
:10BAD00024F480541C621D6A5E6825F40055DC69FC
:10BAE00045EA023224F08074224D24F4E644AB424D
:10BAF00044F4C04403D005F58065AB4201D146F45F
:10BB000080465E60DC6119641A62DA6942F40062A0
:10BB1000DA61DA6922F48062D4E703681C6A24F4EB
:10BB200080341C621D6A5E6825F400355C6D45EA50
:10BB3000024224F480340F4D24F07004AB4244F0F0
:10BB4000600403D005F58065AB4201D146F4803630
:10BB50005E605C6599651A625A6D42F008025A652A
:10BB60005A6D22F004025A655A6D5A65F0E600BF1C
:10BB7000D87E06080000014043685A79032A0FD88E
:10BB8000DFE802F00205080B1868343070471868C7
:10BB90003830704718683C3070471868403070473C
:10BBA00000207047D0E9003251795868054B0B44AA
:10BBB00093F8E01093795B0701D555F0E4B855F0A0
:10BBC000F6B800BFD87E060842681269F8B5C2F31D
:10BBD0000322264B044603EB82029668C26855682E
:10BBE000EFF31187102282F312884068D0F800C06A
:10BBF0004079DCF80C2003EB4000008D00F4F0509D
:10BC000022EA0002985DCCF80C202A5822F00102AA
:10BC10002A50E2681069D2F804C020221F2821D9D6
:10BC200020388240CCF80C20FAB282F31188985D5B
:10BC30006769284443681B0C1B040B434360204680
:10BC4000FFF79AFF0A4B9B5DEA18D7609060EA58AD
:10BC500042F01002EA50EA5842F00102EA50012391
:10BC60002374F8BD8240CCF80820DDE7D87E0608B2
:10BC7000D87E06080268137E012B26D10223137694
:10BC80004FF4007392F83010012904D1022143F4DB
:10BC9000806382F8301092F84810012904D1022103
:10BCA00043F4006382F8481092F8601001290ED125
:10BCB000022143F4805382F8601012680021126858
:10BCC0005162D1680B43D36003E00023DAE7002B15
:10BCD000F3D17047024B0348D3F80015FDF724B8A1
:10BCE000502201200000014010B5064C0648D4F84F
:10BCF0000015FDF719F8D4F824150448BDE81040E4
:10BD0000FDF712B85022012000000140004401401C
:10BD1000034B4FF08040D3F80415FDF705B800BF82
:10BD200050220120024B0348D3F80815FCF7FCBF52
:10BD30005022012000040040024B0348D3F80C15A8
:10BD4000FCF7F2BF5022012000080040024B0348DC
:10BD5000D3F81015FCF7E8BF50220120000C00407A
:10BD6000024B0348D3F81C15FCF7DEBF502201201C
:10BD70000004014010B5064C0648D4F81C15FCF729
:10BD8000D3FFD4F830150448BDE81040FCF7CCBF11
:10BD90005022012000040140001C004010B5064C58
:10BDA0000648D4F81C15FCF7BFFFD4F83415044836
:10BDB000BDE81040FCF7B8BF50220120000401404C
:10BDC00000200040024B0348D3F82015FCF7ACBF1D
:10BDD0005022012000400140024B0348D3F82815AF
:10BDE000FCF7A2BF5022012000480140024B03484B
:10BDF000D3F82C15FCF798BF502201200018004002
:10BE0000704710B501208EB009F008FD012809D156
:10BE1000002109F009FD614B1A6882F308885B680C
:10BE20009847FEE75E4A00245E4BD1685E4821F4E5
:10BE3000E0610904090C0B43D3605C4B596F196B2B
:10BE400041F480211963196B01F480210D910D9942
:10BE5000196B41F480111963196B01F480110C9175
:10BE60000C99196B41F480011963196B01F480017D
:10BE70000B910B99196B41F000511963196B01F08B
:10BE800000510A910A99196B41F080411963196BAD
:10BE900001F0804109910999196C41F4003119644C
:10BEA000196C01F4003108910899196C41F4802152
:10BEB0001964196C01F4802107910799196C41F4F8
:10BEC00000211964196C01F4002106910699196C7E
:10BED00041F480111964196C01F4801105910599E0
:10BEE000196C41F080411964196C01F08041049192
:10BEF0000499196C41F000411964196C01F000417A
:10BF000003910399596C41F010015964596C01F087
:10BF1000100102910299596C41F020015964596C49
:10BF200001F0200101910199596C41F400615964BB
:10BF30005B6C1F4903F400630093009B1D4BD3F817
:10BF4000BC31B3FBF1F1C0F8B818D2F8FC101A48B4
:10BF500041F08071C2F8FC101849C1F8B00F4C6074
:10BF6000086840F0010008604FF47A71B3FBF1F308
:10BF7000013BB3F1807F08D24FF0E0214B61F02309
:10BF800082F8233007238C610B614FF0E0221369A4
:10BF900043F0040313610EB010BD00BF0000F01F9A
:10BFA00000ED00E00003FA055022012000380240B5
:10BFB00040420F000000012055CEACC5001000E04B
:10BFC000074B03EB8000D0F8E43033B193F8AD2099
:10BFD0004A7093F8AC300B7070474B70FBE700BFB2
:10BFE000D87E06082DE9F04117462C4A98460546AA
:10BFF00002EB8003D3F8E44084B304F1AE0302F50E
:10C00000827294F8AD00261DA36104F5D7736260B7
:10C01000E3614FF48073E160C4E904332368C4F83A
:10C02000A830A36308F0CCFC18F0080F19D0013534
:10C03000EDB218B140F20673C380057294F8B622CF
:10C04000022108F09DFC94F9B702D4F8B81252F01E
:10C05000B5F994F9B7023446FDF7E6FE2046BDE88F
:10C06000F081BA0794F8AC800BD56B1CDBB218B129
:10C0700040F206520372C28094F8B622022108F000
:10C080007FFCFB07DFD50135404608F099FCEDB297
:10C090000028D3D040F20663CEE700BFD87E060862
:10C0A0000148FCF71BBF00BFEC0401200148FCF76E
:10C0B00015BF00BFA80701200148FCF70FBF00BF54
:10C0C000640A01200148FCF709BF00BF200D0120D0
:10C0D0000148FCF703BF00BFDC0F0120426B2423A3
:10C0E000816870B580F89D300446136800F134050E
:10C0F00023F0010313600023136053609360816396
:10C100008179C0F8A03080F89C3080F89D3080F8AC
:10C110009E308802A36400F48050E3646365E063AA
:10C120000803637900F4005013F0010620644FEA1D
:10C13000012000F4806060641CBF0420A06413F040
:10C1400002031EBFA06C40F00800A064C8070FD512
:10C1500036B1A06D40F00200A0654FF4803020663B
:10C1600033B1A36D43F00103A3654FF40033E365DE
:10C17000242311F0080F94F89D10284684F89D3070
:10C18000136823F00103136036D0FEF7E3F80128AB
:10C1900018D0A36D13B12846FBF7CAFF636B5A682A
:10C1A00022F490425A609A6822F022029A609A68B9
:10C1B00042F008029A6028461A6842F001021A60AA
:10C1C00054F080FD6179CA070DD5D4F8A4301A68FF
:10C1D00042F480721A609A6842F001029A601A680A
:10C1E00042F020021A608B0705D5D4F8A42013680A
:10C1F00043F08003136070BDFEF7ACF80128E1D076
:10C20000A36D13B12846FBF793FF636B5A6822F4C2
:10C2100090425A609A6822F02A02CBE781605DE77B
:10C2200041715BE710B51C2008F0CAFB04461121E0
:10C2300008F085FB204608F07CFBC8200AF003FDCF
:10C240002046BDE8104008F06FBB934B2DE9F04F3E
:10C25000D3F8BC5887B06B6913F00103029340F028
:10C26000A9816A69AB691A4200F0A4816B69AA6965
:10C2700013409C0701D502236B616B69AA691340C7
:10C28000180300F19A81844CD4F8BC385A69996932
:10C290000A40510311D5D3F8182803F5006304F6BA
:10C2A000BC0705F5106ADB694FF0000913409BB22B
:10C2B0000193019B002B40F02A84D4F8BC0842690A
:10C2C00083691A4216D5D5F8043823F00103C5F85E
:10C2D000043894F8A83C012B15BFD4F8B83C0023CF
:10C2E00093F8FD2184F8A83C18BF83F8FC214FF097
:10C2F000004343614369826913401B050FD5D5F89C
:10C300000838DF0708D5D4F8B83C93F8FC2183F847
:10C31000FD21042283F8FC214FF40063436143694B
:10C32000826913401E010FD54FF00063436194F8FA
:10C33000A83C002B40F0FB84012384F8A83C436D0B
:10C34000C3F38303C4F8AC3C436982691340D90446
:10C350003AD5D5F80438102105F5006623F001031D
:10C36000736054F0D5FAD4F8C00805F510630022C4
:10C37000FF21824240F0E6844FF0FF33B361F3695E
:10C3800043F00113F361D4F8EC38002B00F0E184A2
:10C39000D6F8843043F00B03C6F88430736C43F056
:10C3A0000B037364D5F800383C4A23F4FE6394F819
:10C3B000CC18D4F8BC08C5F8003854F041FAD4F8C9
:10C3C000BC384FF480525A61D4F8BC385A69996924
:10C3D0000A40920472D5D3F8002922F4FF6222F0B9
:10C3E0000702C3F8002903F50062916801F0060115
:10C3F000042905D1D3F8001941F00301C3F800194D
:10C40000516841F480715160D96821F47051D9604C
:10C41000916811F0060F11D0916801F00601022910
:10C4200000F0A184916801F00601062900F09B84C8
:10C43000926802F00602042A00F095844FF400721C
:10C440000027C4F8D028DA68C4F8C87842F410523B
:10C45000DA60D4F8B86C00224FF04008402311464F
:10C46000D6F8300254F050F9434600228021D6F825
:10C470003002C6F8108154F047F90123C6F8208035
:10C4800086F8FC31D6F8183253B9D6F820323BB9C9
:10C49000D6F8283253B103E050220120C82E0120E3
:10C4A000D6F81432304631795B689847D4F8B83CF6
:10C4B0004FF400521F74D4F8BC385A61D4F8BC2829
:10C4C000536991690B40DB062FD5936923F0100364
:10C4D00093612B6AC3F3434003F00F07022840F037
:10C4E000AF8447F6F0710B421BD01C20C3F30A1334
:10C4F00005F5805500FB0740DE1CD0F8C0CAB61019
:10C5000002998E4240F094841C2101FB0741D1F82E
:10C51000C05AD1F8CC0A1D441844C1F8C05AC1F819
:10C52000CC0A936943F010039361536992691340F5
:10C530001F070ED5D4F8B80C90F8FC31032B04D1AA
:10C54000D0F81432DB6903B19847D4F8BC3808221C
:10C550005A61D4F8BC28536991690B40DE0202D5B8
:10C560004FF480135361536991690B409D0202D5CA
:10C570004FF400135361536991690B40580002D581
:10C580004FF080435361536991690B40590711D5AE
:10C5900055686B0709D5D4F8B80C012380F8FC3135
:10C5A000D0F8143201795B689847D4F8BC385A68DF
:10C5B00015435D6007B0BDE8F08FD5F8183805F574
:10C5C0003067D5F81C284FF0000ADFF85C83134071
:10C5D000A8F6BC061B0C0193019B002B3FF453AE45
:10C5E000019BDA0740F14D81D6F8BC385FFA8AF139
:10C5F00003F5306203F5006302EB411292685B6958
:10C6000002EA030919F0010F39D00123BB60D6F803
:10C61000CC38012B0CD13B69D8F80022C3F31203AC
:10C62000D31AC8F81032D8F804321344C8F80432C8
:10C63000D6F8B84C00297AD1D4F8F431032B10D1B4
:10C64000D4E94303984264D9C01AD6F8C02A834279
:10C65000C4F80C0128BF0346D4F830029BB253F053
:10C66000BBFFD6F8CC18012909D1D6F8C83A5AEA46
:10C67000030304D1AB4AD6F8BC0854F0E1F819F032
:10C68000080F00F0F480D6F8B84C96F8780C04F552
:10C69000027B84F8080296F879EC84F809E296F8AF
:10C6A0007B1C96F87A3C03EB01239BB2A4F80A3278
:10C6B00096F87D2C96F87CCC0CEB022C1FFA8CFCA7
:10C6C000A4F80CC296F87F1C96F87E2C02EB01228F
:10C6D000012192B2C4E97D1200F01F01A4F80E22DC
:10C6E000012900F04881022900F05A81002940F018
:10C6F0000B82BEF1090F00F2D480DFE81EF01701B3
:10C700003201D2002701D2008A002400D2000301A6
:10C71000CD00D4F814321B692BB194F8FC21032A04
:10C7200001D120469847204654F044F899E7D4F8C0
:10C7300014329B69002B94D094F8FC21032A90D1E9
:10C74000204698478DE71A0A013A062A00F2A98086
:10C75000DFE802F0041D2AA7A74A5400D4F81032DB
:10C760001B680DF11601207C9847BDF81620002AA1
:10C770007BD0B4F80E32002B77D09A42014628BF06
:10C780001A46ADF81620204654F01DF86DE0227CC4
:10C79000D4F8143232B99B6A0DF11600984702237F
:10C7A0004370E2E7DB6AF7E7DBB2052B79D8DFE815
:10C7B00003F003070B0F1317D4F810325B68D0E7B0
:10C7C000D4F810329B68CCE7D4F81032DB68C8E7A5
:10C7D000D4F810321B69C4E7D4F810325B69C0E7A3
:10C7E000D4F810329B69BCE7237C002B59D1D4F8D4
:10C7F00014320DF116005B6B9847B6E7237C002BD3
:10C800004FD1D4F814320DF116001B6B9847072353
:10C81000C6E75CEA0202D4F8300203D194F8FC11B6
:10C82000032902D154F06AF81FE003F07F0B84F86B
:10C83000FEB190F8B833012B0ED00368D3F800187E
:10C8400021F4FE61C3F80018D3F8001841EA0B1177
:10C85000C3F8001880F8B823204653F0ABFFBBF1B3
:10C86000000F17D0022384F8FC310823BB6019F0B5
:10C87000100F01D01023BB6019F0200F01D020232E
:10C88000BB60019B0AF1010A203708F11C085B0814
:10C890000193A1E60123E6E7D9B2012986F8BC1C81
:10C8A00002D9D4F83002BDE794F8FC31022B0FD046
:10C8B000032BF6D1C9B902232046616084F8FC310C
:10C8C000D4F814325A689047204653F073FFCCE7EF
:10C8D0000029F9D001210323616084F8FC3120464E
:10C8E000FBF730FD0228EFD1DBE761680129EBD0CF
:10C8F000D4F81432C9B220465B68984796F8BC1C3D
:10C900006160ECE7012ACCD194F8FC31022B03D012
:10C91000032BC6D1211D36E72146002341F8083FED
:10C9200031E700BFC82E01200C2B012094F8FC3108
:10C93000023B012BB5D80123E360D4F804320BB1DC
:10C940000323E360022204F10C011CE7012B8CD1CC
:10C95000C4F80432D4F81432594620469B689847EC
:10C96000B2E794F8FC21023A012A9AD8012B7FF40D
:10C970007CAF0023ECE794F8FC31032B91D15FFAF4
:10C980008CFCBCF1030F8CD8D4F8143259462046E5
:10C990009B689847B4F80E32002B7FF466AF93E79C
:10C9A00000F060005FFA8CF1202806D1D4F8143230
:10C9B000594620469B68984757E7BEF1010F46D07D
:10C9C000BEF1030F33D0BEF1000F7FF44EAF94F8E9
:10C9D000FC31022B00F09080032B7FF462AF4FFA02
:10C9E0008CFC01F07F0210234FF0040EBCF1000F0D
:10C9F000B4BF501C02F11000BCF1000F4FF01C0C32
:10CA000013FB00E3D4F83002A8BF0CFB0101234460
:10CA1000B4BF0CFB020291F8FA211946B8BF92F894
:10CA20003A20003A18BF01221A600222ABE694F8BD
:10CA3000FC21022A60D0032A7FF433AF002B89D176
:10CA40004B0687D0D4F8300253F019FF82E794F8F0
:10CA5000FC21022A50D0032A7FF423AF002B7FF45D
:10CA600004AF11F07F003FF42FAF4FFA8CFCD4F8E5
:10CA700030221C23BCF1000F4FEADC7CB4BF03FB67
:10CA8000002103FB01214FF00003B4BF383101F551
:10CA9000FC718B70087081F801C092F8B833012BDB
:10CAA0003FF458AF01234FF0200E82F8B8331368DB
:10CAB000BCF1000F14D0C87803F510630978023870
:10CAC0001EFB01330128196821F40011196003D8F5
:10CAD000196841F080511960002382F8B83339E7B2
:10CAE00003F530631EFB0033186820F40010186053
:10CAF000C97802390129EAE748063FF4B6AED4F80E
:10CB0000300253F0BCFEB0E600F08001F7E7019B75
:10CB1000DA0740F1A980D4F8BC285FFA89FBD2F883
:10CB2000101802F5106252F8CC3C02EB4B1223FABB
:10CB30000BF892684FEAC8185FFA88F848EA0108CB
:10CB400008EA020818F0010F4AD00121D5F834385C
:10CB500001FA09F123EA0103C5F834380123CAF8C0
:10CB60000830D4F8CC38012B02BFD7E910239B182A
:10CB70007B6419F0FF01D4F8B86C40F0A780D6F8B8
:10CB8000F431022B17D1D6E90730834276D91C2223
:10CB90001B1AD6F8300202FB0B420391D2F800298F
:10CBA000F3619BB253F04EFD03990B460A46D6F84B
:10CBB000300253F011FD96F80032012B02D1002310
:10CBC00086F80032D4F8CC18012909D1D4F80839F4
:10CBD00059EA030304D1A64AD4F8BC0853F030FE46
:10CBE00018F0080F02D00823CAF8083018F0100F08
:10CBF00002D01023CAF8083018F0400F02D04023AA
:10CC0000CAF8083018F0020F02D00223CAF8083020
:10CC100018F0800F28D0D4F8BC08D7E9133200F5FB
:10CC2000106600F580519B1A3A6C06EB4918934246
:10CC300001EB0B3BA8BF1346DA1C48BF9A1D9210AC
:10CC4000D8F8181089B2914203D9D7E913218A4242
:10CC50004AD8002B08DC0122D0F8343802FA09F255
:10CC600023EA0203C0F83438019B09F101091C379B
:10CC70000AF1200A5B080193FFF71BBBB269B2FB04
:10CC8000F0F300FB132393B9904210D8D6F8F811B3
:10CC90008A420CD21A461946D6F83002039353F052
:10CCA000D1FC039BC6F8F8311A4619467FE7D6F83F
:10CCB0001432DB682BB196F8FC21032A01D13046EF
:10CCC00098470523C6F8F4310023EDE7D6F814326F
:10CCD0005B69002B3FF476AF96F8FC21032A7FF4C2
:10CCE00071AF304698476DE7521A3B6C94F8CC18F8
:10CCF0009342A8BF1346DA1C48BF9A1D921031B167
:10CD0000796C19447964396D1944396598E71FFACB
:10CD100083FCD7F844E00CF1030C4FEAAC0C8C45D3
:10CD2000EED05EF821600131CBF80060F7E7D4F86F
:10CD3000B83C93F8FC2183F8FD21042283F8FC2100
:10CD4000FFF702BB99600132C3F808122033FFF7E6
:10CD500010BB736943F02B037361336943F00B031A
:10CD60003361FFF71FBB032242494348C4F8C82878
:10CD70004022C4F8D028414AD2F8BC211144814253
:10CD800006D8DA6842F470520127DA60FFF761BB17
:10CD90003B493C481144814203D8DA6842F460526E
:10CDA000F2E7A2F574013848A1F51051814203D889
:10CDB000DA6842F45052E7E7A2F183713348A1F5F3
:10CDC000E741814203D2DA6842F44052DCE730495D
:10CDD00030481144814203D8DA6842F43052D3E734
:10CDE0002D492E481144814203D2DA6842F4205280
:10CDF000CAE72B492B481144814203D2DA6842F436
:10CE00001052C1E7A2F1B7712748A1F558518142EC
:10CE100003D2DA6842F40052B6E724491144244AA6
:10CE20009142DA6834BF42F4E05242F4C052ABE7B8
:10CE3000029928684CF8210001310291FFF760BB8C
:10CE400006287FF46EAB05F58055C3F30A132968F5
:10CE5000C4F8781C2968C4F87C1C1C2101FB07411C
:10CE6000D1F8CC0A0344C1F8CC3AFFF75ABB00BF53
:10CE7000C82E0120405327FFFF340C000000012082
:10CE8000401E1BFF3F420F007F4F120020D61300B1
:10CE900060B6E5FE5FE3160000D3CEFE40771B00D0
:10CEA000C05BB3FEC091210020753800E05459FEEC
:10CEB000E09C410070B5484CD4F8A4321A6991073F
:10CEC00009D5DA68920706D56FF002021A619A69ED
:10CED000002284F8C0221A69560709D5DA68550776
:10CEE00006D56FF004021A619A69002284F8C02204
:10CEF0001A69100709D5DA68110706D56FF008021C
:10CF00001A61DA69002284F8C0221A69D20609D5AA
:10CF1000DA68D60606D56FF010021A61DA690022C7
:10CF200084F8C0221A69D5072ED5DA68D0072BD528
:10CF30006FF001021A61294A934225D1D4E9912563
:10CF4000AA4221D0264B8CBFC2F58055AD1A1A4497
:10CF5000D4F82032A9B2D3F81462C3F80822C3F877
:10CF600010128EB90121D4F83802C3F81412ABB2F2
:10CF7000812153F067FBD4F844321D44B5F5805F3E
:10CF800018BF2E46C4F84462D4F8A4321A691106B8
:10CF900005D5DA68120602D56FF080021A611A69A7
:10CFA000D60505D5DA68150602D56FF080021A613C
:10CFB0001A69540605D5DA68500602D56FF04002AA
:10CFC0001A611A69910605D5DA68920602D56FF0E2
:10CFD00020021A6170BD00BF5022012000140040E1
:10CFE000405101202DE9F041114E0D46D6F8202286
:10CFF000D2F81432002BFBD104464719DFF83480F5
:10D00000BC4202D12846BDE8F081D6F8483214F877
:10D01000012B08F803200133C3F30B03C6F8483291
:10D02000FBF77EFA0028EBD1012009F00CFEF7E7B0
:10D030005022012040510120F8B50D461446FBF75F
:10D0400073F978B1084ED6F8EC73002C0ADD21464E
:10D050002846FFF7C7FFD6F8EC33241A0544DB1B3C
:10D06000322BF2D9F8BD00BF50220120034BD3F878
:10D070009C0208B107F047BC0120704750220120F4
:10D0800010B5FFF7F3FF0E4C18B9002384F8703287
:10D0900010BD94F87032032B04D90021D4F8A002FB
:10D0A00004F0B8FE94F864320133DBB2072B84F845
:10D0B0006432EAD8D4F8EC33C4F860320123E5E7EF
:10D0C000502201202DE9F043CC4C85B0D4F8A002C9
:10D0D000002800F0B381CA4D04F5237694F870322D
:10D0E000013B082B00F29481DFE813F009004000B7
:10D0F000CB009201AF01290171019201E401FCF71B
:10D10000E1FC00210846FCF76FFD0746FCF7EAFC4E
:10D11000012F40F07D814FF0000884F86582FCF714
:10D12000D1FC40F2AB110820FCF75EFD05280CD1C4
:10D1300084F86572FCF7D6FC94F86532002B00F099
:10D140005A81022384F87032C8E70128F2D10423FF
:10D1500042466946D4F8A00252F028FF9DF80330F9
:10D16000AB2B04BF022384F86532E3E7FCF7AAFC8B
:10D1700094F8653200213720022B0CBF4FF0804716
:10D180000027FCF731FD29203946FCF72DFD074625
:10D19000FCF7A8FC002F40F03B8194F86532022B8D
:10D1A00039D1FCF78FFC39463A20FCF71DFD80464B
:10D1B00004233A466946D4F8A00252F0F7FEFCF781
:10D1C00091FCB8F1000F02D0FFF75AFF86E7009BF1
:10D1D0001BBAC3F3807384F86632FCF773FC00213A
:10D1E0000920FCF701FD98B910213046FCF7B4FC8A
:10D1F000804668B901217F2050F086FD012807464E
:10D2000006D10221404650F07FFD38B101282CD0D4
:10D21000FCF768FCFCE084F86672DEE704212C2051
:10D2200050F072FD032181464E2050F06DFD804686
:10D230000C21362050F068FD08F10208411C07FA65
:10D2400009F301FA08F2A2FB03375B0A43EAC7536A
:10D25000C4F87432FCF746FCFCF734FC00210A20C9
:10D26000FCF7C2FC50B903236CE716213A2050F0BA
:10D270004BFD01308002C4F87402EBE7FCF732FC8E
:10D28000A2E710216846FCF767FC002840F0C08048
:10D290009DF8003084F87A32BDF801305BBAA4F80A
:10D2A00078329DF8033084F87B329DF8043084F89E
:10D2B0007C329DF8053084F87D329DF8063084F884
:10D2C0007E329DF8073084F87F329DF808301A09C5
:10D2D00003F00F0384F88532DDF8093084F88422E6
:10D2E0001BBA9DF80E20C4F880329DF80D301B014A
:10D2F000DBB243EA121302F00F0203F5FA6384F87B
:10D300008822A4F88632FCF7EDFB94F8663263B904
:10D31000FCF7D8FB4FF400711020FCF765FC0746C2
:10D32000FCF7E0FB002F7FF44FAF0221D4F8A002FE
:10D3300004F070FD0023C4F86C32042302E794F873
:10D3400054128023D4F84C22D4F8A00202EBC1126C
:10D35000002152F02BFE94F854320133DBB2042B3F
:10D3600084F8543254D102232A460021D4F8A00272
:10D3700052F01CFE012300226946D4F8A00252F0AC
:10D3800015FE9DF8003003F01F03052B10D1072375
:10D39000D4F8585284F87032D4F8EC33C4F86032C0
:10D3A000B5B3D4F85C320120D4E99321A8472FE02B
:10D3B000FFF766FED4F85872002F3FF48FAED4F812
:10D3C0005C320022D4F850120120B84786E652F0B1
:10D3D00013FE002875D0002384F86432D4F86C3230
:10D3E000012B0FD9013BC4F86C32D4F868320133F9
:10D3F000C4F86832082384F8703209E05022012012
:10D400000C8006081DD1FCF7C9FB02283FF400AFD1
:10D4100094F87032013B022B08D8D4F8EC33D4F8DE
:10D4200060229B1AC82B01D9FFF72AFE94F87002DC
:10D4300004284FD0A0F108035842584105B0BDE878
:10D44000F083042384F87032E2E64FF40071D4F8DC
:10D450004C02FCF781FB0128074614D0022819D0A2
:10D460000028D5D1FCF73EFB0423D4F8585284F8A9
:10D47000703284F86472002DCAD0D4F85C32384619
:10D48000D4E9932192E7D4F86032D4F8EC236433E2
:10D490009342BDD2FCF726FBFFF7F2FDD4F8587299
:10D4A000002F3FF41BAE0022D4F85C32D4F85012A7
:10D4B00010468AE752F0A0FD18B1FCF713FB0423D5
:10D4C00099E7D4F86032D4F8EC23FA339342FFF4AE
:10D4D0007BAE9DE70120B1E72DE9F34105460E46FD
:10D4E00090461F46244C94F87032042B0BD0082B26
:10D4F00007D1D4F86832AB4219D0FCF74FFB0228B1
:10D50000F1D001200EE0FCF7DDFA94F8663263B941
:10D5100069021820FCF768FB48B1FCF7E3FAFFF753
:10D52000AFFD032002B0BDE8F0812946F1E794F891
:10D530007032FF220021D4F8A002082B8DF80420BD
:10D5400001AA0CBFFC23FE238DF80530022352F004
:10D550002DFD8023D4F8A0023246002152F026FD92
:10D560000123002084F854320623C4E99365C4E9FA
:10D57000968784F87032D5E75022012070B51B4C95
:10D5800005460E4694F87032042B10D1FCF79AFA37
:10D5900000213720FCF728FB31461720FCF724FB3D
:10D5A00090B1FCF79FFAFFF76BFD032002E0082B18
:10D5B00001D0012070BDD4F86832834212D0FCF74C
:10D5C000EDFA0228F5D1E1E794F8663263B9690211
:10D5D0001920FCF709FB0028E3D10823C4E99A5677
:10D5E00084F870320220E5E72946F1E75022012055
:10D5F000034BD3F8C00C08B103691847704700BF4C
:10D6000050220120002108B5084607F00FFA094B07
:10D61000094A03F5CE71D3F89C31C2F8C01C984773
:10D62000FFF7E6FF0028FBD00121002007F0FEF9FC
:10D63000002008BDF81001205022012008B5FFF796
:10D64000D7FF80F00100404240B208BD2DE9F84FFD
:10D650000E4601210024DFF84C80084617461D467F
:10D6600007F0E4F9A54206DC0021012007F0DEF90D
:10D670000020BDE8F88F06EB442A04EB0709D8F830
:10D68000C03C03B9FEE7D3F804B000235146484636
:10D690001A46D8470028F2D0FFF7AAFF0028FBD08F
:10D6A0000134DFE7502201202DE9F84F0E46012119
:10D6B0000024DFF850A0084615461F4607F0B6F9CB
:10D6C000A74218DD06EB442905EB040801E0FFF74B
:10D6D0008FFFDAF8C03C43B1D3F80CB000234946C1
:10D6E00040461A46D8470028F1D1FFF781FF0028AD
:10D6F000FBD00134E4E70021012007F097F9002076
:10D70000BDE8F88F50220120034BD3F8C00C08B1BC
:10D7100043691847704700BF50220120034BD3F8DC
:10D72000C00C08B183691847704700BF5022012020
:10D73000034BD3F8C00C08B1C3691847704700BF4A
:10D740005022012038B50D461446FFF7F1FF03685B
:10D7500000202B604FF40073238038BD034B1B78EF
:10D76000032B0CBF80204FF4807070471C2F0120CA
:10D770000B4A08B568B1816811B10723937008BDE1
:10D78000FFF7ECFF04231175C2E90100C2E90311A0
:10D79000F4E7012302F58051537081F8B431EEE7CC
:10D7A0001C2F012010B502784368022A0B4A06D1CB
:10D7B000D2E9800100EB410000EB532010BD01696C
:10D7C000D2F818020239D2F810421840D2F80C32BE
:10D7D000400A04FB01001844F0E700BF1C3F012091
:10D7E000074B1B78022B0BBF030AC0F3D413C0B244
:10D7F00000F07F000CBF0B600B601060704700BF33
:10D800001C2F012090F91A305A1C0AD003F581729E
:10D81000124B03EB0213DA796FF30002DA71FF2384
:10D82000837690F91B104B1C16D001F581710B4AC1
:10D8300002EB011302EB0112DB79D179C3F345034B
:10D84000012B8ABF03F1FF33002303F03F0363F38F
:10D850004601FF23D171C376704700BF1C2F012002
:10D8600008B5FFF77BFF034BD3F810325843400253
:10D8700008BD00BF1C3F01200378022B09D10D4BCE
:10D88000D3F820224368B3EB422F2CBF01200020A5
:10D890007047006960B1084B1B78032B16BF80B23C
:10D8A000064B4FF6F773984294BF00200120704753
:10D8B000012070471C3F01201C2F0120F7FFFF0FA4
:10D8C000F7B50D4641680446C1F308032B44B3F590
:10D8D000007F03D22944012061602EE0FFF792FF10
:10D8E0000378022B01D16168F4E7164BD3F81022BC
:10D8F000B5EB422F4FEA422721DCD3F818324668B5
:10D900001E407342AB421ADCAB19BB4210D3016913
:10D9100001AA007E52F040FE012810D12369ED1BC0
:10D9200063613544019B236163683B449B1B6360D7
:10D930002046FFF7A1FF0028D5D003B0F0BD00209E
:10D94000FBE700BF1C3F012070B504460E4615469C
:10D95000FFF7B6FF20B10DB12046A847012007E030
:10D9600094F82800022320B984F82830C4E90B5623
:10D9700070BD1846FCE7054A012392F8B41109B9B5
:10D9800082F8B431024A5370704700BF1C3F012037
:10D990001C2F012008B5074BC31A48BF03F2FF1321
:10D9A000B3F5805F4FEA632003D34FF0FF30FFF7FA
:10D9B000E2FF08BD342F01202DE9F74F12F0020BD2
:10D9C0001746019100F0D280002840F0CF80022657
:10D9D000FFF7D1FF6EE04FF0FF36DFF8C8C100253A
:10D9E000DFF8ACA1B6463446B146DCF800109CF82E
:10D9F0000E8088421BD1B8F1000F00F09980D2F858
:10DA00009840634E0134C2F8984005F581721201C6
:10DA1000B4502C465E4D04F5817805EB08129679DA
:10DA2000042ED4D8DFE806F0315EB15E6800B8F1AC
:10DA3000000F26D0B8F1010F14D105F581780AEB5B
:10DA4000081898F8078018F0010F0BD118F07E0F16
:10DA500008D15FEAD81116D1DCF80880C14501D998
:10DA6000AE46C14601350CF1100C082DBDD1751C18
:10DA70007AD1611C5DD1BEF1FF3F00F08680744613
:10DA800057E02E46EEE72C46ECE717F0010215D0E2
:10DA9000404BD3F8C03C002B77D03F495F68002350
:10DAA0003E4A01EB4421B84700286ED005EB08152B
:10DAB0000223AB71304603B0BDE8F08F05EB0810D0
:10DAC000032B4FEAE70690F807C066F3C71C80F8FF
:10DAD00007C02BD94FF6FF72934228BF134605EBC0
:10DAE00008129380BBF1000F06D005EB041000F57F
:10DAF00080501830FAF73CFD7A0741BF05EB081259
:10DB0000D37943F00103D371FB0608D505EB081563
:10DB1000EB79C3F34502013262F34603EB711E4B0E
:10DB20000126019A03EB44231360C3E71346D6E7AB
:10DB30002C46174E41F2180506EB041C4CF8050064
:10DB4000D2F898500135C2F8985041F21C024CF8B6
:10DB5000025004F581724FEA021C06EB021246F8ED
:10DB60000C500025556055E73446E2E70C4AD2F8E0
:10DB70000862002E3FF42FAFD2E9834505FB06442F
:10DB8000A042FFF428AFFFF7F6FE002692E700BFA1
:10DB90001C2F012050220120342F0120519D00080C
:10DBA0001C3F0120343F01207FB50F4D01AA0C46D8
:10DBB00002A9FFF715FE05F58053029E0322D3F854
:10DBC000000203A900233044FFF7F6FE012808D124
:10DBD0002978039B019A02290CBF23F8124043F8CD
:10DBE000224004B070BD00BF1C2F01202DE9F0477A
:10DBF0000D4686B01646074603AA04A92868FFF713
:10DC0000EFFD374A0499D2F80032A2F5805A01EBB1
:10DC10000308039B013B9C19FFF7A0FD2B68E41A46
:10DC20000444B4FBF0F408EB04092968A9EB0803E9
:10DC3000B14203D3012006B0BDE8F087039A0193F7
:10DC4000FFF78CFD9419019B641A844228BF044697
:10DC5000002A36D1A04294BF0A220B2205A94046D1
:10DC6000FFF7AAFE0128E6D19AF800002A680228E8
:10DC7000059902F10102039B2ED1A34223D32B6805
:10DC8000012F039AA3EB020323442B6014D1B34268
:10DC900012D102280BBF04F1004404F180434FF677
:10DCA000FF734FF0FF320BBF04F1FF3403F1FF337A
:10DCB00021F8143041F82320002308F101080393D0
:10DCC000B3E70B22CAE721F8132001330132D4E76E
:10DCD00041F8232001330132A342F9D3CFE700BF3B
:10DCE0001C3F01202DE9F04F0C4685B083461646B7
:10DCF000FFF734FD01AA814602A92068FFF770FDF5
:10DD00000BF1FF33012B68D9019B63B94D46BBF181
:10DD1000010FDFF8CC808CBF4FF0000B4FF0010BF0
:10DD2000A8F5805A1BE0FFF726FE02202AE0D8F86B
:10DD30007821C2B1D8F89401884214D1D8F81032B1
:10DD4000013A590202EB4323B3FBF1F30344B3FB63
:10DD5000F5F205FB12320AB12B449B1A23602168AD
:10DD6000B142E4D329E0D8F800020023029F09223F
:10DD700003A93844FFF720FE012806D00228D4D09A
:10DD80000028ECD105B0BDE8F08F9AF80020039987
:10DD9000022A07D0032AC8D1019B51F8233023F06F
:10DDA000704302E0019B31F81330B3FA83F3276824
:10DDB0005B095B4504D1BE42E4D803202660E1E75D
:10DDC000019B2F442B4427604B450193E0D3029BDA
:10DDD0000133029300230193C1E7012597E700BFB8
:10DDE0001C3F012037B50446C0690D4698B1002399
:10DDF000032201A9FFF7E0FD012806D1B4F9203084
:10DE0000002B0ADA0220FFF7B6FD03B030BDE5258E
:10DE10005554A2680BE00120F7E7019A012D4FEA63
:10DE2000431102EB4313F4D0022DF0D0E268DA6123
:10DE30002278032A04D100221A775A779A77DA7760
:10DE4000626A110C5A839982DFE770B50446042692
:10DE50002F4D94F83430052B2CD8DFE803F0032441
:10DE60003139424BD5F8082204F130010120023249
:10DE7000FFF738FF012807D00238C0B2012819D8AF
:10DE8000052384F83430E4E7D5F81012E268236BF8
:10DE900002EB4122C5F81432E260E26A236102B962
:10DEA00063620123EDE74FF0FF31206BFFF77CFE4B
:10DEB000012801D0002070BDE36A3BB10223E0E7F6
:10DEC000D4E90B01FFF770FE0128F3D10323D8E753
:10DED00000212046FFF786FF0128EBD184F834604B
:10DEE000B7E794F82830082B02D1002384F82830B3
:10DEF0000120E0E794F8283001220220082B04BF1B
:10DF0000002384F82830024B83F8B521D3E700BF03
:10DF10001C3F01202DE9F7430446DFF8149194F8E3
:10DF20003850032D7FD8DFE805F002106D762046CB
:10DF3000FFF78BFF012802D184F83800EFE70228B1
:10DF400072D1032384F83830E9E7237820466668E5
:10DF5000022B1CBFD9F818321E40FFF723FC0746DE
:10DF6000C6F34F26361A0023022201A93846FFF7CE
:10DF700023FD06EB0708012805461FFA88F853D150
:10DF80004FF400720021019859F002FEE369FBB1E1
:10DF90006368EBB9019B4FF020322E211A605A6062
:10DFA0001970C3F80720606A1A62050C58831020A4
:10DFB0005A6283F8201083F82110D872C3F8272002
:10DFC000E26B9D8222FA00F15A8783F82B00998632
:10DFD000D9F810124B1E984508D24FF40071204614
:10DFE000FFF76EFC013752F003FABCE7C1EBC151F9
:10DFF0002046490201F50071FFF762FC52F0F8F982
:10E0000002239FE7002384F82830236C0BB12046BD
:10E010009847012508E00020236C84F8280003B10C
:10E020009847022500E00025284603B0BDE8F083AC
:10E030001C3F0120F8B52E4E044600F13007A6F52E
:10E04000B87594F83830032B50D8DFE803F0022E6F
:10E05000363FD5F894212261FFF702FCE3681844AB
:10E06000E060FFF77BFB1044C5F89401FFF7F8FB75
:10E07000D5F87831181AC5F87801FFF7F1FBD5F813
:10E080007C31181AC5F87C012263FFF767FBE36A4D
:10E090001044606323B96262012384F83830D0E70A
:10E0A000FFF75CFB101A2063F6E700213046FFF70C
:10E0B00099FE01280ED10223EFE7626B3946012059
:10E0C000FFF794FD012805D10323E6E70021204650
:10E0D000FFF788FE431EDBB2012B06D894F82830E8
:10E0E000062B04BF002384F82830F8BD0220F1E796
:10E0F0008C4001202DE9F7430029454D044614BF0B
:10E100000226002605F5805794F83C30042B71D880
:10E11000DFE803F0290336406300DFF8FC802B784A
:10E12000206B032B53D1404594BF4FF000094FF0B3
:10E130000109B9F1000F48D101A94FF0C1FD012833
:10E1400063D14946206BFFF72FFD01285DD1019B6C
:10E15000D7F814222363013B934294BFC7F81432CB
:10E16000C7F81422DBE731462046FFF73BFE0128C3
:10E17000034648D1626B02B1022384F83C30C3E706
:10E18000626B04F130010020FFF730FD01283AD125
:10E190000323F2E7E26A0021D7F89431C7F894210B
:10E1A0009B1AD7F810221B485343D7F8782102EB6B
:10E1B0004322C7F87821D7F87C2102EB4323C7F824
:10E1C0007C31FFF70FFE01281DD10423D5E71FFA8C
:10E1D00080F94FF6F7739945A6E794F82830042B99
:10E1E00004BF002384F82830A36B0BB12046984766
:10E1F00001200AE0022094F82830042B05D10023E6
:10E2000084F8283001E00228F5D003B0BDE8F0839F
:10E210001C2F01208C400120F7FFFF0F70B5037801
:10E220000446023B012B1CD8237E990623D42046AA
:10E23000FFF7E8FA237E1A070AD51F4D95F89801D3
:10E24000C31F5842584152F0D3F8002385F8983143
:10E250000023237084F82830E36A5BB1BDE8704086
:10E260001847037E13F0060FDED00121FFF7BAFD39
:10E270000128D9D070BDE269002310491801405827
:10E28000824211D10E4903F5817201EB0213DB7951
:10E29000C3F34503012B0BD8002301EB0212D17904
:10E2A00063F34601D171C2E70133082BE6D1BEE723
:10E2B000013B03F03F03F0E71C3F0120343F012006
:10E2C0001C2F012010B580B1027872B190F828207F
:10E2D0006AB9C162D0E9012494422CBF8460826093
:10E2E000032280F82820FFF799FF012010BD0020AD
:10E2F000FCE7B1F904300F2B2DE9F34104460D463C
:10E3000016460BD14FF40071FFF7DAFA18B9002066
:10E3100002B0BDE8F0814FF6FF73AB802046FFF7F7
:10E3200041FA94F91B200746531C11D01E4B41F2B1
:10E33000180103EB021041588F4230D0FFF71BFB4E
:10E340002046FFF799FA0028E1D00023336024E04B
:10E350002046FFF791FA80460028F1D1381E18BFF9
:10E36000012052F045F84346112201A93846FFF733
:10E3700023FB0128E4D10198FFF70CFBE076019A1A
:10E38000002ADDD0AB88204601331BB2AB8002EB04
:10E3900043133360FFF706FA28600120B8E718330B
:10E3A00003EB42230193EAE71C2F01202DE9F04300
:10E3B000A24E87B00446A6F5DC7594F83030042BE5
:10E3C00011D8DFE813F0130005005E00EF003601FE
:10E3D00004F11C0901AA49463046FFF78AFF0128CB
:10E3E0000ED002282FD007B0BDE8F083304650F0A1
:10E3F00071F94FF6FF732384012384F83030DCE792
:10E40000019F0FB13B7863B93046FFF7FBF9237EDC
:10E41000DF061BD550F05EF94FF6FF73238402230D
:10E42000EBE797F80B8018F0080FD3D10B2204F11B
:10E430003101384659F0B0FC0028CBD1637E88EA20
:10E440000303D90604D53046FFF7DCF90423D4E7EB
:10E45000BA8A7B8B43EA0243D5F8102263625202E8
:10E46000FB69B3FBF2F102FB1131A36009B1134464
:10E470005B1A3046E36084F81980FFF7C3F9032381
:10E48000BBE795F8E031002BADD104F11C0809275A
:10E4900001AA41463046FFF72CFF012875D10198AB
:10E4A000002853D00378E52B01D0002BF0D1FFF7E3
:10E4B00071FA634901EB0010FAF75AF801F5D070D0
:10E4C000FFF7A0F920220021019859F061FBD4F850
:10E4D0003120019B03A81A60D4F835205A60B4F8A3
:10E4E00039201A8194F83B209A72019B627EDA727D
:10E4F00002F05EFF00284CD0524B03A902AAB3F8E9
:10E50000C43C0846ADF808304FF03EFB9DF80E20A5
:10E510009DF80F30019943EA4213BDF80C20A2F296
:10E52000BC7243EA42239DF811200B829DF8103003
:10E53000DB0243EA42139DF8122043EA5203CB81E7
:10E54000019B1A8A1A83DA89DA8298E795F8B8313A
:10E55000022B3FF47BAF95F8E031002B7FF476AFD0
:10E56000D5F8CC21304685F8F03185F8EC3185F8C6
:10E57000E071C5F8E421C5E97D33D5F81432C5F85A
:10E58000E831FFF7C7FC012882D002283FF45EAFD4
:10E5900029E7019B6FF07E021A74472298735A7420
:10E5A000D873CDE7237E9A0608D50023112202A94D
:10E5B000E069FFF701FA01287FF415AF204650F01B
:10E5C00089F82269237E8AB91B0708D51E4B93F868
:10E5D0009821002A7FF407AF072283F898210023AF
:10E5E000204684F82830E36A9847FCE603F0F702F7
:10E5F00013F00403227608D00023E26AA1682046C3
:10E6000084F82830FFF7A0F9EDE6122AE7D1E26A94
:10E610000421204684F83C30A263626A84F8281002
:10E6200063636362C4E90B22C4E9023350F052F819
:10E63000D9E60020E36A2070D6E700BFD44001206D
:10E64000343F0120502201201C3F01202DE9F341DD
:10E6500003780446002B72D090F82830013B082B39
:10E660006DD8DFE803F0050947594B5E6C6267001F
:10E6700002B0BDE8F04199E6324B4568D3F810721C
:10E68000D3F818327F021D40216B2046FFF7F4F8C3
:10E69000064605EB0108474526D880B1D4E901328A
:10E6A0009A422CBFA260A360002384F82830E36A5A
:10E6B000002B44D0204602B0BDE8F041184701AA23
:10E6C0002169207E51F068FF012838D123696361F8
:10E6D000019B236163683B445B1B6360236BDB1B13
:10E6E0001D4425633546CFE763680028D6D10B4427
:10E6F0006360D3E702B0BDE8F0418FE50121FFF789
:10E70000F9FC01281BD10023216C204684F8283015
:10E7100002B0BDE8F041D5E5002102B0BDE8F0410E
:10E72000E8E402B0BDE8F04184E402B0BDE8F041A5
:10E73000FFF78BBB02B0BDE8F041FFF7EBBB02B0C7
:10E74000BDE8F0811C3F01204FF0FF31314A00232A
:10E750002DE9F0410D46304C107804280ED103F518
:10E76000817004EB0010C079C70707D46E1C52F803
:10E770000A0C01D0884201D21D46014601331032F5
:10E78000082BE9D16B1C42D0234C05F58177234E31
:10E7900004EB0713998849B1D6F8C03C33B104EBB8
:10E7A000051041F218029B6880589847D6F8C03C83
:10E7B0009BB11B4E04EB051C41F21800D3F80C80F2
:10E7C000184A002306EB45215CF80000C04720B141
:10E7D000022810D00020BDE8F081134B04EB071491
:10E7E000D3F89C20013AC3F89C200322A271012295
:10E7F00083F8A020EEE706F6E87604EB0714D6F8D7
:10E800009C30013BC6F89C300123A371E2E7012054
:10E81000E1E700BF423F01201C2F012050220120D0
:10E82000342F0120A99D00081C3F012008B50021BC
:10E8300044220E4859F0ACF90D4B4FF6FF7203F528
:10E8400080501B78A0F8D221022B4FF0030200F574
:10E85000DC7018BF134602760370436E43621023C8
:10E8600043764FF037FF012008BD00BFD4400120A0
:10E870001C2F01202DE9FF47BB4CDFF8FCA2A37839
:10E88000072B00F2B080DFE813F008003900B10078
:10E89000BC00C000520163016C010023092203A9DE
:10E8A0001846FFF789F8012840F09D80039B93F8F4
:10E8B000FE21552A1BD193F8FF21AA2A17D103F56F
:10E8C000DF7203F5FF73906870B11179A1F10B0548
:10E8D000012D05D8A54BC3F8FC010123A370CEE799
:10E8E00001F0F7010629F5D010329342EBD19F4B8E
:10E8F000022283F8B4210123637074E09B4D00234E
:10E90000092203A9D5F8FC01FFF756F801286AD1BE
:10E910000022039B2270B3F80B20B2F5007F45D193
:10E920001A7C022A42D193F8FE21552A3ED193F84F
:10E93000FF21AA2A3AD1B3F80EE0D5F8FC6176445B
:10E94000C5F8006293F80DC00CF1FF32C5F810C293
:10E950007F2A2BD8CCF100023CEA020226D14FEAF2
:10E960004C22013AC5F81822DF8A07B95F6AC5F858
:10E970000472B3F81100400100F2FF104012C5F814
:10E980002002B3F8131001B9196A0EEB00024FEA26
:10E99000470802EB47028A1A40F6F471B2FBFCF218
:10E9A0008A42C5F8082205D801232370032385F87D
:10E9B000B431A0E74FF6F47106448A42464497BF4B
:10E9C000022303222370002384BF2270DB6AC5F870
:10E9D0000C62C5F81C3295F8E0310BB9FFF726FF41
:10E9E000A3780133A37004B0BDE8F08703230522A8
:10E9F0005F49A3705F4B60480093302351F087FC60
:10EA0000F1E75D48FFF722FEEDE7DFF86091FEF7E2
:10EA1000A5FE0546A9F6FC77A9F6F878207D38B35F
:10EA20000128FCD1D9F810020021636842024FF09E
:10EA3000FF30B0FBF2F0D9F808221B184FF00200AB
:10EA400002F102024941934271F10001414638BF8F
:10EA50001A46FFF747F90328E0D801A353F820F03E
:10EA6000E7E90008A5EA0008E7E90008A5EA0008C8
:10EA7000D9F8082239460232FFF734F90328CDD8F5
:10EA800001A353F820F000BFE7E9000899EA000865
:10EA9000E7E90008CFEA000863680133A3600123B7
:10EAA0002375BBE7D4E901232669991AB14288BFCF
:10EAB000C4E9032103280AD00133B3FBF5F205FBB7
:10EAC00012320AB12B449B1A63600023E8E72169E4
:10EAD00006236529A3707FF6D2AEA1F164036539E0
:10EAE0002361FEF73BFE4042014001312161FEF708
:10EAF00035FE81427FF6C3AE1C4FD4F80C80D7F8A8
:10EB0000080201EB08050230A84294BF0020012052
:10EB100051F06EFC2369D7F81022C7F89481534353
:10EB20005B02C4E90185C7E95E330523D6E6A26826
:10EB300001201249FFF75AF8012801D10623CDE63A
:10EB400002287FF450AF0123084A82F8B431D3E69B
:10EB500000215046FFF746F90128F1D1A37801338F
:10EB6000BCE60323C8E600BF1C2F01201C3F012088
:10EB7000E30F070871D700088C400120202F0120E7
:10EB8000704700BF002070472DE9F74FCDE9001214
:10EB90004F4AD38911681B025689178AC91A93896B
:10EBA0006EEB0E0EA3FB010403FB0E44C009138998
:10EBB00040EA44601B04E411C018A6FB013506FBC3
:10EBC0000E554FEA1323D68844F1000443EA056347
:10EBD000F6032D129B19A7FB012607FB0E664FEAD1
:10EBE000D25245F1000542EA4622F61512F5FA6CBA
:10EBF00046F1000BBCF5FA6F7BF100074CDAA2FB83
:10EC000002784FF0050A02FB06F908EB4909A7FB59
:10EC10000A780AFB09884FEA5709BF0849EAC87908
:10EC200047EA8877B0EB090064EB6804DB1B294FE7
:10EC300065EBA805BC454FF0FF377BEB070720DAF3
:10EC400040F6AC57D21946F100065643A2FB0272B9
:10EC500002EB4606FA004FEAC608BA1A48EA5778A5
:10EC600066EB0808101844EB08044FF00B08A7FBEC
:10EC7000087208FB06267F0847EAC677DB1B65EBB0
:10EC8000660501FB0EFEA1FB011202EB4E0EC90F41
:10EC900041EA4E01BCEB010C009A8AB10C4A516961
:10ECA000A1FB032301FB0535520D009B42EAC5225F
:10ECB0006D15121A65EB0404D20B42EA44421A6045
:10ECC000019B0BB1C3F800C0012003B0BDE8F08F79
:10ECD0004061012024FAFFFF31B10A4BD3ED0C7AD9
:10ECE000FDEEE77AC1ED007A52B1064B9FED067A50
:10ECF000D3ED0D7A67EE877AFDEEE77AC2ED007A02
:10ED000001207047406101200000C842007970472F
:10ED10000079C0F34010704700794009704700BF88
:10ED2000704700BF704700BF9FED047AC7EE007ABE
:10ED300077EEA07A80EEA70A704700BF72C7D13D78
:10ED4000002380ED020A03604360704703685A1C89
:10ED500002601970704700BF03690133012B036122
:10ED60001CD0D0ED005A07EE903AD0ED026A30EE9A
:10ED7000656AF8EEE77A86EE277A77EE257A30EE46
:10ED8000670AC0ED017AC0ED007AF0EE667AE6EE31
:10ED9000007AC0ED037AC0ED027A7047002380ED5F
:10EDA000010A80ED000A8360704703685A1C026004
:10EDB0001970704790F83020034602F0FF0012B13E
:10EDC000002283F8302070474FF40063838170473E
:10EDD0004FF4006383817047064A002352F8041BF6
:10EDE000814204D00133042BF8D100207047012068
:10EDF000704700BF786101200120704701207047F3
:10EE00002DE9F8435F4F15460E46BC6CB7F84C2011
:10EE1000B7F85290C2EB24135200C2EBE402B7F9E8
:10EE20004E40624303FB03F4B7F9503024135C43B4
:10EE3000B7F95630A4134FEAE37804EBE224A4F5C3
:10EE4000FA317C6681FB01CE03FB0EF20CFB08223B
:10EE5000A3FB0C389044B7F954201B0A82FB010233
:10EE600043EA0863120342EA105200031B184FF0F2
:10EE7000000042EB2822A3FB093802F5004209FBFF
:10EE800002884FEAE8734FEA680253EA68086CD0D8
:10EE9000B7F95C904FEAE97809FB0EFE0CFB08EE2F
:10EEA000A9FB0C9CE644B7F95AC08CFB01814FEAE0
:10EEB000414C4FEA48414CEAD83C11EB0909B96E84
:10EEC0004EEB0C0CC1F5801E10EB0900B7F9581081
:10EED0000EF000480CEBC10148EA5E084FEACE7E16
:10EEE000BEEB000068EB010C40F63548A0FB0801C2
:10EEF00008FB0C1153F030F8B7F962304FEA613E6D
:10EF000080464FEA503C03FB0EF24FEAE3794CEAAD
:10EF1000C14C0CFB0929A3FB0C324A4403FB0EFE37
:10EF20000CFB02EEB7F96020A3FB0C3C4FEAE27940
:10EF3000E6445B0E43EACE1313EB000C02FB01F335
:10EF4000A2FB082841EB6E6E09FB0031D00CB7F92B
:10EF50005E30414440EA41301CEB00004EEBE141A1
:10EF6000000A40EA016000EB03100EB1000A3060B5
:10EF700025B104EB8404803424122C600120BDE808
:10EF8000F88300BF4061012001207047084B1868DA
:10EF9000084B10B5DC6E001BFA2807D809B1186FB2
:10EFA00008600AB15B6F1360012000E0002010BD13
:10EFB0003C26012040610120034B00220120C3E9CF
:10EFC0001E22C3E92022704740610120094B1A68C4
:10EFD000094BD3F88410521AFA2A9FBF9A6FC2863F
:10EFE000DA6FD3F880309DBF02874387012000206D
:10EFF000704700BF3C260120406101202DE9F0410F
:10F000000C4D0127DFF830802C686B691C400CB96F
:10F01000BDE8F081B4FA84F3C3F11F0307FA03F6E5
:10F0200008EB8303D3F8880024EA060403689847B2
:10F030006E61ECE7003C01404061012008B50068CA
:10F0400051F001F8014B1860012008BD406101201A
:10F0500008B5006850F0F7FF014B5861012008BD6A
:10F060004061012038B514460D46002943D0344B89
:10F070009FED346AD3ED327AB3F9E020F8EEE77A07
:10F08000C7EE866A07EE902AB3F9DC2007EE102A55
:10F09000B3F9DE20F8EEE77AB8EEC77AA6EEA77AE3
:10F0A000D3ED357AF8EEE77AE6EE877A93ED347AA7
:10F0B000B8EEC70AA6EEA70A07EE902AB3F9DA203F
:10F0C000F8EEE77A07EE102AB3F9D820B8EEC77A3F
:10F0D000A6EEA77A07EE902AF8EEE77AE6EE877AB0
:10F0E00093ED397AB8EEC77AC7EE066AA6EEA70A9C
:10F0F00055F032FC28600CB3114BDFED126AD3EDF2
:10F10000397AB3F9CC20F8EEE77AB3F9CE3007EECE
:10F11000102A87EEA60A07EE903AF8EEE77AB8EEE4
:10F12000C77AF6EE006A60EE277A9FED070AE7EEEF
:10F13000267A27EE800A55F00FFC2060012038BDAA
:10F14000406101200000F04A0000C8422DE9F04F64
:10F1500004463C2200218BB0654858F019FD621E20
:10F160006449033412F8013F581E032888BF002366
:10F17000944241F8043BF5D10120FFF72DFE40B148
:10F180005D4B322283F8F42093F82421013283F876
:10F1900024210220FFF720FE40B1574B312283F893
:10F1A000002193F82421013283F824210320FFF762
:10F1B00013FE40B1504B302283F80C2193F82421E8
:10F1C000013283F824210420FFF706FE40B14A4BA8
:10F1D000142283F8182193F82421013283F8242182
:10F1E000434C4FF00F084FF00009444E444F207B32
:10F1F00038B394F90D5005F0E3FB28B1052380F8EE
:10F200000780837100230372032105F098FB227BA2
:10F21000002316F83310914265D106EBC3035B68F7
:10F220002361C02303FB0575D5F8BC305A1C237538
:10F230000723C5F8BC20A37501239944637585F89D
:10F24000B83008F101080C345FFA88F8B8F1130FF0
:10F25000CDD1B9F1000F43D02A4B0025284C2A4EBE
:10F26000049394F8B830002B33D060794EF0AEFFA1
:10F2700020794EF0ABFF0122D4F8BC104FF440339C
:10F280001F4FC020914263614FF00003A2622264CD
:10F29000D8BF4FF0000CA361C8BF4FF0010CE36171
:10F2A000636200FB05720191E162C4F820C0C4E909
:10F2B0000E33C4E90C3323682361116D01B9516524
:10F2C00000FB0570016D11F010011FD0002384F8C0
:10F2D0004C30049B0135C034C833032D0493C0D196
:10F2E0000BB0BDE8F08F0133102B92D1002397E7CC
:10F2F0002862012078610120406101203C800608DD
:10F30000B41201206862012000230140026D4FF415
:10F31000005822F4885222F0020242F002020265F2
:10F32000726822F440327260726842F44032726055
:10F330005A6822F480725A605A6842EA0C225A6073
:10F340005A6822F040725A605A685A609A6822F4E9
:10F3500000629A609A689A609A6822F070629A6075
:10F360009A689A609A6822F040529A609A689A6005
:10F370009A6822F002029A609A6842F002029A6049
:10F380005A6822F400625A60DA6A22F47002DA6281
:10F39000019AD3F82CE002F1FF3C4EEA0C524FF4F4
:10F3A000806EDA629A6822F400729A609A6842F477
:10F3B00000729A609A6822F480629A609A689A60F1
:10F3C0004165026D22F0030242F0010202654FF432
:10F3D0000062D4F80CC084F84C106166C4F8881040
:10F3E000C4E91AE24FF48072DFF898E3C4E91C82A2
:10F3F0004FF40032C4E91E210322C4E92021A2688F
:10F40000C4E917C1A265DEF8008084F88C100221DF
:10F4100080F88D10116821F0010111601168C90791
:10F4200000F130811168182022F47F7EDFF85893B4
:10F4300021F0FF512EF0030E21F4772121F47C619D
:10F4400041EA0C0C4CF40B3141F4807111605169AC
:10F4500021F007015161D1B21039B1FBF0FCC04875
:10F460005F294FF03F01604488BF0EF1040E90F811
:10F470008000C4F8B0E08140C4F8B40004F1580042
:10F48000CEF808100591C02101FB05770021C7F8CF
:10F49000AC10012187F88D10A06404F110000391D5
:10F4A000C4F8900068B2079099F8150000285CD065
:10F4B00099F90D00079FB84257D101F1010C94F85A
:10F4C0004CA0D9F810005FFA8CF7BAF1010F99F847
:10F4D000168006974FF0000708973FF4FAAE4FF0FA
:10F4E0000107092884F84C7087B2029740F2E28045
:10F4F00007EB470C4FF0070BD3F80CA0ACF11E0C38
:10F50000984F0BFA0CFBB8422AEA0B0AC3F80CA07E
:10F5100040F0C980D3F80CC04CEA086CC3F80CC0AA
:10F52000062901EB810C00F2DA80ACF1050C4FF0FA
:10F530001F08596B08FA0CF8029F21EA080107FA24
:10F540000CFC5963596B4CEA0101596386498B42A3
:10F5500006D1122840F01A81716841F4800171606F
:10F560004FF0000184F84C100699039809F10C093A
:10F5700001300528039097D10021099194F84C108F
:10F5800001293FF4A6AE012184F84C109968CF07F9
:10F5900040F1CB809968C8077FF59BAE734FC020C0
:10F5A00000FB0570016D21F4E06121F0010141F4DF
:10F5B000807101655968490505D5016D21F44051F7
:10F5C00041F480510165C02101FB0571086D10F403
:10F5D000805002D0486D20F0060048650021644844
:10F5E00084F84C10C4F894006248C4F8980062484B
:10F5F000C4F8A4006FF022001860586840F08060E2
:10F600005860986840F480709860012084F88C00FD
:10F61000C02000FB057797F88D00012840F0988006
:10F62000022087F88D00C7F8AC101168019821F40A
:10F63000802111601421484303F14C015060916016
:10F640000499D1600599CEF80810116841F01601AF
:10F650001160516941F080015161116841F0080168
:10F660001160116841F0010111607268D20672D117
:10F670009A6812F0405F7FF42CAE9A6842F08042A4
:10F680009A6026E6DEF80010A1EB080105297FF656
:10F69000C5AEC02303FB05772023C7F8AC30032396
:10F6A00087F88D3015E6D3F80CA008FA0CFC4CEA6C
:10F6B0000A0C33E700EB400B4FF0070AD3F810C0F9
:10F6C0000AFA0BFA08FA0BF82CEA0A0CC3F810C075
:10F6D000D3F810C048EA0C08C3F8108020E70C29C2
:10F6E0004FF01F0110D8ACF1230CD3F83080029FEB
:10F6F00001FA0CF107FA0CFC28EA01011963196BF5
:10F700004CEA0101196321E7ACF1410CD3F82C80DC
:10F71000029F01FA0CF107FA0CFC28EA0101D962F8
:10F72000D96A4CEA0101D96210E79968134841F09F
:10F730000101996012490968B1FBF0F101EB410147
:10F740000991099900293FF425AF09990139F7E793
:10F7500084F88C1089E7044A93427FF4BAAD87E7B6
:10F760003C8006081200001000200140B412012065
:10F7700001800008578000085980000840420F00AF
:10F78000BC01012050220120286201200E4988423C
:10F7900002D011287FF4E4AE716841F40001716079
:10F7A000094988427FF4DCAE084909480968B1FB81
:10F7B000F0F10A2041430891089900293FF4D0AEA6
:10F7C00008990139F7E700BF12000010BC010120C1
:10F7D00040420F00024BD3F8800307F0C5B800BFCA
:10F7E000406101204A09012301F01F0103FA01F1E0
:10F7F00050F822300B4340F8223070474A09012369
:10F8000001F01F0103FA01F150F82230194214BF30
:10F8100001200020704780EA0120082341F22102E4
:10F8200010F4004F4FEA400018BF5040013B80B237
:10F83000F6D1704738B50C468D18AC4200D138BDB2
:10F8400014F8011BFFF7E7FFF7E74840082310F023
:10F85000800F4FEA400018BF80F0D500013BC0B2D6
:10F86000F5D1704710B50A440C46944200D110BD42
:10F8700014F8011BFFF7E9FFF7E738B50A4604461D
:10F8800005680020AA4203D36B1C2360287038BD92
:10F8900012F8011BFFF7D9FFF4E700BF82B08DED2E
:10F8A000010A019802B07047C31783EA400070470D
:10F8B0009FED087A0023C0ED020AC7EE007A0360CC
:10F8C00030EEA77AC0ED017AC0EE877AC0ED037AF8
:10F8D000704700BF83F9223E80ED010A704700BFE8
:10F8E000D0ED016AD0ED007A70EEA66AC0ED020A92
:10F8F00030EE677A80EEA66AE6EE077AB0EE670A27
:10F90000C0ED007A704700BF80ED000A704700BF6D
:10F910009FED047AC7EE007A77EEA07A80EEA70A10
:10F92000704700BF4E2DA63D002380ED030A036003
:10F9300043608360704700BF80ED030A704700BFDB
:10F94000F5EEC00AF1EE10FA06DCF0EE407A80ED3A
:10F95000000AB0EE670A704760EE810A90ED007A07
:10F9600077EE607AF4EEC07AF1EE10FA03DC77EE0F
:10F97000200AC0FEC07AB0EE670AC0ED007A704778
:10F98000B4EEE00AF1EE10FA02D480FE410A7047AC
:10F99000B0EE600A704700BF874BB3FBF2F39942A9
:10F9A0000DD300234FF07E52436083600260C3603A
:10F9B00003610023836143610362C361704707EE03
:10F9C000902ADFED7E6AB8EE677A07EE901AF8EEBD
:10F9D000677A27EE267A27EE277AFDEEC77A17EEAA
:10F9E000903A2033402B00F2D880DFED757AB4EEE8
:10F9F000E77AF0EE477AF1EE10FA0CDDDFED715A9E
:10FA00009FED716AF0EE676A77EEE57AF4EEC66A0A
:10FA1000F1EE10FAF6DCDFED6D6AF4EEE67AF1EE67
:10FA200010FA0CD5DFED675A9FED696AF0EE676A50
:10FA300077EEA57AF4EEC66AF1EE10FAF6D4DFEDB1
:10FA4000656AF4EEE67AF1EE10FA00F39C80DFEDE1
:10FA5000626AF4EEE67AF1EE10FA03D5DFED5B6A46
:10FA600076EEE77A27EEA76A9FED5C4ADFED5C4A07
:10FA7000F7EE006A9FED5B5AE6EE044ADFED5A5A54
:10FA800067EE863A9FED594AA6EE245AE6EE055AED
:10FA9000E3EEA57AF0EE665AE7EEC46AE7EE845A22
:10FAA000C6EEA53ADFED4B6A77EE267ABDEEE76A41
:10FAB00016EE103A2033402B68D8B4EEE67AF1EE19
:10FAC00010FA0CDD9FED3F6ADFED3F6AB0EE677A1A
:10FAD00077EEC67AB4EEE67AF1EE10FAF6DC9FED38
:10FAE0003B7AF4EEC77AF1EE10FA0CD59FED356A49
:10FAF000DFED376AB0EE677A77EE867AB4EEE67AB3
:10FB0000F1EE10FAF6D49FED337AF4EEC77AF1EE07
:10FB100010FA47DD9FED2A7A77EE677A67EEA76ADB
:10FB20009FED2E7A9FED2E4AB7EE006ADFED2D4A4B
:10FB3000B8EE003AA6EE874A9FED2B5A67EEA62A4A
:10FB4000B6EE007AE6EE844AA6EEA45AE2EE857A94
:10FB500036EE676A67EE837A26EE077AB7EE005ACA
:10FB6000C0ED043AC5EE256A26EE877A26EE866A4F
:10FB700066EEA77A80ED007A80ED016A80ED027A68
:10FB8000C0ED037A15E7DFED0E6A69E7B6EE007A9D
:10FB9000DFED177AB7EE006AE0E7F7EE003AF0EE35
:10FBA000635A7FE79FED0C7AF4EEC77AF1EE10FA14
:10FBB000B4D59FED067AAFE720A1070027D4D2364F
:10FBC000DB0F4940DB0FC940E4CB1641DB0F49C0D6
:10FBD000E4CB16C1DB0FC93FDB0FC9BF9A7C2E36C1
:10FBE000FAAF4FB93587083CA4AA2ABEF304353FC3
:10FBF00000000000FDEEC07A17EE903A2033402B53
:10FC000051D8DFED2A7AB4EEE70AF1EE10FA0CDDF6
:10FC1000DFED276A9FED277AF0EE407A30EE660A34
:10FC2000F4EEC77AF1EE10FAF6DCDFED237AB4EEEB
:10FC3000E70AF1EE10FA0CD5DFED1D6A9FED1F7A91
:10FC4000F0EE407A30EE260AF4EEC77AF1EE10FAC2
:10FC5000F6D4DFED1B7AB4EEE70AF1EE10FA18DD08
:10FC6000DFED127A37EEC00A60EE007ADFED155A4A
:10FC70009FED156ADFED156AA7EEA56A9FED147A70
:10FC800060EE275AE7EE866AA7EEA67AA5EE870A07
:10FC90007047DFED107AB4EEE70AF1EE10FAE3D523
:10FCA000DFED057ADEE79FED0C0A7047DB0F494078
:10FCB000DB0FC940E4CB1641DB0F49C0E4CB16C1D2
:10FCC000DB0FC93F9A7C2E36FAAF4FB93587083C17
:10FCD000A4AA2ABEDB0FC9BF000000009FED2F7A47
:10FCE00070EE077AFDEEE76A16EE903A2033402B6D
:10FCF00051D8B4EEC70AF1EE10FA0CDD9FED286A78
:10FD0000DFED286AB0EE677A77EEC67AB4EEE67A6F
:10FD1000F1EE10FAF6DC9FED247AF4EEC77AF1EEFC
:10FD200010FA0CD59FED1E6ADFED206AB0EE677AFF
:10FD300077EE867AB4EEE67AF1EE10FAF6D49FED1D
:10FD4000177AF4EEC77AF1EE10FA1ADD9FED187A01
:10FD500077EE677A27EEA77A9FED165ADFED165AEF
:10FD60009FED166AE7EE055ADFED156A27EE875A12
:10FD7000A7EE256AE7EE066AE5EE267AB0EE670A98
:10FD800070479FED107AF4EEC77AF1EE10FAE1D5E4
:10FD90009FED057ADCE79FED0C0A7047DB0FC93F4A
:10FDA000DB0FC940E4CB1641DB0F49C0E4CB16C1E1
:10FDB000DB0F49409A7C2E36FAAF4FB93587083CA5
:10FDC000A4AA2ABEDB0FC9BF00000000B5EE400A9E
:10FDD000F1EE10FA25D007EE902AF0EE406AF8EE28
:10FDE000670ADFED107A08B5034660EEA70A0846F9
:10FDF0004BB9FFF75DFDFCEEE66A16EE903A99B25C
:10FE0000BDE80840C8E5022B06D0032BF3D1FFF76D
:10FE10007FFDBDE8084087E5FEF786FFFEF790FF0F
:10FE2000E9E77047BD378635B5EE400AF1EE10FAC6
:10FE300002D1044B0B60704703280CBF024B034BED
:10FE4000F8E700BF21ED000865000000F1000000A8
:10FE5000D0ED0E7AF0EE405AB0EE605AF5EEC07A70
:10FE6000F0EE414AF1EE10FA08B503467DDC30EEC3
:10FE7000604AD3ED013A1A7864EE233A002A5DD144
:10FE800001F00102D3ED117A002A60D074EE677A96
:10FE9000B0EE445AD3ED0F0A87EEA40A83ED115A4F
:10FEA000F5EEC00AF1EE10FA54DCD3ED036A60EE11
:10FEB000266A93ED057A93ED106A25EE877A77EE40
:10FEC000067A77EEA37A77EEA67AF4EEE71AF1EEE9
:10FED00010FA54DC82FE670A70EE677A93ED045ADA
:10FEE000D3ED025A480783ED157AB0EE467A67EEF5
:10FEF000857AC3ED133A83ED126AC3ED146AE4EE1A
:10FF0000257A83ED160AA4EEA77A08D5F0EEC77A13
:10FF1000F0EEC66AF4EEE67AF1EE10FA32D583ED31
:10FF2000107A0A0700D408BDF4EEC71AF1EE10FAF1
:10FF300001DCC2FE471AC3ED101A08BD11F0010220
:10FF40004FF0000045FE047A1870002A9ED177EE2B
:10FF5000C57A9FE793ED035AB0EE641A03F12800C7
:10FF600057F0B2FF65EE006AA3E730EE600A183082
:10FF7000F0EE670A57F0A8FFB0EE404A79E7B0EE1E
:10FF8000610AA9E7B0EE467ACBE700BF0023012261
:10FF9000C3640270836403650364436443658362DE
:10FFA00083657047DFED1D7A80ED010AF4EE670A84
:10FFB000C0ED020A80ED031AC0ED051AF1EE10FA49
:10FFC00020DDB4EE670AF1EE10FA1BDD81EE007A57
:10FFD000C0EE207AF0EE006A77EE877A86EEA77A96
:10FFE00080ED047A0023012280ED0F2AC0ED0E2A55
:10FFF0000270C3648364036503644364436583627E
:020000040801F1
:1000000083657047DFED057A0023F4EEE70A0361AC
:10001000F1EE10FAD8BF8360E4E700BFBD37863544
:10002000B0EEC07AF0EEE06A86FE876AB5EE406A0E
:10003000F1EE10FA3DD0C6FEC75AC5EE867ADFED66
:100040001E2ADFED1E3ADFED1E4A9FED1E5A9FED80
:100050001E3AB7EE006A9FED1D4ADFED1D5AE7EE2E
:10006000E23AA7EE834AE7EEA34AA7EE846AA7EE38
:10007000A45AE7EE855AC5EE867AF4EEC76AF1EE29
:1000800010FAF5EEC00A44BF9FED127A77EE677A58
:10009000F1EE10FAB5EEC00A44BF9FED0F7A77EE8D
:1000A000677AF1EE10FA48BFF1EE677AB0EE670AB0
:1000B0007047DFED077AE0E739094E3DE3B59E3E34
:1000C00088FA163E45FE7F3F99FB243F69A2163E03
:1000D000A7DFA834DB0FC93FDB0F4940B7EE007A3A
:1000E000F0EEC07AF4EEC77A77EE676AF1EE10FAB6
:1000F0001DD89FED105AB1EEE67ADFED0F5A9FED55
:100100000F6ADFED0F6AE7EE855AA7EEA56AE7EE04
:10011000866A67EE266AB5EEC00AF1EE10FA44BFB1
:100120009FED087A77EE666AB0EE660A7047DFEDFB
:10013000066AF0E7306E99BC2716983D843459BEA4
:10014000A40DC93FDB0F494000000000B0FBF1F3F4
:1001500001FB130308463BB11946B0FBF1F301FB69
:1001600013030846002BF7D1704700BF44F25063D9
:10017000984203DD054B034418467047044B9842F0
:1001800002DA48F6A043F6E70346F5E76073FFFF9F
:10019000B0B9FFFF48F69F43984203DD054B034487
:1001A00018467047002802DA48F6A043F7E70346EE
:1001B000F6E700BF6073FFFF80EAE073A3EBE07334
:1001C0008B4203DB002803DD401A70470020704794
:1001D000FDD00844704700BF884203DB9042A8BFAF
:1001E000104670470846704700230361704770B59A
:1001F00003780446012B32D103691F4D1BB94268B5
:100200000AB92A684260D4ED067A013304F11C066B
:1002100077EE807A23613046C4ED067AFEF79CFDC6
:1002200062682B689B1AA268934218D9E06A94ED21
:100230000A0A50F039F8D4ED057AB4EEE70AF1EE87
:1002400010FA0DDD237B43B92A6830462361002371
:100250006260A361BDE87040C6E70323237070BDF0
:10026000D4ED047A0223D4ED066AF8EE677A86EEBE
:10027000A77A84ED067AF1E73C2601202DE9F041CA
:1002800004461C30254604F16402064650ED017A0E
:10029000B1EC010A77EE807A40ED017AFEF75CFD61
:1002A00018309042F2D12369274F013362682361ED
:1002B0003B689B1AA268934244D904F13008E86A6B
:1002C00095ED0A0A4FF0F0FFA845D4ED057A1AD053
:1002D000B4EEE70A1835F1EE10FAF0DD237B7BBBB4
:1002E0003A683046236162600022A261FFF77CFF1A
:1002F00004F134002263FFF777FF04F14C00A2649D
:10030000BDE8F04170E7B4EEE70AF1EE10FAE5DC83
:10031000D4ED047A0223D4ED066AF8EE677A86EE0D
:10032000A77AD4ED0C6A84ED067A86EEA77AD4ED2E
:10033000126A84ED0C7A86EEA77A84ED127A00E0D8
:1003400003232370BDE8F0813C26012010B4019CFA
:10035000401A511AA4EB030C5DF8044B00FB0CFC93
:100360009CFBF1FC0CEB0300704700BF30EE600A11
:1003700032EE612A71EE600A22EE002A82EE200A35
:1003800030EE210A704700BFDFEDE26AD1ED007A5E
:1003900037EEA67ABDEEC76A16EE103A2033402B30
:1003A00000F25882F4EEE67AF1EE10FA0CDDDFEDA1
:1003B000DB5A9FEDD96AF0EE476A37EE657AF4EEC4
:1003C000C66AF1EE10FAF6DCDFEDDE6AB4EEE67A2C
:1003D000F1EE10FA0CD5DFEDD15A9FEDD16AF0EEB7
:1003E000476A37EE257AF4EEC66AF1EE10FAF6D4D3
:1003F000DFEDC86AB4EEE67AF1EE10FA40F302825D
:10040000DFEDC96A36EEC77A67EE076ADFEDC74AE5
:100410009FEDC75ADFEDC75AA6EEA45A9FEDC66AF4
:1004200027EE264AE6EE855AA6EEA56AA4EE067ADF
:10043000F0EE474ABDEEE77A17EE103A2033402B34
:1004400000F205829FEDB87AF4EEC77AF1EE10FA69
:100450000CDD9FEDB26A9FEDB07AF0EE676A77EE41
:10046000C67AF4EEC76AF1EE10FAF6DC9FEDB57AC3
:10047000F4EEC77AF1EE10FA0CD59FEDA86A9FED65
:10048000A87AF0EE676A77EE867AF4EEC76AF1EE44
:1004900010FAF6D49FED9F7AF4EEC77AF1EE10FAD7
:1004A00040F3DB819FEDA07A77EE677A27EEA77A9B
:1004B0009FED9E5ADFED9E5A9FED9E6AE7EE055A2C
:1004C000DFED9D6A27EE874AA7EE256AE7EE066A0A
:1004D000E4EE267AB0EE675A91ED017ADFED8D7A7F
:1004E00077EE276ABDEEE66A16EE103A2033402B0F
:1004F00000F2A681B4EEE77AF1EE10FA0CDDDFED42
:10050000875ADFED857AB0EE666A76EEE56AB4EE7C
:10051000E76AF1EE10FAF6DCDFED8A7AF4EEE76ACC
:10052000F1EE10FA0CD5DFED7D5ADFED7D7AB0EEFD
:10053000666A76EEA56AB4EEE76AF1EE10FAF6D4D2
:10054000DFED747AF4EEE76AF1EE10FA40F39B8186
:10055000DFED757A77EEE66A66EEA67ADFED733A3E
:100560009FED734A9FED736AA7EEA34ADFED725ABF
:1005700066EEA73AA7EE846AE7EE865AE3EEA56A2E
:10058000B0EE666A66EEC52A24EEA63AFDEEC77A9C
:1005900017EE903A2033402B00F24F81DFED627A64
:1005A000B4EEE77AF1EE10FA0CDDDFED5C5ADFED28
:1005B0005A7AF0EE476A37EE657AF4EEE76AF1EEC2
:1005C00010FAF6DCDFED5F7AB4EEE77AF1EE10FABE
:1005D0000CD5DFED525ADFED527AF0EE476A37EE76
:1005E000257AF4EEE76AF1EE10FAF6D4DFED497AF7
:1005F000B4EEE77AF1EE10FA40F33A81DFED4A7A91
:1006000037EEC77A67EE077ADFED483A9FED484A42
:10061000DFED486AA7EEA34ADFED475A67EE273AB7
:10062000E7EE846AE7EEA65AA3EEA57AF0EE476AF3
:10063000D1ED027ADFED375A37EEA57ABDEEC74A23
:1006400014EE103A2033402B00F2EC80F4EEE57A01
:10065000F1EE10FA0CDDDFED313A9FED2F4AF0EEAE
:10066000475A37EE637AF4EEC45AF1EE10FAF6DC2C
:10067000DFED345AB4EEE57AF1EE10FA0CD5DFED89
:10068000273A9FED274AF0EE475A37EE237AF4EEE9
:10069000C45AF1EE10FAF6D4DFED1E5AB4EEE57A44
:1006A000F1EE10FA40F3FA80DFED1F5A35EEC77A0B
:1006B00067EE075ADFED1D1A9FED1D2ADFED1D3A8B
:1006C000A5EEA12A9FED1C4A67EE251AE5EE823AB7
:1006D000A5EEA34AA1EE847A25EE072A64EE871AD6
:1006E00026EE077A26EE821A26EEA10AFDEEE75ADA
:1006F00015EE903A2033402B00F28F80DFED0A5A3E
:10070000F4EEE57AF1EE10FA27DDDFED043A9FED25
:10071000024A19E0DB0FC93FE4CB1641DB0FC940A9
:10072000E4CB16C1DB0FC93FDB0F49409A7C2E3664
:10073000FAAF4FB93587083CA4AA2ABE00000000D2
:10074000DB0FC9BFDB0F49C0F0EE675A77EEE37AE3
:10075000F4EEC45AF1EE10FAF6DC5FED065AF4EE50
:10076000E57AF1EE10FA0CD55FED143A1FED144A5C
:10077000F0EE675A77EEA37AF4EEC45AF1EE10FA6F
:10078000F6D45FED185AF4EEE57AF1EE10FA40F384
:1007900090805FED1B5A75EEE77A27EEA74A5FED72
:1007A0001D5A5FED1D3A5FED1D0AE4EE253A67EE36
:1007B000845AE4EE230A5FED203AE4EE203AE5EEB7
:1007C000A37A64EEA74A65EE275A67EEC67AA6EECC
:1007D000A42AE6EEE51A31EE241A75EEC05A80ED31
:1007E000007AC0ED017AC0ED026A80ED031AC0ED17
:1007F000041AC0ED052AC0ED065A80ED072A80EDE7
:10080000083A70475FED326AB4EEE67AF1EE10FA1C
:100810007FF5FAAD5FED356AF4E55FED385AF0EE3D
:10082000657ADAE71FED3B2AF0EE421AB0EE420A93
:10083000B0EE421AB0EE427A58E75FED406AF7E652
:100840001FED423AF0EE432AB0EE436A9EE61FEDFA
:10085000455A41E65FED474AECE51FED477AF4EE75
:10086000C77AF1EE10FA7FF521AE1FED4A7A1BE64A
:100870005FED4D7AB4EEE77AF1EE10FA7FF5C2AE95
:100880005FED507ABCE65FED527AF4EEE76AF1EE86
:1008900010FA7FF561AE5FED557A5BE65FED585A71
:1008A000B4EEE57AF1EE10FA7FF502AF5FED5B5A38
:1008B000FCE65FED5D5AF4EEE57AF1EE10FA7FF5B5
:1008C0006CAF5FED605A66E70023036143618361AB
:1008D000C3610360036243628362C3624360036374
:1008E00043638363C3638360036443648364C36457
:1008F000C3607047D1ED016AF7EE000A91ED007A0E
:10090000F8EEE66AD1ED027AB8EEC77A90ED044AC5
:10091000F8EEE77AD0ED054A26EEA62A90ED065AC3
:10092000E7EE264AD0ED075AA7EE275A90ED080ABF
:10093000B0EE426AD0ED0A1AA7EE074AD0ED0C2AB3
:1009400075EE875A90ED0D3AA7EE076AD0ED0E3A94
:1009500090ED091AA7EE260AE6EEA71AC0ED054AA1
:10096000E7EE272AD0ED104AA6EEA73A80ED044A1A
:10097000E7EEA73A90ED0F4A31EE021A80ED065AE3
:1009800090ED0B2AA7EEA76A90ED115A34EE274A94
:10099000C0ED075A74EE874AD0ED125A35EE265A4A
:1009A00032EE262A80ED0F4A75EEA75AC0ED104AA6
:1009B00080ED115A80ED080A80ED091AC0ED0A1A7F
:1009C00080ED0B2AC0ED0C2A80ED0D3AC0ED0E3AF9
:1009D000C0ED125AD0ED004AD0ED025AE7EE064AB9
:1009E00090ED015AB0EE657A90ED134AA6EE865A64
:1009F00074EE206AA7EE867AD0ED037A37EE866A27
:100A0000C0ED136AC0ED004A80ED015A80ED036A23
:100A100080ED027A704700BF10B50024034684467B
:100A20008646002C00F00D81DEED006A012C9CED65
:100A3000007AD3ED007AE6EEC77AC3ED007A00F0D3
:100A40000F81DEED016A032C9CED047AE6EEC77A95
:100A5000C3ED007A6CD1DEED026A9CED087AE6EE19
:100A6000C77AC3ED007AD2ED007AD0ED044A90ED5A
:100A7000085AD0ED0C5A92ED017AD2ED026A92ED4D
:100A8000036AA7EEE47AE7EEC56AD0ED094AA7EE5D
:100A9000E56A90ED0D5AD0ED0E5AE7EE646AA5EEC8
:100AA000476AA5EEE66A81ED036A90ED0F5AC1ED43
:100AB000026AC6EE055AC1ED035A90ED0B6AE5EEE7
:100AC000C66AC1ED026A90ED0A5A81ED017A86EE9E
:100AD000856A81ED026AD0ED066AA6EE667A81ED3E
:100AE000017AD0ED076AA5EEE67A81ED017A90ED04
:100AF000055AC1ED007AC7EE056AC1ED016A90EDB5
:100B0000017AE7EE667AC1ED007A90ED027AE7EEBF
:100B1000467AC1ED007A90ED037AE7EE657AC1ED91
:100B2000007AD0ED006A87EEA67A81ED007A10BDDA
:100B30009EED007A022CDCED016AD3ED017AB1EE74
:100B4000476AE7EE667AC3ED017ADEED016A9CED55
:100B5000057AE6EEC77AC3ED017A40F0AC80DEEDAF
:100B6000046A012C9CED007AD3ED047AE6EEC77A94
:100B7000C3ED047A40F28780DEED056A032C9CED1C
:100B8000047AE6EEC77AC3ED047A7FD19EED066A59
:100B9000DCED086A93ED007AE6EE667AC7EE876AC6
:100BA000C3ED046A9EED086A012CDCED006AD3ED0A
:100BB000087AE6EE667AC3ED087A70D99EED096A86
:100BC000032CDCED046AE6EE667AC3ED087A07D101
:100BD0009EED0A6ADCED086AE6EE667AC3ED087AF5
:100BE00093ED086A032CD3ED0C7AC6EE076AC3EDC9
:100BF000086A9CED006ADEED0C6AE6EE667AC3EDEB
:100C00000C7A9CED046ADEED0D6AE6EE667AC3EDC1
:100C10000C7A07D19EED0E6ADCED086AE6EE667A84
:100C2000C3ED0C7AD3ED0C6AC6EE877AC3ED0C7A6D
:100C3000013414330EF1100E0CF1040C002C7FF46F
:100C4000F3AED3ED047A93ED007A93ED086AC7EE24
:100C5000876AC6EE077AC3ED046AC3ED087AE1E756
:100C6000DEED006A9CED016A93ED017AD3ED027A24
:100C7000A6EEC67A83ED017A9CED027AE7EE667AFB
:100C8000C3ED027A6BE793ED007A87E793ED007A84
:100C9000022CC7EE876AC3ED046AC9D082E7C7EEAB
:100CA000876AC3ED086AC3D09CED006ADEED0C6A6A
:100CB000D3ED0C7AB2E79CED027A032CD3ED027AE5
:100CC000E6EE077AC3ED027ADCED066A9EED017A64
:100CD000E6EEC77AC3ED027A7FF441AFDEED026A39
:100CE0009CED0A7AE6EEC77AC3ED027ABBE600BF56
:100CF00010B584B00C46024610306946FFF78CFEF2
:100D0000B6EE006ADDED006A01209DED017ADDEDB1
:100D1000027A66EE866A27EE067A67EE867AC4ED78
:100D2000006A84ED017AC4ED027A04B010BD00BF00
:100D3000F0EE407A9FED060ABEEE007A60EEA00A61
:100D400067EEA77A67EE877AC7EEA00A53F060BF16
:100D500054F82D4008B550F0A1FF07EE900AF5EECB
:100D6000C07AF1EE10FAACBFB1EEE70A9FED010ACE
:100D700008BD00BF0000000060EEA00AE0EE000A1F
:100D8000B1EEE00A704700BF21EE011AA0EEA01AF2
:100D9000A0EE001AB1EEC10A70472DE9F74F904658
:100DA0009DF8302005460F46002A0D9A14BF4FF0DB
:100DB00030094FF020091C1EBABF644201230023F2
:100DC00012F8011B01B12CB9A24663B100240D9E9B
:100DD000A41B12E0013CF3E7BD4204D24946284679
:100DE0000193C047019BBAF1010AF5D2EFE7BD427A
:100DF00003D228460193C047019B06EB040B16F86B
:100E0000011B0029F3D133B15446002C07DCBAF1A1
:100E1000000FA8BFD344584603B0BDE8F08FBD42D1
:100E200002D249462846C047013CEEE70FB437B529
:100E300006AB0A4D53F8042BD5E9E10101934DF0BF
:100E40003DF80446D5F8800305F0FDFD0028F9D0F3
:100E5000204603B0BDE8304004B070474061012037
:100E60000EB403B503AB084953F8042BCDE90030A9
:100E700001A84DF023F8019B00221A7002B05DF822
:100E800004EB03B0704700BFABED00080CB430B505
:100E90002C4CA5B0D4F88C331BB9D4F89033002B6C
:100EA00039D094F89433994206D9012303FA00F01B
:100EB000D4F8983318422ED0234B04A819684FF465
:100EC0007A73B1FBF3F203FB12132049FFF7C8FF5B
:100ED00004AB289A054603441D4903A8039329AB94
:100EE00002934CF0EBFF039B0246D4F88C03591C91
:100EF00003910A211970039B591C03910021197059
:100F000090B103681B6A03B19847D4F88C5304ACC2
:100F100014F8011B21B925B0BDE8304002B070477C
:100F2000284605F021FDF3E7D4F89033002BF2D0EA
:100F300002212A44FD200A44009104A923F044F927
:100F4000E9E700BF406101203C260120EE0F0708C1
:100F50004DED000830B54FF4004087B021F0D6F9D0
:100F60000446A0B34FF4004121F032FB02281CD10B
:100F7000226848F201039A4229D1234C00254FF4FC
:100F8000004084F830564CF0EBFB00B3D4F89C33AF
:100F900083421ED0D4F8783483422FD0D4F854350D
:100FA00098422ED0C4F8905311E00023022294F905
:100FB00004004FF40041CDE901234FF46122009277
:100FC0001A4621F06CFB104BC3F88C0328B907B00C
:100FD00030BD04F56773C4F890330C4B02210C4A02
:100FE000002004930B4B03930B4B02930B4B019389
:100FF0000B4B00930B4BFFF749FFE8E704F58F63BA
:10100000E9E704F25453E6E740610120FA0F0708CC
:101010000D1D0708031007080C1007081810070813
:101020001E100708860F0708174A033038B5D2F894
:10103000344604EB9003B3F5007F18D802F5C7657A
:10104000C2F8343602EB810220F00300C3F50073CE
:1010500005EB8404D2F8381E9B0008440421C2F832
:10106000380E0020094AFFF711FF204638BD002145
:10107000074A00240846FFF709FF064A136843F0B1
:1010800000731360F1E700BF4061012031100708D1
:10109000541007080000002003685A1C02601970F1
:1010A000090A03685A1C02601970704703685A1CC9
:1010B0000260197003685A1C02600A0A1A700368F9
:1010C0005A1C02600A0C090E1A7003685A1C02604E
:1010D0001970704703685A1C02600A0A1A70036884
:1010E0005A1C02601970704738B5044600681546EE
:1010F00056F004FB23682B44236038BD03685A1C58
:1011000002601878704703685A1C02601A4612F889
:10111000021B0260587841EA0020704702681146BD
:10112000531C10B50360D31C11F8024B01605178B9
:10113000036093781B0443EA0123111D23430160DC
:10114000D07843EA006010BDD1E900329A4206D05F
:101150005A1C0A6008B11B780370012070470020F8
:101160007047D1E9002310B59B1A04460846012BAD
:1011700004DDFFF7C8FF2080012010BD0020FCE740
:1011800030B50A440446914201D1002011E014F820
:10119000013BA3F14100192811F8010BA0F1410511
:1011A00098BF2033192D98BF20301B1A02D1002878
:1011B000E9D130BD1846FCE7028810B5A2F5FA6205
:1011C000C37840F2B5549108013B02F0030204FBDE
:1011D000013381780C24013904FB02120C49847913
:1011E00001EB42021821B2F888201344027901FB76
:1011F00003223C214379008901FB0233054A224442
:1012000001FB03224FF47A730021C2FB030110BDDE
:101210003C80060880436D382DE9F04190461F461A
:1012200005464FF47A7200234046394650F094FE4A
:10123000274B3C21034493FBF1F201FB1233AB71CA
:1012400092FBF1F301FB132240F2B5516A711822AF
:1012500093FBF2F402FB143394FBF1F201FB124412
:101260002B719300B4F5896F2EDA40F2DA229442A2
:101270002CDCB4F5B77FB4BF00210121154A18203A
:101280000B2600FB012232F81600A04201DD013ED0
:10129000F9D103F5FA6301344FF47A7240460B44F6
:1012A0002B80731CAB700C2303FB01660A4B394681
:1012B00003EB4606B6F88830E41A0023EC7050F0D1
:1012C0004BFE2A81BDE8F0810321D7E70221D5E753
:1012D00080BC92C7C48006083C800608F0B5274D44
:1012E0008DB006460F466C460FCD0FC40FCD0FC410
:1012F00095E80F0084E80F0016F0030339D164214C
:1013000096FBF1F201FB126242B94FF4C87296FBF0
:10131000F2F302FB1363003B18BF0123721EC3F1FB
:101320001D0369460024002A019340F26D13104604
:10133000B8BFB01C07257343013F03EBA0006FF05B
:10134000630392FBF3F318444FF4C87392FBF3F278
:101350001044063051F8042BA74202EB000393FB24
:10136000F5F0C0EBC000A3EB000004D1101A0DB0E3
:10137000F0BD0123D2E70134ECE700BF2481060869
:10138000094BD3F8C01ED3F8C42E51EA020308D08B
:10139000064B1B685B1842F10002C0E900320120D5
:1013A00070470020704700BF406101203C260120AB
:1013B00037B505466846FFF7E3FF044638B12846CF
:1013C000DDE90023FFF728FF204603B030BD40F2DF
:1013D00001132880A8806B80A8712881F4E700BFE2
:1013E000884270B54FF001045AD301FB04F4B0FBFE
:1013F000F4FC8C45F9D2002C4ED0BAB10025BCF1DA
:10140000000F1A4604FB1C00D4BF00260126B4FBC3
:10141000F1FE85BB7EBBA142354639D91A460CF197
:10142000300C02F801CB0023137070BD154605E0A7
:10143000A1427546F2D83446B0FBF6FCBCF1000F71
:101440001A4604FB1C00B4FBF1F606DCB5F1000EF5
:1014500018BF4FF0010E002DEAD0BCF1090F05F1C5
:101460000105CCBF57233023A1429C4402F801CB95
:101470001346E0D9D7E7BCF1090F05F10105CCBF50
:1014800037233023A1429C4402F801CB1346CAD82B
:101490007446B0FBFEFCB2E71A460023137070BD21
:1014A0008446002AAAD1C1E70028BCBF2D234042B0
:1014B00070B5B8BF01F8013B092884464FF001031D
:1014C00007DD03EB83035B00B0FBF3F2092AF8D8D6
:1014D00043B30024164EA6FB03508E46BCFBF3F22A
:1014E000002A4FEAD00003FB12CCD4BF002501250F
:1014F00054B94DB9092B2C4612D830320EF8012BB5
:1015000000238EF8003070BD092A04F101048CBF5D
:1015100057213021092B0A440EF8012B7146EFD9CF
:101520000346D8E78E4600238EF8003070BD00BF1A
:10153000CDCCCCCC90420B462DE9F041B0FBF2F67D
:101540000446154608D2124A05FB16441846135D98
:1015500000F8013BBDE8F0819642B6FBF2F706D2F7
:101560000B4A05FB1767D15D03F8011BECE7BA4294
:10157000B7FBF2F807D905FB1878054A12F80810EE
:1015800003F8011BEDE74046FFF7D4FF0346F2E7FF
:1015900094100708B5EEC00ADFED317A0023F1EEB2
:1015A00010FA70B5C8BF30EE270A86B0D8BF30EE4B
:1015B000670ADFED2C7A054603A902936E4620EEFA
:1015C000270ACDE90033FDEEC07A17EE904A84EA8F
:1015D000E470A0EBE4704CF03BFF002C03A8ACBF20
:1015E00020232D238DF800304FF0C4FE012827D092
:1015F00002282ED003281DD003A9304656F086FBC2
:1016000030464FF0B7FE044631462846033CE4B26C
:10161000224656F073F8002328462B554FF0AAFEB9
:101620002E22431C31192A54E81856F08BFB284609
:1016300006B070BD302303A930468DF80130DDE7D8
:1016400043F23002302303A9ADF801208DF80330B6
:10165000D3E743F2300303A93046ADF80130CDE7BC
:101660006F12033A00007A440378092B01D0202B33
:1016700005D110F8013F202BFBD0092BF9D02D2BE1
:1016800000F0AC802B2B78D0A3F13002B7EE000A2B
:10169000D1B209297AD8F2EE046ADFED5C7A07EE5E
:1016A000102A10F8013FB8EEC77AA3F13002D1B288
:1016B000A7EEA67A0929F0EE477AF0D92E2B69D049
:1016C00003F0DF03452B40F0868010B442782D2ACA
:1016D00000F091802B2A0DBF8278A2F130030130F7
:1016E000023008BFA2F13003092B7BD8002400236D
:1016F00003EB830302EB430310F8012FA2F1300147
:10170000303B0929F4D9B3F59A7F1A46B7EE007A2F
:1017100028BF4FF49A72072B09D91346DFED3C6AB4
:10172000083B27EE267A072BFAD802F00702DAB137
:10173000F2EE046A012A27EE267A15D0022A27EE55
:10174000267A11D0032A27EE267A0DD0042A27EE16
:10175000267A09D0053A27EE267A05D027EE267A92
:10176000012A18BF27EE267A002C3DD0C7EE877AD3
:101770005DF8044B20EE270A7047B7EE000A437865
:10178000A3F130020130D1B2092984D92E2BDFED2B
:101790001F7A95D143780130A3F13002D1B20929E3
:1017A0008ED8B2EE047AF0EE475A06EE902A10F880
:1017B000013FB8EEE66AA3F13002D1B2C6EE076A85
:1017C000092927EE257A77EEA67AEED903F0DF0312
:1017D000452B3FF47AAF20EE270A7047BFEE000A90
:1017E0004378CDE7B7EE007A67EE877A5DF8044B71
:1017F00020EE270A704782780230A2F13003092BCD
:1018000001D8012473E7B7EE007AAFE700000000CB
:1018100020BCBE4C0246037801E012F8013F202BA9
:10182000FBD0092BF9D0303B0020DBB2092B0AD8C2
:1018300012F8011F00EB8000303903EB4000CBB2FF
:10184000092BF5D970477047037801E010F8013F84
:10185000202BFBD0092BF9D02D2B06BF01304FF0E8
:10186000FF3C4FF0010C0178A1F13002D3B2092BFB
:101870004FF0000302D903FB0CF0704710F8011F72
:1018800003EB830302EB4303A1F13002D1B2092938
:10189000F0E7002310B5802804D893420AD2C85438
:1018A000581C10BD934205D060F07F04C009CC5491
:1018B0000133F0E74FF0FF30F3E770B5124C01222F
:1018C000124E00201249FDF7B5FF228862B1A31D18
:1018D000B34217D2A518B54214D2052A12D921460F
:1018E0002C46FDF7A7FFF0E721460222FDF7A2FFF5
:1018F00063880849C31A084A641A5842A2F8C84EB5
:10190000584170BD0020FCE701400008008000083D
:1019100000400008FC3F00084061012003682DE9F9
:10192000F04113440446406883421AD80D468E188D
:10193000002704F10C08B542606901D1BDE8F081CF
:1019400023695A1C23442261042A15F8011B1973C8
:10195000F1D118B941462046F9F718F8C4E90470E6
:10196000E9E74FF0FF30E9E7034AD2F8CC3E23EA3B
:101970000000C2F8CC0E70474061012003460649C2
:101980000648884201D3002070470288C2F30B0248
:101990009342F9D01430F4E7EC8D07081489070856
:1019A00042880B4613B5C2F30B02044600211846C9
:1019B000019256F0EDF8216903460A48814209D3A5
:1019C0000948019A814205D2184602B0BDE810408C
:1019D00055F094BE21B1184602B0BDE8104008474A
:1019E00002B010BDEC8D07089292070810B4B0F950
:1019F00002400B464288002C41685DF8044BBEBF94
:101A0000C2F30B02DBB203FB0211C9E730B5094B8D
:101A1000094CA34200D330BDB3F902205988002AF3
:101A200006DA5A68C1F30B01DD6800FB01222A6067
:101A30001433EEE714890708EC8D070802460144C9
:101A4000002030B512F8015B082480EA0503400845
:101A50006D0813F0010F1CBF80F08C03D8B2631E19
:101A600013F0FF04F1D18A42ECD130BD144901EBEF
:101A70008000806B70B500B30C2202FB001292F95B
:101A8000E930581C1AD092F8F100B0B1C81864259A
:101A900092F8F040142290F824616B4300201D1945
:101AA000013A344401EB4505B5F8285110FA85F0A8
:101AB000F5D11423B0FBF3F080B270BD0020FCE739
:101AC0004061012010B5427A044632B101464068B7
:101AD00051F80A3B98470023637210BD10B4447A52
:101AE000621C0444D2B24272A172037A934202D8B9
:101AF0005DF8044BE6E75DF8044B7047036810B5EA
:101B00001A790446022A02D1987A4EF08DFA0023FF
:101B10002360237110BD2DE9F0471F46AB4DAC4B40
:101B20009D4221D26C798C4240F06E812C798442A6
:101B300002D0002840F06881EC79944240F0648142
:101B40002C68DCB11C220021201D56F021F82560F4
:101B50002B792371012B95F80680C4F808802A7A26
:101B6000E26003D0022B0CD0002407E0E87A02F0F8
:101B700027FF6B7AA0612374AB7A63742046BDE8BB
:101B8000F087E87A02F01CFF95F90960A0612674DD
:101B9000A87A02F015FF6061002800F0318114235B
:101BA0008C4D734305EB0309EB58002B00F02881A3
:101BB00099F81230002B40F0EE8099F808004CF0B4
:101BC00005FB99F80830012103F01F025B09023B75
:101BD00001FA02F2032B08D8DFE803F0827C0276D8
:101BE0007D490B6923EA02020A61142306F1010A06
:101BF00003FB06535FFA8AFA587902F0E1FE814648
:101C000020B140F60A3380F808A0C380142303FBF8
:101C10000653D87902F0D4FE20B140F60A5380F87A
:101C200008A0C380142303FB0653987902F0C8FE72
:101C300020B140F60A4380F808A0C3801423484628
:101C40004FF0140918F0040803FB065309FB06596A
:101C500018BF4E215A7A08BF2E2102F091FE99F842
:101C6000070002F0ADFE99F80A202E2102F088FE4E
:101C700099F8060002F0A4FE99F80B200E2102F05C
:101C80007FFE99F8040050B102F09AFE20B140F6B0
:101C90000A6380F808A0C3800D2102F050FE1423CF
:101CA0007343EA58136823F0400313604B4B9A4286
:101CB0001CD103F58433596A41F480515962596A41
:101CC00021F4805159622AE043494B6923EA020218
:101CD0004A618AE740490B6A23EA02020A6284E702
:101CE0003D494B6A23EA02024A627EE73C4B9A4234
:101CF0000CD003F580639A425BD1374B196A41F4EB
:101D000000411962196A21F4004107E0324B196A57
:101D100041F480411962196A21F4804119625368C3
:101D2000B8F1000F43F4805314BF00200220536029
:101D300013685B0615D4116821F47F4121F0BF01BF
:101D4000B8F1000F08BF41F00101014341F44571B2
:101D50001160536823F4706323F0040343F4E063D9
:101D60005360D36923F40063D361136843F04003E5
:101D70001360536843F480535360142303FB0653EA
:101D8000187918B102F01CFE02F0CEFD142303FBFB
:101D900006550123AB74606920B10E238771C371AE
:101DA000002303720D2102F0CAFD606902F0BCFD40
:101DB000E4E60C4B9A4217D1074B596A41F40051A3
:101DC0005962596A21F400517CE700BFE80100081C
:101DD0006803000800000120003802400030014084
:101DE0000038004000340140084B9A4297D1084B1C
:101DF000596A41F480115962596A21F4801161E7EE
:101E00002046FFF77BFEAFE60C3589E60050014027
:101E10000038024073B50279022A38D190F91030A7
:101E2000142603200025734302AE8DF8030001241D
:101E300031441A488DF80050C3588DF801408DF890
:101E4000022011F8086C16498B4222D0A1F5784186
:101E50008B4220D001F580618B4205D0114A93421C
:101E600014BF4FF0FF3203221968142421F04001FF
:101E700004FB02021960D068196821F0380250F89A
:101E800026100A431A601A6842F040021A6002B033
:101E900070BD2A46E8E72246E6E700BF00000120C1
:101EA0000030014000340140C36910B5044623B935
:101EB00009211420FFF7B8F8E061E06910BD10B502
:101EC00004460068FFF7F0FF837853B183885BBA5C
:101ED000E381C3885BBA2382038901205BBA6382F2
:101EE00010BD1846FCE710B500680C46FFF7DCFF94
:101EF00083784BB1438922220120DBBA93FBF2F3B2
:101F000003F26D13238010BD1846FCE710B504469C
:101F10004FF4FA7004F018FE6069BDE8104002F05A
:101F200003BDF7B515461E46142290F9103004463D
:101F300053430E4AD75883689A0704D440690191E5
:101F40004EF02CF8019938464EF06AFC33462A468A
:101F500000213846F9F76AFBA3689B0702D42046A4
:101F6000FFF7D4FF012003B0F0BD00BF0000012047
:101F7000F7B507791646012F0AD0022F15D18468CC
:101F8000E40758BF41F0800103B0BDE8F040C8E766
:101F9000826802F00102CDE900620A46417C90F9B4
:101FA0001000F8F7E9FE03B0F0BD0020FBE7F7B53D
:101FB00015461E46142290F91030044653430E4A2B
:101FC000D75883689A0704D4406901914DF0E6FF21
:101FD000019938464EF024FC334600222946384603
:101FE000F9F724FBA3689B0702D42046FFF78EFF76
:101FF000012003B0F0BD00BF00000120F7B5077954
:102000001646012F0AD0022F15D18468E40758BF65
:1020100041F0800103B0BDE8F040C8E7826802F0FB
:102020000102CDE900620A46417C90F91000F9F7FF
:1020300067F803B0F0BD0020FBE713B506236A463E
:10204000F7210068FFF7DAFF134BE8B19DF80110A4
:102050009DF8002009019DF8034041EA02319DF8F6
:10206000022041EA12119DF8042012019966C3F87A
:10207000D01E42EA04329DF8054042EA14129A64E6
:10208000C3F8D42E02B010BDD3F8D02E9A66D3F880
:10209000D42E9A64F6E700BF40610120032307B500
:1020A000194601AA0068FFF7A9FFA0B19DF8043006
:1020B0009DF904209DF805101B04002A43EA012322
:1020C0009DF80610B4BF4FF07F4200220B4313432C
:1020D000024AC2F8E43003B05DF804FB406101201D
:1020E00007B5032301AA00210068FFF787FFA0B10D
:1020F0009DF804309DF904209DF805101B04002A6A
:1021000043EA01239DF80610B4BF4FF07F4200223E
:102110000B431343024AC2F8C83003B05DF804FB16
:102120004061012070B5066805463046FFF7BCFEE9
:102130000446021D0E233B213046FFF75FFFA070CF
:1021400040B1A3895BBAAB83E3895BBAEB83238A93
:102150005BBA2B8470BD13B5044600686A460379E8
:10216000022B4FF006030CBF43210321FFF746FF6C
:1021700018B9E086A06302B010BDBDF800305BBAAC
:10218000E386BDF802305BBA6387BDF804305BBA02
:102190002387F0E713B5062304466A461121006839
:1021A000FFF72CFF18B9E086A06302B010BDBDF99F
:1021B0000030F7EE086A07EE103AB8EEC77A27EE5D
:1021C000267ABDEEC77A17EE103AE386BDF90230E3
:1021D00007EE103AB8EEC77A27EE267ABDEEC77A38
:1021E00017EE103A2387BDF9043007EE903AF8EE67
:1021F000E77A67EEA67AFDEEE77A17EE903A638704
:10220000D3E7002313B5C386044683636A460623D7
:1022100003210068FFF7F2FE78B1BDF8003003EB50
:102220004303E386BDF902305B4203EB430323879C
:10223000BDF8043003EB4303638702B010BD73B5F0
:1022400090F9103015461422044653430C4AD658D0
:1022500083689A0704D4406901914DF09FFE01996B
:1022600030464EF0DDFA294630464EF0D9FAA368E2
:102270009B0702D42046FFF749FE012002B070BD43
:10228000000001207FB503790D46012B0AD0022BF7
:1022900019D18368DB0758BF01F07F0104B0BDE8A6
:1022A0007040CCE781688DF80F200DF10F0201F02E
:1022B000010100922A460191417C90F91000F8F743
:1022C0005BFD04B070BD0020FBE7012258210068CF
:1022D000D8E7012248210068D4E73122F4210068C0
:1022E00008B5FFF7CFFF012008BD022208210068D2
:1022F000C8E7012208210068C4E7F022FF21006836
:10230000C0E7B422FF210068BCE7CA43006841EA85
:102310000212D221D2B2B5E70A460068A521B1E780
:102320005521F9E79622FF210068ABE70A460068CD
:102330008721A7E7C901006801F080027821A1E7A1
:10234000F7B5C16A0446424F056890F82900B7FB0B
:10235000F1F189B24AF0CCFE4388064600212846B6
:10236000B7FBF3F76763FFF755FD80226B21284623
:10237000FFF788FF962004F066FC032268212846B8
:10238000FFF780FF962004F05EFC03226B212846B5
:10239000FFF778FF0F20002104F044FC10226A218F
:1023A0002846FFF76FFF0F20002104F03BFC0022BE
:1023B0006C212846FFF766FF0F20002104F032FC55
:1023C000727919212846FFF75DFF0F20002104F0E4
:1023D00029FC18221B212846FFF754FF0F2000215B
:1023E00004F020FC18221C212846FFF74BFF0F2089
:1023F000002104F017FC32791A212846FFF742FF2A
:102400000120002104F00EFC03212846FFF702FD05
:1024100006236A4643212068FFF7F0FD58B1BDF856
:1024200000305BBAA383BDF802305BBAE383BDF82A
:1024300004305BBA238494F91E30013306D194F939
:102440001C30013302D1062004F04AFC03B0F0BD79
:1024500040420F00F8B5C16A05462B4F046890F85A
:102460002900B7FBF1F189B24AF042FE43880646E3
:1024700000212046B7FBF3F76F63FFF7CBFC802208
:102480006B212046FFF7FEFE642004F0DCFB0722F0
:1024900068212046FFF7F6FE642004F0D4FB0022FA
:1024A0006B212046FFF7EEFE642004F0CCFB0122F6
:1024B0006B212046FFF7E6FE0F2004F0C4FB182234
:1024C0001B212046FFF7DEFE0F2004F0BCFB182284
:1024D0001C212046FFF7D6FE0F2004F0B4FB327912
:1024E0001A212046FFF7CEFE0F2004F0ACFB7279D4
:1024F00019212046FFF7C6FE642004F0A4FB204605
:102500000321BDE8F84085E440420F0010B5782271
:10251000044600210068FFF7B5FE052004F093FB98
:10252000202201212068FFF7ADFE052004F08BFB7F
:10253000002202212068FFF7A5FE642004F083FB3F
:10254000012010BD10B52422044641210068FFF788
:1025500099FE80B1202230212068FFF793FE50B110
:10256000062231212068FFF78DFE20B100223421A0
:102570002068FFF787FE052004F065FB012010BDF1
:1025800010B5072204460A210068FFF77BFE0520EC
:1025900004F059FB242241212068FFF773FE052037
:1025A00004F051FBC02242212068FFF76BFE05209A
:1025B00004F049FB012010BD10B504460022212182
:1025C0000068FFF75FFEFC2220212068FFF75AFE1B
:1025D000402224212068FFF755FE0C222321206889
:1025E000FFF750FE002222212068FFF74BFE01205A
:1025F00010BD10B50122044610210068FFF742FE0D
:1026000040B1142004F01FFB2068A0221121BDE876
:10261000104037E610BD10B5012204460B210068BA
:10262000FFF730FE20B11D2209212068FFF72AFEA6
:1026300000F0010010BD044B0246D3F8D80E08B1DB
:1026400080211FE6704700BF4061012073B590F9FB
:10265000103015461422044653430E4AD658836858
:102660009A0704D4406901914DF098FC01993046D5
:102670004EF0D6F80123002229463046F8F7D6FF5F
:10268000A3689B0702D42046FFF740FC012002B05C
:1026900070BD00BF0000012073B503791646012B01
:1026A0000AD0022B15D18368DB0758BF41F08001A7
:1026B00002B0BDE87040C9E7826802F00102CDE9CE
:1026C00000620A46417C90F91000F8F719FD02B04B
:1026D00070BD0020FBE7F8B504460E461546071D01
:1026E0003A46FF212068FFF7D7FF30B116B12379B2
:1026F000DB07F5D40DB123792B70F8BD0022012141
:10270000E9E710B50446FFF7FCFD18B12046BDE827
:102710001040F3E710BD10B50446FFF7FDFD18B1FA
:102720002046BDE81040E9E710BD73B50546CDE988
:102730000023FFF7E6FFA8B12846FFF7F1FD88B1B7
:102740002846FFF7DBFF68B16E46082416F8011B28
:102750002846FFF7E0FF28B1013C14F0FF04F5D153
:1027600002B070BD0020FBE7CC21D4E770B506466F
:102770000C468D18AC4201D1012006E014F8011B73
:102780003046FFF7C8FF0028F4D170BD38B50546C4
:102790001446FFF7CBFD2846FFF7B0FF20B11CB170
:1027A0002B79C3F34013237038BD10B50446FFF7EF
:1027B000A8FF38B12046FFF7D7FF18B12046BDE883
:1027C00010409BE7002010BD2DE9F04F002587B099
:1027D000804604930195CDE90212039B4046EC002C
:1027E00003EBC50AFFF78DFF024600286CD00022DC
:1027F00001214046FFF76FFF0246002864D098F899
:102800000430990760D5F0214046FFF784FF024667
:10281000002859D0A4F108024FF0000B0127039BB8
:102820005E4613443C460593029B002B54D0082C73
:1028300052D804F1FF3943FA09F909F00109494670
:102840004046FFF777FD024600283DD000220121D7
:102850004046FFF740FF0246002835D098F80410A4
:1028600001F0600CC809BCF1600F16D0029B1BB1CF
:10287000082C01D8814527D1002841D01AF806102C
:1028800039437F0001340AF8061017F0FF07E4B25D
:10289000CAD10136F6B2082E1CD1402C10D907211E
:1028A00050460592FFF7CAF89AF80710059A814238
:1028B00006D10135EDB2BBF1000F05D0CDF804B063
:1028C000049B1B78AB4288D8049B10461D7007B050
:1028D000BDE8F08F0127A7E75DB1019BA34208D9AE
:1028E000059B9A5D174214BF4FF001094FF0000994
:1028F000A5E7019B1B1BD3F1000949EB03099EE7E8
:10290000880940EA511111F0010F1AF8061008BFAA
:10291000A34621EA0701B4E7C90138B501F08001F7
:1029200004461546FFF706FD08B9002038BD002211
:1029300001212046FFF7CFFE0028F6D023795B095E
:102940002B70F3E710B5021D0446FF210068FFF766
:10295000A3FE18B12079C04300F0010010BD38B5C6
:102960000446154600680A46E121FFF78BFC28B1B2
:102970002A462068FF21BDE838408DE638BD0A466A
:10298000C321ECE738B5021D0D46F0210446FFF7E0
:10299000E6FF08B123792B7038BD0A46E121DEE756
:1029A00038B504460D46FFF7BDFC40B12046FFF7A1
:1029B000A5FE20B129462046BDE83840EDE70020BD
:1029C00038BD70B506460C468D18AC4201D10120C9
:1029D00006E0214630460134FFF7E2FF0028F4D13B
:1029E00070BDF7B515460DF107021C4606460F46A9
:1029F000FFF752FE9DF8073005EA0302A24208D015
:102A000023EA050239463046224303B0BDE8F040D0
:102A100038E403B0F0BD09230C211A4630B5044652
:102A200087B0FFF7DEFF282004F00DF901AA082186
:102A30002046FFF731FE9DF904209DF80430002A5E
:102A400003DB0025284607B030BD5D06F9D512230B
:102A500001AA10212046FFF7D1FA05460028F0D040
:102A60009DF805209DF804301109120241EA031176
:102A7000DB09544B02F4706218BFA1F580511005B8
:102A80009DF8070019839DF8061041EA02019DF8A0
:102A9000082048BFA1F580511201598342EA003253
:102AA0009DF8091042EA11101203BDF80A204FEAFE
:102AB000014148BFA0F5801052BA01F47021D861DD
:102AC00092B20A43090348BFA2F580121A62BDF808
:102AD0000C2052BA91B21204BDF80E2048BFA1F5E5
:102AE000803152BA9984100491B2BDF8102048BFC9
:102AF000A1F5803152BAD98491B21204BDF81220E6
:102B000048BFA1F5803152BA1985100491B2BDF8C1
:102B10001420204648BFA1F5803152BA598591B2A0
:102B200012044FF0070248BFA1F5803199850023B8
:102B30000821FFF756FFA5220E212046FFF7A2FB32
:102B400096220F212046FFF79DFB0222622120469C
:102B5000FFF798FB00220E212046FFF793FB00228F
:102B60000F212046FFF78EFB022307220821204673
:102B7000FFF737FF282004F066F85423204606218B
:102B80001A46FFF72EFF0DF1030228212046FFF71A
:102B900083FD9DF803302046072123F07F0343F097
:102BA00054031A46FFF71DFF0C23204609211A463D
:102BB000FFF717FF0723082120461A46FFF711FFEA
:102BC00040E700BF4061012013B504466A46082172
:102BD0000068FFF761FD9DF8003013F010037ED010
:102BE00006236A4600212068FFF708FA002874D0FF
:102BF0009DF801309DF800201B029DF804109FED08
:102C0000396A03EB02439DF8022009021A441C02B0
:102C10009DF8033048BF02F17F4201EB03419DF86C
:102C2000053007EE902A0B440902F8EEE77A48BF18
:102C300003F17F43C7EE866A07EE903A2A4BB3F959
:102C40002C20B8EEE77A07EE902AB3F92820F8EEA8
:102C5000E77AC7EE065A06EE102AB3F92420B8EE3A
:102C6000C66AA6EEA76AD3ED087AB8EEE77AD3ED86
:102C7000077AF8EEE77AA6EE867A26EEA55AE6EE11
:102C8000877A07EE102AB3F92A20B8EEC77A06EE43
:102C9000102AB3F92620B8EEC66AE5EE877A07EE69
:102CA000102AB3F91820B8EEC77AA6EE867AF6EEA7
:102CB000006AE5EE077A07EE102AB3F91A20B8EE9B
:102CC000C77AC3ED0C7A07EE902AF8EEE77A67EE42
:102CD000A57AE7EE267AC3ED0D7A02B010BD18464C
:102CE000FBE700BF000078484061012013B50022D7
:102CF00004460A210068FFF7C5FA142003F0A3FF79
:102D00000F220A212068FFF7BDFA0A2003F09BFF7B
:102D1000032301AA10212068FFF770F90A2003F0AD
:102D200092FF00220A212068FFF7ACFA0A2003F084
:102D30008AFF0DF1030202212068FFF7ADFC0DF1BF
:102D4000030209212068FFF7A7FC01220A2120685D
:102D5000FFF798FA012002B010BD30B5002385B00E
:102D600004460221C3860DF1070283630068FFF762
:102D700093FC18B90025284605B030BD9DF80730F2
:102D8000DB07F7D5062302AA03212068FFF736F9EF
:102D90000DF1070209212068FFF77EFC0546002897
:102DA000E8D09DF8073013F00C0FE3D1BDF80830E0
:102DB00001220A212068C3EB83339B00E386BDF820
:102DC0000A309B002387BDF80C30C3EB83339B0094
:102DD0006387FFF757FACEE71FB5002304460DF1CE
:102DE0000702272100688DF80730FFF755FC68B10E
:102DF0009DF8073013F0080320D0062302AA2821EB
:102E00002068FFF7FBF818B9E086A06304B010BD96
:102E1000BDF90830002BB8BF03339B10E386BDF922
:102E20000A30002BB8BF03339B102387BDF90C3049
:102E3000002BB8BF03339B106387E7E71846E5E72D
:102E40001FB5002104460DF10702C18681630068A9
:102E5000FFF722FCC0B19DF8073013F0080315D02E
:102E6000062302AA01212068FFF7C8F860B1BDF867
:102E700008305BBAE386BDF80A305BBA2387BDF839
:102E80000C305BBA5B42638704B010BD1846FBE7A9
:102E900030B5002585B004460621C5860DF1070230
:102EA00085630068FFF7F8FBA0B19DF8073013F0C9
:102EB000040311D0062302AA29462068FFF79EF8D2
:102EC00040B1BDF80830E386BDF80A302387BDF86D
:102ED0000C30638705B030BD1846FBE70368DB6B39
:102EE00013B504462BB923685B6B3BB9FF23E38220
:102EF00002E098470028F6D102B010BD214601A893
:102F000098470028F2D0BDF80630013B9BB2EEE7AF
:102F1000036810B59B680446984701236374FF2338
:102F2000A37410BD036810B504461B689847236856
:102F300020469B689847E37C0133E37410BD036827
:102F400010B504465B689847236820469B689847FD
:102F5000E37C013BE37410BDF0B5044685B00D463B
:102F60001846164603934EF005FA226828440021BD
:102F7000E673A07320460091294657693246039BA9
:102F8000B84705B0F0BD30B5046885B0E469089D68
:102F900034B10DB90DF10F050095A04705B030BD56
:102FA0002046FBE703689B6A184738B58B680446E0
:102FB00001600D4698470B4B2361002323752B6B53
:102FC00013B1204698472075074B93F8DC3E1BB1A0
:102FD000237D23F00103237500232046E382BDE80F
:102FE00038407BE70001FF004061012003681B6857
:102FF00003B11847704703685B6803B1184770470F
:1030000003681B6A03B11847704703685B6A03B122
:103010001847704730B40468A46A14B1A44630BCA1
:10302000604730BC704730B40468E46A14B1A44609
:1030300030BC604730BC704703685B6C03B1184715
:10304000704703689B6C03B11847704703689B6F18
:1030500003B1184770470368D3F8803003B11847AD
:1030600070470368D3F8843003B11847704703688A
:10307000D3F8883003B11847704721B10B68D3F8F3
:103080008C3003B118470020704710B5B0204FF4C2
:103090008064FFF7D0FA4020FFF7CDFA0020FFF759
:1030A000CAFA1020FFF7C7FA013C00204CF0F8FEE6
:1030B000A4B2002CF8D110BD503910B50446C8B2E6
:1030C000FFF7B9FA04EB440004EB4404400000F0BD
:1030D0000E00FFF7B0FAC4F3C300BDE81040103093
:1030E000FFF7A9BA503808B5C0B2FFF7A4FA00201C
:1030F000FFF7A1FA1020BDE80840FFF79CBA38B5E9
:103100000524094B04FB0030A0F1A005013C15F893
:10311000010B4CF0C5FE14F0FF04F7D12046BDE8CA
:1031200038404CF0BDBE00BF5481060810B5441EA7
:1031300014F8010F00B910BDFFF7E1FFF8E738B54B
:1031400000221E2331210120FEF7E5FC3C4BC3F891
:10315000D80E10B90024204638BDAE20FFF76BFA18
:1031600004460028F6D0D4204FF48065FFF763FAB8
:103170008020FFF760FAA820FFF75DFA3F20FFF7F5
:103180005AFAD320FFF757FA0020FFF754FA4020ED
:10319000FFF751FA8D20FFF74EFA1420FFF74BFA94
:1031A000A120FFF748FAC820FFF745FADA20FFF719
:1031B00042FA1220FFF73FFA8120FFF73CFACF20B6
:1031C000FFF739FAD920FFF736FAF120FFF733FA83
:1031D000DB20FFF730FA4020FFF72DFAA420FFF79D
:1031E0002AFAA620FFF727FAAF20FFF724FAA62035
:1031F000FFF721FAAE20FFF71EFA2020FFF71BFA97
:103200000020FFF718FAB020FFF715FA4020FFF76B
:1032100012FA0020FFF70FFA1020FFF70CFA013D19
:1032200000204CF03DFEADB2002DF8D18120FFF71B
:1032300002FAC820FFF7FFF9AF20FFF7FCF98AE791
:1032400040610120FBF7DABEFBF7D8BEFBF7D6BE24
:10325000FBF7D4BEFBF7D2BEFBF7D0BEFBF7CEBE6A
:1032600030B1006800F13F4000F57E00800A7047F1
:103270004FF0FF30704790F85F3230B53BB990F8AF
:103280005D12012490F85E32DAB2914200D830BD6E
:1032900004FA03F2B0F8665201332A43A0F866221A
:1032A000F2E7437913F001031FBFD0E90732C0688A
:1032B0009B1A00F1FF3014BF18401846704743793D
:1032C00013F002031FBFD0E9093200699B1A00F115
:1032D000FF3014BF98431846704710B54379014634
:1032E00013F001030DD0FFF7DCFF60B10A6A4B69F0
:1032F000C8689B5C0132B2FBF0F4DBB200FB142225
:103300000A62184610BD0346FBE743799B070AD5BE
:10331000436A8269D154436A02690133B3FBF2F113
:1033200002FB11334362704741717047D0E90920B5
:10333000131A584258417047014B1B685B68184785
:10334000DC790120024B08301B689B68184700BFDE
:10335000DC7901200120704701207047012070476F
:103360000120704731B10C4BD3ED007AF8EEE77ACB
:10337000C1ED007A72B1094BDFED096A1B68A3F554
:10338000D543333B07EE903AF8EEE77A87EEA67A1C
:1033900082ED007A704700BFE4810120E8810120BE
:1033A0000000C8420120704701207047704700BFED
:1033B00040F2FF72034B914203EBC000A8BF1146DD
:1033C00081807047B8970120154B164A9B79032BD3
:1033D00082F860301AD9191F022914D8052B17D08A
:1033E000062B14BF4FF47A614FF47A510E4B002034
:1033F000B3FBF1F39FED087B0C49D06682ED1C7B9B
:10340000C2E9191370470A4B53667047094BFBE733
:103410004FF4FA51EAE700BF00000000000000008E
:1034200058750120B897012040420F00B1330108C0
:10343000AD33010871430108034B03EB8000836F38
:103440000BB19B6819607047B8970120084AD2F801
:10345000B8305BB140B1B2F8BC00064A9968B2FB23
:10346000F0F35B100B6070479B681860704700BFFB
:10347000B897012040420F0007B50DF10702FFF792
:103480000BF9034B18709DF8070003B05DF804FBBF
:103490009016012008B5FEF7F5FE014B187008BD27
:1034A00090160120F8B5144E41F0010200210446A7
:1034B000124FFFF7EFFF3568C7F8C05013212046C1
:1034C000FFF7DAFF10F007000BD001220B21204696
:1034D000FFF7E0FF002220461146FFF7DBFF012047
:1034E00008E0D7F8C420002AE8D033689BB25B1B01
:1034F0009A42E3D2F8BD00BF3C260120B8970120D4
:103500000C4A13787BB10C4B93F8C81059B193F85F
:10351000C91059B150680021FA2883F8C910A8BF12
:103520004FF0FF3070476FF0010070476FF00200FE
:10353000704700BF90160120B89701200B4B93F8FD
:10354000CA206AB193F8CB206AB1002283F8CB205D
:10355000074B9868B0F5967FA8BF4FF0FF307047D3
:103560006FF0010070476FF002007047B8970120BC
:1035700090160120014B1B685B681847D079012029
:10358000014B1B689B681847D0790120014B1B68D1
:10359000DB681847D0790120014BD868704700BF1D
:1035A00090160120044B93F8CC3013B1034B1869EB
:1035B00070476FF001007047B89701209016012006
:1035C00020B10078B0FA80F04009704701207047C0
:1035D0002DE9F04FA54D0026A7B00A2405F1D00C27
:1035E00095F814113346B646674605F5867A9FE08E
:1035F00002EBCE0205EB4200C2F30726D7B2B0F8C9
:103600001801019646075FFA80FE4FEA102B40F141
:10361000C480480614D403F1020941F04001B9F115
:103620008C0F00F2FB8026A803F1010803444FF041
:10363000040003F88C0C26AB98444B4608F88C1C0D
:1036400003F102080198B8F18C0F40F0020900F272
:10365000E58026A8184400F88B9C4FF0050900F877
:103660008C9C03F10409B9F18C0F00F2D78026AECF
:103670004FEA8E0EB0444FF006065FFA8EFE08F851
:103680008C6C03F1060800F8897CB8F18C0F00F20D
:10369000C58026AEB1444FF0070609F88C6C00F8DF
:1036A00087EC03F1080EBEF18C0F00F2B78026AE56
:1036B0004FF00509B044019E08F88C9C00F8856C19
:1036C00003F10A068C2E00F2A9800DF198094FF043
:1036D0000608CE440EF88C8C00F8837C03F10C07AE
:1036E0008C2F00F29B804FF007004E440B3306F8FE
:1036F0008C0C4846034403F88CBC3B465709012018
:1037000002F01F06013C00FA06F65CF8270020EAEA
:1037100006004CF8270000F08480561CB6F5F07FB8
:103720007FD272090CEB82074FEA820E574578D29E
:103730004FF0FF3206F01F06386802FA06F606EA76
:10374000000292FAA2F2B2FA82F2D2B2202A7FF4F6
:103750004FAF381D504518D2454AD21B083722F0CA
:103760000302174401E0B8420FD006460430326825
:1037700092FAA2F2B2FA82F2D2B2202AF3D0A6EBE7
:103780000C0612EBC6027FF535AF85F81411002B3D
:1037900049D1184627B0BDE8F08F4E0603D401F09A
:1037A0003808F04515D021F0780103F102080143F3
:1037B000B8F18C0FC9B231D826A803F1010E034429
:1037C0004FF0040003F88C0C26AB9E4443460EF8E1
:1037D0008C1C981C8C2821D826AE06EB030E019E6B
:1037E0000EF88B6C4FF005060EF88C6C1E1D8C2E9F
:1037F00014D80DF1980840444FF0060800F88C8C5E
:103800000EF8897C9F1D8C2F08D826A80533064406
:103810004FF0070006F88C0C26A86BE76FF000430A
:103820006CE785F81411D5F80C41124894F9102072
:10383000A16802EB820250F822508A070FD503AA32
:1038400000212846F7F7F2FEA3689B0703D5012065
:1038500027B0BDE8F08F2046FEF758FBF7E7606918
:1038600001934CF09BFB019BE9E700BFB897012057
:10387000BF980120000001206E4B2DE9F04F93F816
:103880001251C7B005B1FEE76A4A012304460E464D
:1038900092F8137182F8123107F0F707D2F80C3161
:1038A00082F8137102931B79012B00F0A980022B7F
:1038B00040F0A48002983A46836813F0010118BFD3
:1038C000294605ADFEF7BBFC5A4BD3F80C310293E9
:1038D000FF2C4FF009036C704FF002008CBFA4085E
:1038E0004FF000084FF0000C4FF00A0988BF04F0B9
:1038F000C0080DF1150A4FF00B0B2B7011E0BEF54F
:10390000827F05F8009016F80C700AF8002016D88F
:103910000CF1010C05F804B070466F54BCF1360F81
:1039200016D0841C48EA0C02034600F1040EB4F5DC
:10393000827FD2B200F1030103F10603DFD90CF15B
:10394000010C6FF0004E3C4BBCF1360F7046E8D1D5
:10395000B3F5827F9DBF08230DF11502A0216FF002
:1039600000439EBF05F80E30831C11540298334962
:1039700090F9102002EB820251F8224082689207EF
:1039800052D52A4620460021F7F750FE029B9B683D
:103990009B0745D5274B0DF11304294DD3F80C0196
:1039A0000379012B18D0022B0CD12246A021FEF75F
:1039B0004DFE18B1237813F0200319D01D4BD3F816
:1039C0000C010379D5F8A810012BB5F8AC204E698D
:1039D00082EA06024A61E6D18668A022417C06F0AE
:1039E000010690F91000CDE90046F7F789FBE0E702
:1039F000104A82F8123147B0BDE8F08F05AD67E795
:103A000002982A46816801F00105014690F91000EC
:103A1000497C019505AD2F700095F7F7ADF953E797
:103A20000298FEF773FAB5E7406903934CF0B6FAD3
:103A3000039BA6E7B8970120010000800000012049
:103A400020700120C36B59680A6848790349136ADA
:103A500051F820100B431362704700BFCC86060854
:103A6000836837B51C686379DB0727D5A57994F897
:103A70005C3205F001010D4613B3E06B03685B682F
:103A80001A68D36A5B08536294F86D32012B07D031
:103A900094F8613223B1B4F868320133A4F8683283
:103AA00085F001014AF06EF92046FFF7CBFF0023B5
:103AB000A4F866324FF08073C4F85C3203B030BDB6
:103AC00094F85F3220460191012B04BF94F85D32D7
:103AD00084F85E32FFF7CFFB94F85F32019963B947
:103AE000012385EA030184F85F32E06B4AF04AF96A
:103AF000204603B0BDE83040A4E7002384F85F32DD
:103B0000F3E738B50D4603201446FDF7AFFF07EE87
:103B1000900A8DB1F8EE677A9FED097AF0EE006AAF
:103B200067EE877AB8EE047AA7EEA67ADFED057A1B
:103B300067EE277AC5ED007A0CB1034B236038BDE0
:103B40006740533A00007A443313904307B501238A
:103B500001AAFF210068FEF751FA03B05DF804FBEB
:103B600007B5022301AAFEF749FA044B1870BDF805
:103B7000040040BA80B203B05DF804FB9016012047
:103B800070B53B4C054694F8C830002B36D094F8FD
:103B9000D864012E33D0022E4FD07EBB012280216B
:103BA0000068FFF777FC0122FF212868FFF772FC0D
:103BB000324631462868FFF76DFC94F8D9249121EC
:103BC0002868FFF767FC012231462868FFF762FC8E
:103BD0003246FF212868FFF75DFC324680212868C5
:103BE000FFF758FC012231462868FFF753FC214BB0
:103BF0001B68C4F8C030012384F8D83470BD00219C
:103C00000068FFF739FCC20711D5D4F8C420002A98
:103C1000F4D0184BD4F8C0101B689BB25B1A9A42C0
:103C2000ECD2154B4FF0FF325A600023E4E7114B02
:103C30001B68C4F8C0300223DEE713210068FFF7D9
:103C40001BFC4307E1D01E212868FFF789FF0122F2
:103C500006460B212868FFF71DFC0A20064BB6FB21
:103C6000F0F6B6B25E60012384F8C930DDE700BF2C
:103C7000B89701203C2601209016012007B50223A9
:103C800001AA00210068FEF7B9F90F4B83F8CC00B8
:103C900050B1BDF804300D4A5BBA9BB2B3F5FA6F70
:103CA00005D34FF0FF33136103B05DF804FB0A2125
:103CB000B3FBF1F307EE903AF8EEE77AFDEEE77A20
:103CC000C2ED047AF0E700BFB897012090160120FA
:103CD00013B502230C4601AA00210068FEF78EF9F5
:103CE00060B15CB19DF805309DF90420DB0902EB61
:103CF000820203EB830303EB4203238002B010BD77
:103D0000F7B505460068FEF7CFF800230446FF210B
:103D10000370042328680DEB0302FEF76FF910B956
:103D2000002003B0F0BD04236A46FF212868FEF797
:103D300065F90028F4D09DF804108A09023A012A96
:103D4000EED99DF800209DF805309DF8015003EB59
:103D5000012305EB0225C3F30D03C5F30D055A1B23
:103D6000002AB8BF5242FF2ADADC9DF806109DF8FF
:103D700007209DF8027002EB01229DF8031001EB71
:103D8000072156114911C1EB5212002AB8BF524205
:103D9000FF2AC5DC01222B4431441341227011411A
:103DA000C4F80530C4F80110BBE738B500680D460B
:103DB0001446FEF779F8D0F8013007EE103ACDB18D
:103DC000D0F80530DFED166A07EE903A9FED156AE0
:103DD000F8EE677A77EEE67A77EEA77AC7EE866A2C
:103DE000F7EE007A76EEE77ADFED0F6A67EEE67AB5
:103DF000C5ED007A9CB1B8EEC77ADFED0C7ADFED45
:103E00000C6A27EE277AC7EE267A9FED0A7A77EEBC
:103E1000C77A9FED097A77EE877AC4ED007A38BDCC
:103E20009AC9CC449AC94C460E76D74500004843FF
:103E300000E0FF4400004842339388433B4BF0B519
:103E40002DED028B1B7E83B00E461546022B69D1E9
:103E5000374B384C1B6894F8DA2403F00203002A2D
:103E600045D0002B59D0344F0DF106001DF090FEC7
:103E7000BDF80630D7F8E823F0EE408A9FED2F7AA0
:103E800004F2DC449B1A07EE903AF8EEE77A87EEEC
:103E9000870ADFED2B7A20EE270AFBF71FFF97ED4D
:103EA000FF8AA0EE688A3AF0E1FBD4ED020AD0ED79
:103EB000057A70EEA70AB0EE480AFCF75DFF7EB106
:103EC00020EE000ADFED1F7A9FED1F7A20EE270A11
:103ED000C0EE077A9FED1D7A77EE877AC6ED007AFD
:103EE0000DB11B4B2B6003B0BDEC028BF0BDA3B139
:103EF000B4F90A3501EE103AB4F9083500EE903AFB
:103F0000B4F90635B8EEC11A00EE103AF8EEE00A40
:103F1000B8EEC00AFCF738FFD1E7D4F8203593EDAE
:103F2000350ACCE79FED0B0AC9E700BFD077012027
:103F300008000020B8970120208701200000C84217
:103F400035FA8E3CCDCC9C3F00409C4682E6C5476E
:103F500033139043000000002DE9F04F8BB0BDF803
:103F600050B09DF854A000900391CDE90123F7F7DC
:103F700093FB0646002800F0AC805C4F97F8245570
:103F8000072D00F2AB805C22002305EB45096C1C79
:103F900002FB0572C5EBC90107F5A569C2F8283512
:103FA000E4B282F82C3509EB8109009B87F824459F
:103FB0001A794FEA121802F00F0208F1FF38B8F12F
:103FC000030F3FD84A4931F8180040FA02F1CB07F5
:103FD00038D5012101FA02F2013A10404EF024F8DE
:103FE000444A0221039B12F808201044424A00EB85
:103FF000400002EB800888F8084000FA01F488F8D5
:10400000063088F80710BAF1000F46D13B4B404606
:10401000FFF726F91844007C4AF0D8F8B8F80430C5
:10402000354A05A90593112310590693CDF824A00C
:10403000CDE907AAF5F706FFB8F804302E4A1B04AD
:10404000A25893615C233046012403FB0575DDE92A
:104050000121C5F82865F7F7C7FB5946D5F82805AB
:10406000F7F750FCD5F82805F7F79CFDD5F828059B
:10407000022203685B68196883F83D200A682243BE
:104080000A6083F83D40F7F777FD0023C5F8300557
:10409000036048460BB0BDE8F08F4046009BFFF739
:1040A000DFF8DFF858C093F808A06044007C4AF0BD
:1040B0008DF8114A022100231059B8F80420069106
:1040C00005A9CDF824A00592CDE90733F5F7BAFE8E
:1040D000B8E7814648460BB0BDE8F08F0021084A9A
:1040E00004208946FCF7D2FED3E700BFB897012031
:1040F000F8830608C486060820700120CC860608CE
:10410000BC1007082DE9F0437E4D83B00C461346E2
:1041100095F860C0BCF1060F00F2EF80DFE80CF00C
:104120002DBA629204040400BCF1050F00F0D9809E
:10413000754A7649BCF1060F08BF0A464FF00009E0
:10414000019302211423CDF80090FFF705FF0746E5
:10415000002800F0D0808046122258F8140B414607
:104160004CF042FE0646002840F0BD80012645F88E
:104170003470304603B0BDE8F083654A00210193F6
:10418000644B16684FF6FF720091A3FB067102EBB9
:10419000D1120221120CB6FBF2F6A3FB0623324623
:1041A000C3F3CF13FFF7D8FE98B107EE906A9FEDE7
:1041B0005A7ADFED5A6A0123F8EE677A67EE877A5A
:1041C00027EE877A0371E7EE667A80ED047AC0ED18
:1041D000037A061E45F8340018BF0126304603B0A6
:1041E000BDE8F0834A4A002101934D4B16684FF613
:1041F000FF720091A3FB067102EBD1120221120C97
:10420000B6FBF2F6A3FB06233246C3F3CF13FFF748
:10421000A3FE0028DDD007EE906ADFED426A9FED35
:104220003F7A0123F8EE677A9FED3F6A037167EEEC
:10423000A66A27EE667AC0ED046AA7EE867A80ED5C
:10424000037AC6E701930026384B4FF6FF71304AD8
:104250009B8812680096B2FBF3F63144090CB2FB5E
:10426000F1F2B2FBF3F60221B3B2FFF775FE0028BC
:10427000AFD007EE906ADFED286A9FED287A012320
:10428000F8EE677A037167EEA67A27EE677AC0EDDB
:10429000047AD4E71E4A00210193214B16684FF699
:1042A000FF720091A3FB067102EB91120221120C26
:1042B000B6FBF2F6A3FB06233246C3F38F13FFF7D8
:1042C0004BFE002885D007EE906A9FED196A9FED9E
:1042D000127A0123F8EE677ADFED106A67EE867ACC
:1042E0006EE7144A2AE749464046482253F050FCFC
:1042F00001233B713BE7064639E700231E4645F89C
:10430000313036E7B8970120C0C62D00001BB7003A
:10431000BC0101201F85EB516F12833A00007A44E3
:10432000D34D621077CCAB32ACC5A736587501209F
:104330006F120339808D5B0010B582B00A4C009378
:104340009DF810300193B4FBF2F322469BB20C4669
:104350000321FFF701FE034620B10449012001EBD0
:1043600084018B6702B010BD40420F00B897012056
:104370000B4B10B553F8304082B001916CB107EE91
:10438000901A94ED047A94ED030AF8EEE77AA7EE1A
:10439000870A50F0E1FAA368186002B010BD00BFB0
:1043A000B897012010B5C04C04EB80039B6F0BB194
:1043B0009B6819600F2822D8DFE810F02200310036
:1043C000480063007A009100AC00C300D500E4000F
:1043D000FB0016012D0144015F011000084623F087
:1043E00055FB94F81D3800F00702C0F3C70003F036
:1043F0001F0384F81E0843EA421384F81D3810BDD9
:10440000084623F043FB94F80A38C0F3022284F8EC
:10441000090823F00703134384F80A3810BD08463F
:1044200023F034FB94F80A2894F80B3800F01F01AD
:1044300002F00702C0F3451023F03F0342EAC10235
:10444000184384F80A2884F80B0810BD084623F0A6
:104450001DFB94F80B2800F0030194F80D3802F0CE
:104460003F0223F0010342EA8112C0F38021C0F32E
:1044700087000B4384F80B2884F80C0884F80D3867
:1044800010BD084623F002FB94F80D2894F80E386E
:1044900000F07F0102F00102C0F3C31023F00F030C
:1044A00042EA4102184384F80D2884F80E0810BD32
:1044B000084623F0EBFA94F80E2894F80F3800F031
:1044C0000F0102F00F02C0F3061023F07F0342EA4F
:1044D0000112184384F80E2884F80F0810BD08460E
:1044E00023F0D4FA94F80F2800F0010194F8113861
:1044F00002F07F0223F0030342EAC112C0F341211C
:10450000C0F347000B4384F80F2884F8100884F8A0
:10451000113810BD084623F0B9FA94F8112894F820
:10452000123800F03F0102F00302C0F3841023F0C0
:104530001F0342EA8102184384F8112884F8120804
:1045400010BD084623F0A2FA94F8123800F00702D2
:10455000C0F3C70003F01F0384F8130843EA4213B3
:1045600084F8123810BD084623F090FA94F81538F4
:10457000C0F3022284F8140823F00703134384F8DD
:10458000153810BD084623F081FA94F8152894F8E0
:10459000163800F01F0102F00702C0F3451023F0A7
:1045A0003F0342EAC102184384F8152884F816082C
:1045B00010BD084623F06AFA94F8162800F00301AB
:1045C00094F8183802F03F0223F0010342EA811206
:1045D000C0F38021C0F387000B4384F8162884F8C9
:1045E000170884F8183810BD084623F04FFA94F8DD
:1045F000182894F8193800F07F0102F00102C0F386
:10460000C31023F00F0342EA4102184384F818282C
:1046100084F8190810BD084623F038FA94F81928D0
:1046200094F81A3800F00F0102F00F02C0F30610E0
:1046300023F07F0342EA0112184384F8192884F812
:104640001A0810BD084623F021FA94F81A2800F041
:10465000010194F81C3802F07F0223F0030342EAC0
:10466000C112C0F34121C0F347000B4384F81A285C
:1046700084F81B0884F81C3810BD084623F006FA9D
:1046800094F81C2894F81D3800F03F0102F0030252
:10469000C0F3841023F01F0342EA8102184384F818
:1046A0001C2884F81D0810BDB897012010B5094CCE
:1046B00094F82C38012B05D0022B07D0064BC4F8F8
:1046C000303810BD4BF042F9044BF8E74BF03EF99F
:1046D000034BF4E7B897012039340108A5E102083B
:1046E000A543010810B50023094C84F8343803238E
:1046F00084F83518FF2184F8362804F63402FDF7D3
:1047000037FC00280CBF6FF00C00002010BD00BF6C
:10471000B8970120F8B5124D00241646022305F67D
:10472000340285F83518FF21074685F83448FDF72F
:104730001FFC05F6340210B96FF00C00F8BD02231F
:10474000FF213846FDF75AFC0028F5D095F83428AB
:10475000204695F8353803EB02233380EEE700BF9F
:10476000B89701200023024A51210068FDF700BCE0
:10477000ECA0012013B5022301AA044651210068D0
:10478000FDF73CFC114AF0B1BDF804305BBA9BB2B6
:10479000D360D368B3F5C87F02DD4FF0FF33D36039
:1047A0000B4B0C4A1968D2F8343932338B4208D299
:1047B000C2F83419002302F6341251212068FDF7A3
:1047C000D7FB02B010BD6FF00103E8E7901601209F
:1047D0003C260120B897012037B5124D044695F8C4
:1047E000CA30E3B10DF1050100684BF0BEFA9DF847
:1047F00005307BB10DF1060296212068FFF78AFF94
:104800000A22BDF80630B3FBF2F3074A9360012396
:1048100085F8CB30012286212068FFF763FF03B0C3
:1048200030BD00BFB897012090160120FDF756B9A2
:104830000FB413B504AB094C094953F8042BD4F851
:104840003809019349F03AFBD4F83809FDF73AF9F1
:1048500002B0BDE8104004B0704700BFB897012017
:104860002D480108202108B553F05FFA034618B11E
:104870001A780130202AF9D0184608BD2DE9F041F8
:104880000D461646044600274FF019082046FFF74C
:10489000E9FF044690B1FCF7D7FF40F634024FF42D
:1048A0006171FBF799FCA0F5617090FBF8F030287E
:1048B00004D84FB9287033780133337017B12046CC
:1048C000BDE8F0810127E1E76870F4E737B50546F8
:1048D000084601914CF04EFD0199044602462846D7
:1048E000FCF74EFC68B92B5DA3F13002092A06D90A
:1048F00023F02003413B192B01D90134281903B0BF
:1049000030BD0020FBE730B1036882881B691A4282
:1049100014BF01200020704718B10268838809B1D4
:10492000936170471B04FBE710B1036882889A61AA
:10493000704718B1838802681B049361704730B5D3
:104940000C4687B00546B8B10C4BFEF789FC1844FD
:10495000007C49F03BFC002301A928680593AB8843
:10496000019304F013030293C4F34113C4F38104CD
:1049700003930494F5F766FA07B030BDCC860608B9
:1049800070B50C4686B016460546A8B10B4BFEF72F
:1049900067FC1844007C49F019FCAB8801A9286821
:1049A000019304F0130302936309C4F38104039396
:1049B000CDE90446F5F746FA06B070BDCC86060888
:1049C00010B5040900F00F02013C032C17D80D4B61
:1049D00033F8141041FA02F313F001000ED0012352
:1049E00003FA02F2013A02EA01004DF01DFB064B08
:1049F0000C221B5D1844054B02FB003010BD00204B
:104A0000FCE700BFF8830608C48606082070012072
:104A1000054B03EB8000826922B1116893884869D5
:104A200043404B61704700BFCC860608034B81F0C2
:104A3000010103EB800080696EE700BFCC860608A9
:104A40002DE9F84F6A4FD7F83C09037C03F0FF0CBF
:104A5000002B40F0CB8097F8422907F6461E97F8C6
:104A60004339E24697F844993C25A7F840C99EF897
:104A700002109EF80360C1F1FF0189B2002900F025
:104A8000B180BEF80040C1F1FF01B4FBF5FB7143FA
:104A90000912BBF1050F22D8DFE80BF0030E637497
:104AA0008593731A5FFA81F96343B3FBF5F353FA05
:104AB00081F3DBB2324610E0B4FBF5F205FB1242A3
:104AC000741A5FFA81F992B2C2F13C026243B2FBFE
:104AD000F5F252FA81F2D2B233464FF0010A1602D1
:104AE000002146EA034646EA09064FF00108C1F1F3
:104AF000170B0CEB010408FA0BFB4144A4B21BEAB0
:104B0000060F07EB840414BF4FF0020BC3461829AD
:104B1000C4F8C8B9E9D10CF1180C0EF1040E1FFA53
:104B20008CFCBCF5407FA2D13249A1F878C5BAF11E
:104B3000000F05D087F8422987F8433987F8449950
:104B40002023A7F8403991F87A35002B4ED040F257
:104B50002A31F7F739F8D7F83C09BDE8F84FF7F7ED
:104B600089B8B4FBF5F305FB1344A6EB0109CAB2FF
:104B7000A4B204FB09F9B9FBF5F959FA81F15FFA1E
:104B800081F9A9E7B4FBF5F305FB1343741ACAB224
:104B90009BB2C3F13C036343B3FBF5F353FA81F3D8
:104BA000DBB2B14699E7B4FBF5F905FB1944721A7B
:104BB000CBB2A4B26243B2FBF5F252FA81F2D2B2A6
:104BC000EFE7B4FBF5F205FB1242741ACBB292B2D6
:104BD000C2F13C026243B2FBF5F252FA81F25FFA93
:104BE00082F967E7B1463346324676E7BDE8F88F8B
:104BF000B8970120B0A80120F8B500211820F6F7D9
:104C0000DBFD054650B31C4FF6F746FD0446C7F8DA
:104C10003C0918B3194E1820FFF7D2FEC6F87C05E0
:104C200020B14FF40573C380002303722A7A4E210A
:104C3000FFF7A6FE124A03212046F6F7D5FD002114
:104C4000D7F83C09F6F75EFE40F22A320D49D7F854
:104C50003C094CF0C9F810B986F87A05F8BD40F661
:104C6000A8420021074852F093FF012386F87A35C5
:104C7000BDE8F840E4E600BFB8970120B0A80120E5
:104C8000009F240080A10120084B93F811214AB114
:104C900093F8133113F0400F14BF4FF4F0704FF43A
:104CA000C37070474FF4F070704700BFB897012091
:104CB000054B93F8110130B193F8133113F0400F05
:104CC0000CBF0D2010207047B8970120F0B5564C4E
:104CD0008DB005461023002228210220FCF71BFF7F
:104CE000C4F80C01002800F090800221FDF792F832
:104CF00002220021D4F80C01FDF7C4FA002104F5CA
:104D00008C7304F59B6284F814114FF0202184F811
:104D1000105143F8041B9342FBD1444E444F356875
:104D20003235D4F80C010379012B70D0022B0ED14F
:104D3000836880213E4ADB075CBF3D4A8021FDF746
:104D400085FC10B133689D42EBD8D4F80C011024D7
:104D50001123122113224FF0140E152716261725A2
:104D60008DF80C4018248DF80E3019238DF8101092
:104D70001A218DF812201B224FF0010C8DF814E03F
:104D80008DF816704FF01C0E8DF818601D278DF8E9
:104D90001A501E268DF81C401F254C248DF81E30FD
:104DA0008DF8201022238DF82220002103AA8DF8EF
:104DB0000DC08DF80FC08DF811C08DF813C08DF89F
:104DC00015C08DF817C08DF819C08DF81BC08DF86F
:104DD0001DC08DF81FC08DF821C08DF823C08DF83F
:104DE00024E08DF825C08DF826708DF827C08DF849
:104DF00028608DF829C08DF82A508DF82BC08DF8C9
:104E00002CC08DF82D404BF0D1F80DB0F0BD82686C
:104E1000417C02F0010C90F910008022CDE9007C69
:104E2000F6F76EF98DE700BFB89701203C26012008
:104E3000CB9801200F4A002370B54FF4005601248F
:104E400002F5707EA2F1460532F8020F4FEA531CBC
:104E500003F01F010133B0F5005F04FA01F11FBF39
:104E600055F82C001680014345F82C107245EBD103
:104E700070BD00BFCE9801204FF01E0C43EA022304
:104E8000FF2A0CFB01011BB288BF43F00403B1F5FC
:104E9000F07F07DA0C4A9BB202EB4100B0F818C170
:104EA0009C4500D170474FEA511CD032A0F8183110
:104EB00001F01F01012052F82C3000FA01F10B43E0
:104EC00042F82C30704700BFB89701204FF01E0CFD
:104ED0000CFB0101B1F5F07F01DB002070470B48AE
:104EE00000EB4101B1F81811080AC9B2108019701D
:104EF000490709D51188012041F4807111801A7881
:104F000022F004021A70704701207047B897012000
:104F10002DE9F0471E2404FB010114787CB31D2801
:104F20002DDC184E0FFA83FEC1F10105012706EBB7
:104F3000410C483E02E003441D2B20DCB1F5F07F1C
:104F40004EEA042405EB010311D2BCF800A04FEA9D
:104F5000511901F01F08A24507FA08F81FBFACF865
:104F6000004056F8294044EA080446F8294012F85F
:104F7000014F0CF1020CDBB20131002CDBD1BDE89A
:104F8000F08700BFD0980120F0B54F4C85B0D4F821
:104F90000C5115B194F812310BB105B0F0BD0123DD
:104FA00084F812312B79012B78D0022B35D1284689
:104FB0000DF10E028421FDF749FBD4F80C5194F851
:104FC00014212B7942F00402012B75D18DF80F20AA
:104FD000AA6895F9100002F00102697C01920DF1B6
:104FE0000F0200920422F5F7C7FE13E0022B0CD14A
:104FF000AB680DF10E0284212846DB075EBF0DF180
:105000000E0284212846FDF721FB9DF80E3013F097
:10501000040616D0D4F80C512B79012BE6D1AA68DE
:10502000697C95F9100002F001020DF10E05CDE941
:1050300000528422F6F764F89DF80E3013F004064F
:10504000E8D1224D31463C22214884F81431012711
:1050500052F09EFD3146A5F1460E05F5707635F805
:10506000023F4FEA511C01F01F0001311A0A03F000
:10507000040307FA00F022F0200213431EBF5EF87B
:105080002C3018434EF82C00B542E8D1FEF7A0FAB8
:105090000028FBD184F8120105B0F0BDAA68697C34
:1050A00002F0010295F9100001920DF10E0200923A
:1050B0008422F6F725F880E7022BAED1284604219A
:1050C000FDF7BDF8A6E700BFB8970120CE980120F4
:1050D0008898012070B5394D84B0D5F80C416CB377
:1050E00095F81031012B42D0022B29D1082304223C
:1050F00085F813318DF80D30002094F910308DF8BB
:105100000E208DF80F2003EB8303A2682C49920731
:105110008DF80C0051F8236036D5042303AA3046DD
:105120000021F6F783FAA3689B0729D53C22FF21CB
:10513000244852F02DFD95F81131D3B104B070BD63
:105140002379012B2BD0022B22D09DF80B3003F0BA
:105150000503012B09D013B9D5F80C41C6E71A4A4B
:1051600040F2DC5312689A42E8D9D5F80C41482342
:10517000BDE7FFF709FF012385F8113104B070BDC9
:105180002046FCF7C3FED1E760694AF007FFC4E799
:105190000DF10B02A0212046FDF758FAD5E7A268D1
:1051A000617C02F0010294F9100001920DF10B02F2
:1051B0000092A022F5F7A4FFC7E700BFB89701202F
:1051C00000000120889801203C260120F0B53E4CCB
:1051D00085B0D4F80C5195B194F81331180702D565
:1051E00094F812316BB194F8113143B9FFF772FFA3
:1051F00094F81131002B3BD1002384F8123105B013
:10520000F0BD012294F8113184F81221002BEDD069
:105210002B79012B2FD0022BE8D10DF10E0280212A
:105220002846FDF713FA0028E0D094F813219DF8E2
:105230000E309A42DAD194F81051002DD8D1234B78
:10524000234E1F68D6F88035FB1AB3F57A7FCFD985
:10525000A0210DF10F02D4F80C01FDF71DFA9DF805
:105260000F30590715D5C6F88455C6F88075BFE7C5
:10527000FEF7AEF9C0E7AA68697C02F0010295F971
:10528000100001920DF10E0200928022F5F738FF16
:10529000C9E703F00503012B0ED0002BE5D194F8EC
:1052A00013315B06E1D5D6F8843553B1FB1A642B74
:1052B000DBD9FFF70FFFD8E794F813315A06F2D580
:1052C000D3E7C6F88475D0E7B89701203C260120C3
:1052D000B0A801202DE9F0438D4E85B0D6F80C41E1
:1052E000002C6DD096F81291B9F1000F00D0FEE7B6
:1052F00096F813C1012305460F460CF0F70C86F80B
:10530000123186F813C12379012B00F0DD80022BC6
:1053100000F097800DF10F08B5F5807F00F0B280A6
:105320002379012B00F0B980022B07D120465022AF
:105330000821FCF784FFD6F80C412379012B754D29
:1053400019D0022B0DD142462046A021FDF77EF94F
:1053500020B19DF80F4014F0200450D0D6F80C4135
:105360002379D5F8A810012BB5F8AC20486982EA5A
:1053700000024A61E5D1A268617C02F0010294F961
:105380001000CDE90082A022F5F7BAFEE0E7B9F1FE
:10539000000F12D196F81341D6F80C5104F0F7041F
:1053A00086F813412B79012B00F0A380022B04D146
:1053B000224649462846FCF742FF002386F8123170
:1053C00005B0BDE8F083022B16D162460A212846BB
:1053D000FCF735FFD6F80C0107EB040C0379012B21
:1053E00028D18568C022417C05F0010590F91000A4
:1053F000CDE900C5F5F784FE0134362CC7D0D6F8C8
:105400000C515FFA84FC2B79012BDCD1AA6895F949
:105410001000697C02F001050A228DF80FC0CDE969
:105420000085F5F7A9FCD6F80C0107EB040C03790D
:10543000012BD6D0022BDFD16246C021FDF706F941
:10544000DAE74946204662460DF10F08FCF7F7FE01
:10545000D6F80C4181462379EAB2012B2CD1A16800
:1054600094F9100001F0010C617C8DF80F200922E5
:10547000CDE9008CF5F780FCB5F5807FD6F80C41BE
:105480007FF44EAF204640220A21FCF7FBFED6F8FF
:105490000C412379012B7FF447AFA26894F91000E7
:1054A00002F00102617CCDE9008250228DF80F20CC
:1054B0000822F5F761FC3EE7022B7FF42DAF204672
:1054C0000921FCF7BCFED7E7A1680DF10F0894F99C
:1054D00010004A4601F0010E617CCDF80080CDF845
:1054E00004E08DF80FC0F5F747FCD6F80C41814673
:1054F000B1E7A9684A4695F9100001F00107697CF7
:105500008DF80F40CDE90087F5F736FC55E700BF71
:10551000B897012020700120034BD3F80C310BB158
:10552000FEF7AAB9704700BFB89701208379806B56
:10553000DB0748BF81F0010109B1FFF7F5B9FFF7BB
:10554000F8B910B58379044613F0010F03F0200277
:10555000C36B13D0002A5B6818BF02211A7A08BFF8
:105560004221606BFFF70CFA0123204684F8603279
:10557000A4F85C32BDE81040FEF764BA002A5B680C
:1055800018BF02211A7A08BF2221EAE7036C806B58
:1055900023B15B6801211A7AFFF7F2B90121FFF705
:1055A000CEB9836870B51C6863799A0731D594F8D1
:1055B0006152D5B194F962329BB1B4F864122046BD
:1055C0004B0801F00101A4F86432FFF7AFFF94F833
:1055D0006232A279013B50065BB284F8623218D580
:1055E000BBB9002384F8613213E0A36A626A94F8BD
:1055F00060129A4227D161B9A3791B0709D5236CA0
:10560000A06BE3B15B681A7AFFF7BAF92046FFF79F
:1056100098FF6379D90740F1868094F85C32002BBB
:1056200040F0818094F85D320133DBB2092B84F8BD
:105630005D323AD12046BDE87040FDF71CBE1946E8
:10564000FFF77DF9E2E75A1CA0692669A262C35CF4
:10565000B24234BF104628465B00A06243F4007398
:10566000A4F864320A2384F86232012384F8613298
:10567000B9B1A3791E0714D5E36B2B485B68196891
:105680005E790A6A50F8260022EA0002606B0A621C
:1056900029461A7AFFF774F9204684F86052FFF71A
:1056A00075FFA3795D0685D4B3E70A2B3BD194F847
:1056B0005F322BB9B4F8663243F00103A4F86632C6
:1056C000B4F86602820501D4C30719D4B4F86A326B
:1056D0000133A4F86A320123A4F85C3294F85F32F3
:1056E000012B20D1A1790023E06B84F85F3201F017
:1056F000010148F047FB2046BDE87040FEF7A2B923
:10570000E36AC0F3470013B1216B9847E3E7E3690D
:105710006269D054E369E2680133B3FBF2F102FB42
:105720001133E361D7E770BDCC8606081D4B1A68BC
:1057300010B513460446B3FBF1F0B0F5803F03D338
:10574000012BFAD95B08F6E781B22046F6F74CF850
:1057500023681B68587948B140B2032148F02EFEF7
:1057600023681B6893F90500F4F75EFB23681B6848
:10577000987948B140B2032148F020FE23681B68A5
:1057800093F90600F4F750FB236802225B6819685E
:1057900083F83D200A6842F001020A60012283F882
:1057A0003D2010BDBC0101208160C06BBEE7002A16
:1057B0004FF0200CBCBF80185242002BBCBFC91850
:1057C0005B420028BCBF121A00200029F0B500EB94
:1057D000020501EB0304B8BF00210F4EA5F11D0522
:1057E000B8BF23460F3C3C27002DC8BF521B002CDE
:1057F000C8BF1B1B02440B4490420CDC06EB400567
:105800000C4604E007FB04FE013425F80EC09C4260
:10581000F8DD0130F0E7F0BDD0980120014B53F8DE
:105820002000704750280040014B43F8201070477B
:10583000502800401A4B07B51A6C1A4942F08052A2
:105840001A641A6C02F080520192019A0A6842F4BA
:1058500080720A60FF211A6C42F480621A641A6C2A
:1058600002F480620092009A0F4A5162CA2151628A
:10587000532151625B6FDB0005D50020FFF7CEFF9F
:105880000A4B984209D000210120FFF7CDFF0749BC
:10589000002003B05DF804EBC6E703B05DF804FB3D
:1058A00000380240007000400028004076614E69D8
:1058B0002DE9F74F0026054688466A4C3746DFF843
:1058C000B0A1C0E9006614F029FE81469AF80630BE
:1058D000022B29D1E3685A0742BF23F0040343F0A7
:1058E0000803E360E368980604D523F0200343F03F
:1058F0004003E360012001A9F6F762FB01201CF0E0
:10590000C5FE38B323799DF805209A421ED133464F
:10591000554A01210420FBF7B9FA013614340B2E45
:10592000D4D103B0BDE8F08F012BE3D1E3681907B0
:1059300042BF23F0080343F00403E360E3685A0620
:10594000D8D523F0400343F02003D2E79DF804208C
:105950009A42DCD0022001A9F6F732FB02201CF0AB
:1059600095FE40B123799DF805209A42CFD09DF84D
:1059700004209A42CBD0032001A9F6F721FB032093
:105980001CF084FE40B123799DF805209A42BED0D8
:105990009DF804209A42BAD0052001A9F6F710FB21
:1059A00005201CF073FE40B123799DF805209A4232
:1059B000ADD09DF804209A42A9D02C4BD3F800B06A
:1059C0001BF0400F08D000211220F5F7F5FE18B1AA
:1059D000026823689A429AD01BF4803F08D00021C5
:1059E0001820F5F7E9FE18B1226803689A428ED0B4
:1059F0002379A3F13002022A89D9142B87D09AF88F
:105A00000120E3680AB1032A1AD1580722D5B94503
:105A100024D923F008030137E360FFB2B8F1000F87
:105A200002D0E368190710D4E36813F0040F3FF4C1
:105A300074AF2B685A1C02332A6045F823406CE788
:105A40005A0602D413F0200FF1E76B685A1C0A3390
:105A50006A60F2E7B8F1000FE3D15EE7B8F1000F3A
:105A6000E7D0DEE70C040120F7100708040000204F
:105A7000907F0120F7B5054614F050FD0C28044630
:105A80000CDD224B01221A700C23214A009303469D
:105A900000210420FBF7FAF903B0F0BDFDF794FCF8
:105AA0001C4B9A791C4B03EB420393F824303BB90F
:105AB0001A4A0221042003B0BDE8F040FBF7E6B922
:105AC0002B68A34219DB08350026154FA642E3DAFE
:105AD0003A68F1B255F8040BC2F30072FEF712FBFC
:105AE000014688B9094B052204201A7033460D4A35
:105AF00003B0BDE8F040FBF7C9B9044A03211170B7
:105B000000932346084AC3E70136DFE764750120A6
:105B10000F11070858750120CC8606083B110708AD
:105B20000400002092110708591107082F4B2DE996
:105B3000F3411C78064634B12D4B93F8884593F811
:105B400089350134E41A2B4B1B783BB92A4A0221D0
:105B5000042002B0BDE8F041FBF798B9102C0DDD30
:105B6000264B0222002104201A701023244A00939D
:105B70002346FBF78BF902B0BDE8F081214FFEF719
:105B800095FD97F82C1811F0FD0101D01E4ADEE7B3
:105B90007368A34220DB28360D46DFF87880A542E3
:105BA000E9DAD8F80030E9B2B7F82628C3F3007371
:105BB0000093B7F8243856F8040BFEF7BDFB0146F6
:105BC00088B90E4B052204201A702B460F4A02B0EA
:105BD000BDE8F041FBF75AB9084A04201070009361
:105BE00023460B4AC5E70135D9E700BF54750120AC
:105BF000B0A8012056750120B7110708647501206F
:105C0000D1110708B8970120FD1107086F12070886
:105C10003912070804000020014B00221A75704752
:105C200090160120014B01221A7570479016012031
:105C3000044A054B92F8602003EB420393F82500D9
:105C4000704700BFB8970120CC8606081049114B59
:105C500091F8602003EB420393F8253003B97047B5
:105C60000D4B10B41C7884B100234FF0010C51F897
:105C700033203AB112792AB1984204BF01EBC30232
:105C800082F806C001339C42F1D15DF8044B7047A5
:105C9000B8970120CC8606081810002010B5154CC6
:105CA00082B0D4F89C25D4F8A035D4F8941502FB22
:105CB00003F38DF807008B421AD0D4F890350DF11C
:105CC0000701D4F89805184451F018FDD4F8903520
:105CD000D4F89C25D4F894151344D4F8A025B3FB2C
:105CE000F1F0013201FB1033C4F8A025C4F890355F
:105CF00002B010BDB0A801200B4B0022012003F21E
:105D0000A45110B40824C3F88C25C3F89C05C3F82B
:105D10009445C3F898155DF8044BC3F89025C3F873
:105D2000A025C3F8B0257047B0A801200F4B93F809
:105D30006030062B17D8DFE803F00416070A0D10B1
:105D400013004FF4C87070474FF4FA607047084B67
:105D5000988870474FF47A6070474FF4FA50704754
:105D60004FF47A5070474FF47A707047B89701201B
:105D700058750120034B53F8300010B103685B687D
:105D800018797047B8970120034BD3F8302812B127
:105D90000F2800D810477047B8970120130A07B59D
:105DA0008DF8043002238DF8052001AAFCF7E0F8F5
:105DB000024B187003B05DF804FB00BF9016012081
:105DC00050B10138002330F0FF019AB203F1010312
:105DD00003D140EA022080B270474008F3E710B5D3
:105DE0000C460121FDF748FBC0F300132370C0F3FC
:105DF000C003A370C0F380036370C0F38013C0F3CB
:105E0000C010E370207110BD2DE9F0478846502185
:105E100014460646FDF730FB01304621304F400066
:105E20004FF47A794FF4FA6AC0B220803046FDF719
:105E300023FB2378013051217B4380B203F5FA73B1
:105E4000A080B3FBF9F2B3FBFAF300FB0233304658
:105E5000B3FBF9F3E360FDF783FEC0F30F22C3B297
:105E60002578304603FA02F27D43013293B205F5FC
:105E7000FA72B2FBF9F1B2FBFAF203FB01227021D4
:105E8000E380B2FBF9F22282FDF7F6FA01307121CC
:105E90004000C0B260803046FDF762FE98F80320F3
:105EA000C3B2C0F30F20834001339BB2238112B1F0
:105EB000E2889B1A2381A3784FF47A724FF4FA6533
:105EC00020897B4303F5FA73B3FBF2F1B3FBF5F3DF
:105ED00000FB0133B3FBF2F36382BDE8F08700BF40
:105EE000002F3A002DE9F0474FF4FA730026834F54
:105EF0008CB0044689210068C7F8C43087F8C860B0
:105F0000FDF7BAFA40F001008921DFF8F481C2B24E
:105F10002068FDF7BFFA324688212068FDF7BAFAFB
:105F2000012280212068FDF7B5FA0122FF212068B7
:105F3000FDF7B0FA324631462068FDF7ABFA912101
:105F40002068FDF799FA3146012287F8D9042068C4
:105F5000FDF7A0FA3246FF212068FDF79BFA324692
:105F600080212068FDF796FA60212068FDF784FA09
:105F700040F012006021C2B22068FDF78BFA2022A7
:105F800044212068FFF70AFFFF2201212068FDF766
:105F900081FA2568012280212846FDF77BFA01223B
:105FA000FF212846FDF776FA324631462846FDF7AE
:105FB00071FA0622FF212846FDF76CFA8321284654
:105FC000FDF75AFA40F004008321C2B22846FDF7DB
:105FD00061FA0722FF212846FDF75CFA01228121A0
:105FE0002846FDF757FA012280212846FDF752FA8C
:105FF0006B2294212846FDF74DFA3246832128462C
:10600000FDF748FAD8F80060C7F8C0608321284639
:10601000FDF732FA002800F055830122284683213B
:10602000DFF8E080FDF736FA92212846FDF724FAE2
:106030000022C0F3C716814681212846FDF72AFABF
:1060400006222846FF21FDF725FA8321284609F07C
:106050007F09FDF711FA832100F0FB022846FDF7C6
:1060600019FA28460122FF21FDF714FA28460122D9
:106070000021FDF70FFA28460022FF21FDF70AFA5A
:10608000284600228021FDF705FA062305AAB02143
:1060900020680025FBF7B2FF0122FF2188F80000ED
:1060A0002068FDF7F7F900224F212068FDF7F2F98B
:1060B0002C224E212068FDF7EDF90022FF212068F7
:1060C000FDF7E8F9B422B6212068FDF7E3F9002EC8
:1060D0002A464FF0010C18BF0C260CAB5FFA85FE68
:1060E000C5F3C40005F007017645184410F81C3CC0
:1060F0000AD8914540F0F18206E000BFB897012030
:106100003C260120901601200CFA01F123EA01033C
:1061100000F81C3C0135302DDFD1062305AAB02143
:106120002068FBF725FF0122FF2188F80000206886
:10613000FDF7B0F9002220681146FDF7ABF9002207
:10614000FF212068FDF7A6F9002209212068FDF74C
:10615000A1F9002210212068FDF79CF900221121ED
:106160002068FDF797F9012224212068FDF792F9B4
:10617000FF2225212068FDF78DF900227521206876
:10618000FDF788F90122FF212068FDF783F92C2211
:106190004E212068FDF77EF9002248212068FDF796
:1061A00079F9294620222068FDF774F90022FF21A1
:1061B0002068FDF76FF9294609222068FDF76AF982
:1061C000002254212068FDF765F90422312120685E
:1061D000FDF760F9032232212068FDF75BF9832285
:1061E00040212068FDF756F9252246212068FDF759
:1061F00051F9002260212068FDF74CF90022272187
:106200002068FDF747F9062250212068FDF742F982
:10621000002251212068FDF73DF996225221206885
:10622000FDF738F9082256212068FDF733F92A4690
:1062300057212068FDF72EF9002261212068FDF723
:1062400029F9002262212068FDF724F90022642147
:106250002068FDF71FF9002265212068FDF71AF973
:10626000A02266212068FDF715F90122FF21206890
:10627000FDF710F9322222212068FDF70BF91422D4
:1062800047212068FDF706F9FF2249212068FDF724
:1062900001F900224A212068FDF7FCF80022FF21C5
:1062A0002068FDF7F7F80A227A212068FDF7F2F856
:1062B00000227B212068FDF7EDF82122782120685B
:1062C000FDF7E8F80122FF212068FDF7E3F834220A
:1062D00023212068FDF7DEF8002242212068FDF727
:1062E000D9F8FF2244212068FDF7D4F82622452161
:1062F0002068FDF7CFF8052246212068FDF7CAF88F
:10630000402220681146FDF7C5F806220E212068BC
:10631000FDF7C0F81A2220212068FDF7BBF84022C3
:1063200043212068FDF7B6F80022FF212068FDF721
:10633000B1F8032234212068FDF7ACF8442235215E
:106340002068FDF7A7F80122FF212068FDF7A2F8D9
:10635000042231212068FDF79DF809224B21206895
:10636000FDF798F805224C212068FDF793F80422E8
:106370004D212068FDF78EF80022FF212068FDF7EF
:1063800089F8002244212068FDF784F82022452165
:106390002068FDF77FF8082247212068FDF77AF88A
:1063A000282248212068FDF775F80022672120681F
:1063B000FDF770F8042270212068FDF76BF80122C8
:1063C00071212068FDF766F8FE2272212068FDF732
:1063D00061F8002276212068FDF75CF80022772121
:1063E0002068FDF757F80122FF212068FDF752F8D9
:1063F00001220D212068FDF74DF80022FF212068C1
:10640000FDF748F8012280212068FDF743F8F822C3
:1064100001212068FDF73EF80122FF212068FDF7E9
:1064200039F801228E212068FDF734F8012200217D
:106430002068FDF72FF80022FF212068FDF72AF8D9
:10644000002280212068FDF725F804220A21206817
:10645000FDF720F8256884212846FDF70DF88421F2
:1064600000F0EF022846FDF715F801220B21206805
:10647000FDF710F8206803A90190FFF7B0FC07AA08
:1064800003A90198FFF7C0FC9DF80C30002B00F029
:106490002A810A9D05F684559DF80E30002B00F0E8
:1064A00025810A9B03F2B22305EB43059DF80F30CB
:1064B00023B1BDF82C3003F525731D449DF8103031
:1064C00023B1BDF82E3003F226231D44DFF83482B9
:1064D000E82201212068C8F8B455FCF7DBFF44F638
:1064E0001F639D4203D92946206849F05EFC0122C2
:1064F00020681146FCF7CEFF40212068FCF7D2FF50
:10650000002800F0E780012120680222FCF7C2FF8A
:1065100000212068FCF7C6FF002800F0DB80E8229D
:10652000012120684FF47A7AFCF7B4FF202244213D
:106530002068FFF733FC256803A948F20E66284659
:10654000DFF8C491FFF74BFC07AA03A92846FFF721
:106550005BFC502257212846FCF79CFF082256215D
:106560002846FCF797FF082250212846FCF792FFA7
:10657000BDF82C000AFB0060B0FBF9F080B2FFF719
:106580001FFC512102462846FFF708FC0A9A5C4B83
:1065900046210AFB026628469E429BBFB6FBF9F2E3
:1065A00002F1FF32FF22D2B2FCF774FFD8F8B41523
:1065B00044F61F63994202D9284649F0F6FB0121AF
:1065C0002846FCF759FF0222064601212846FCF71F
:1065D00061FF00212846FCF765FF3246012128466D
:1065E000FCF758FF246803A92046FFF7F8FB07AA29
:1065F00003A92046FFF708FC482220461146FCF775
:1066000049FF082247212046FCF744FF032232219C
:106610002046FCF73FFF072230212046FCF73AFFD7
:106620000122FF212046FCF735FF202230212046A1
:10663000FCF730FF0022FF212046FCF72BFF06224B
:1066400020467021FCF726FFBDF82E304FF47A72F9
:1066500046F6440002FB03004DF28803B0FBF3F062
:106660009DF80F3080B21BB1BDF82230184480B2C3
:10667000FFF7A6FB712102462046FFF78FFBD8F8F3
:10668000B41544F61F63994202D9204649F08DFBA8
:1066900001212046FCF7F0FE02220546012120469A
:1066A000FCF7F8FE00212046FCF7FCFE2A460121FB
:1066B0002046FCF7EFFE6423C7F8C430012387F8B7
:1066C000C83007E0D8F800309BB29B1BB3F5FA7FC7
:1066D0007FF69CAC0CB0BDE8F0870B41DB0744BFF4
:1066E0000132D2B216E540F63635D5E69DF80D30CA
:1066F000002B3FF4DBAE0A9B03F525731D44D5E662
:106700001B280D01B0A801201C0C010010B50023AE
:106710000A4C84F83438130A84F83518FF2184F8B9
:106720003638042384F8372804F63402FBF720FCBB
:1067300000280CBF6FF00C00002010BDB89701209E
:106740002DE9F3410023744D06460468DFF8D48137
:106750002D2785F8CA30B9B2013718F8012B204629
:10676000FDF7C0FF882FF6D1402287212046FDF794
:10677000B9FF00238DF806300DF10601204649F0DF
:10678000F4FA9DF80630002BF6D00122862120462F
:10679000FDF7A8FF002287212046FDF7A3FF09226D
:1067A00008212046FDF79EFF00220B212046FDF721
:1067B00099FF002851D137680DF106025E21384655
:1067C000FDF7A8FFBDF80630B3F5D77F00F09F8036
:1067D00053D8512B00F0998047D81D2B6AD01E2B1F
:1067E00000F093802121306849F02EFA34680DF1D1
:1067F0000602DE212046FDF78DFFBDF80630282277
:106800009FED467AC3F30903FF212046ADF8063019
:106810005343002207EE903A85F834286C22F8EEB4
:10682000E77A85F8352867EE877AFCEEE77A17EE87
:10683000903A1A0E85F8393885F836281A0C85F8FA
:1068400037281A0A062385F83828354AFBF790FBC3
:10685000402287213068FDF745FFB0FA80F04009FB
:1068600085F8CA0002B0BDE8F081AD2B4FD0D62B21
:1068700001D0602BB6D121241DE040F2E1329342D9
:1068800047D00CD840F2D922934242D040F2E122C4
:10689000934202D0B3F5E67FA4D164240BE040F22A
:1068A0008F42934203D040F2915293429AD14FF4D7
:1068B000FA7400E00F24002894D10A224B213846B4
:1068C000FDF710FF0F2260213846FDF70BFF0D2268
:1068D00063213846FDF706FFB82269213846FDF7E7
:1068E00001FF40F60D7278213846FFF70FFF40F6A2
:1068F0000E627A213846FFF709FF00287FF472AF55
:106900002146384649F0A0F96CE71424D3E7322435
:10691000D1E7C824CFE700BFB89701209A99893FF3
:10692000EC9F0120FE86060838B50B0A15460D4A75
:10693000044682F83438022382F8351802F634020D
:10694000FF21FBF715FB10B96FF00C0038BD0123D8
:106950002A46FF212046FBF751FB0028F4D00020F7
:10696000F4E700BFB897012003681B681847036865
:106970005B68184703689B6818470368DB6970B554
:1069800006460C46154683B1BDE8704018473046B0
:10699000FFF7F0FF0028FAD014F8011B3046FFF78C
:1069A000E3FF2B1B002BF2DC70BD0D44F9E7E4E79D
:1069B0000368DB68184708B51F4B204CD3F8B8555F
:1069C000A0681BF0DFFF28461BF0DCFFA0684179C0
:1069D0008B0704D4036841F002019B6998470021AA
:1069E0000846FEF723F800210120FEF71FF8A068F3
:1069F000FFF7BDFF70B101210020FEF717F8A06876
:106A0000FFF7D6FF01462846FFF7AEFF00210846F4
:106A1000FEF70CF82846FFF7AAFF0028E7D001216F
:106A20000846FEF703F82846FFF7C2FF0146A068B4
:106A3000FFF79AFFD7E700BFB0A80120C876012072
:106A400003681B69184703685B69184703689B6AFA
:106A500003B1184770470368DB6A03B118477047F2
:106A60000D4B01461B68DB0606D50C4B93F8BC3575
:106A700013F0040F18BF0021094B9B7A13B108468D
:106A8000FCF7E4BC074B1868074B1B780BB981F087
:106A90000101FDF741BF00BF00000020B0A80120A8
:106AA000347601202C76012030760120BFF34F8F01
:106AB0000549064BCA6802F4E0621343CB60BFF39A
:106AC0004F8F00BFFDE700BF00ED00E00400FA05B6
:106AD00008B572B600224FF0FF319300013203F186
:106AE0006043082A03F56143C3F88010C3F880119E
:106AF000F3D1FFF7DBFF012108B50846FEF794FE4E
:106B0000FFF7E6FFEFF31183102282F312880B499F
:106B1000DBB20A6801320A604FF0E022084990694E
:106B2000C1F8CC050020C1F8D005126983F31188A3
:106B3000044A136801331360704700BF3C260120EC
:106B4000B0A8012050220120064B074A1B6851685B
:106B500058434FF47A73B0FBF3F053685B1A8342E7
:106B6000FBD97047082B0120001000E010B5EFF3AF
:106B70001182102383F312884FF0E0239C69196976
:106B800011F4803F0D4903D00120C1F8D0059C6964
:106B90000B4BD2B21868D1F8D03582F31188094A6C
:106BA000034411684FF47A7202FB01F0001BB0FB42
:106BB000F1F00021E3FB020110BD00BFB0A80120ED
:106BC0003C260120082B0120124B5B68C3F308030D
:106BD00030B4EBB9EFF31183D3B90F4B4FF0E0258D
:106BE0000E481968AC691A688A42FAD1D0F8CC15F7
:106BF000A142F6D30A4B19684FF47A7303FB01F0F4
:106C0000001BB0FBF1F0002130BCE2FB0301704738
:106C100030BCABE700ED00E03C260120B0A801202D
:106C2000082B0120F8B506460D46FFF7CDFF0446B8
:106C30000F46FFF7C9FF031B61EB0702B34272EB7C
:106C40000503F6D3F8BD10B50446013C00D210BDD3
:106C50004FF47A700021FFF7E5FFF6E70023F7B560
:106C6000174F1A4634210120FAF755FF04463860C1
:106C700048B9144B1B780C2B03D1134B0122C3F8DA
:106C8000D425254618E005269620FFF7DCFF0DF1F8
:106C9000070200212046FBF7FFFC054660B9013ED4
:106CA000F2D1084B38681B780C2B02BF064B02222E
:106CB000C3F8D425FAF722FF284603B0F0BD00BF81
:106CC000E081012078730120B0A8012008B50122DD
:106CD00009210068FBF7D6FA6420BDE80840B2E756
:106CE00006460B2580B5013D01D1FFF704FF0121C8
:106CF000771C4FF0320805240846FDF797FE002167
:106D00000846FDF793FE0120FDF782FE0020FDF707
:106D10007FFE0120FFF7A4FE4046FFF794FF01200D
:106D2000FDF776FE0020FDF773FE0020FFF798FECA
:106D30004046FFF788FF7CB1013C05D14FF0FA08CF
:106D40004FF4FA70FFF77FFF54EA0703DBD14FF4EB
:106D50007A70FFF778FFC6E7013FF5E718B10368DF
:106D60005B6803B11847FF20704718B103689B6840
:106D700003B118470020704770B450B106798E42B5
:106D800007D34579954204D30368DB680BB170BC27
:106D9000184770BC704710B440B184798C4205D359
:106DA00003681B6913B15DF8044B18475DF8044B89
:106DB000704718B103685B6903B11847704718B191
:106DC00003681B6A03B118470020704730B568B1EB
:106DD000041D0A4600F114032068083454F8041C0A
:106DE00015469C4203C52A46F6D1012030BD10B598
:106DF0000C4670B92D23002023750A4B2061C4E98D
:106E000006333023C4E90000C4E9020084F82030CE
:106E100010BD0368DB6A002BECD098470028E9D04E
:106E2000F6E700BF1618070838B5441E044D14F8DD
:106E3000011F01B938BDD5F83809FAF74FFEF6E75A
:106E4000B897012013B50D4C01900D480091FFF744
:106E5000EBFF0C49D4F83809DDE9003247F02EF891
:106E6000D4F83809FAF72EFE074B93F8F42512B13F
:106E7000012283F8F52502B010BD00BFB8970120AC
:106E8000941207082D480108B0A8012008B504464F
:106E90000748FFF7C9FF074BD3F83809FAF712FE86
:106EA000054BD3F8B8051BF06DFD20460BF080FCB8
:106EB000A0120708B8970120B0A80120034808B520
:106EC000FFF7B2FF0120FFF7E1FF00BFAC12070898
:106ED0007FB5174B1A78012A27D15B790A2B04D08A
:106EE000144807B05DF804EB9EE71122002101A8C9
:106EF00050F04EFEA623152168468DF80030412340
:106F00008DF802108DF80130EB238DF803300A4B19
:106F10005B7D8DF80430B2238DF8053003238DF8A6
:106F2000063020F0C2FD0548DBE707B05DF804FB42
:106F30006C7B0120C512070890160120D4120708A7
:106F400010B504460948FFF76FFF05F0DFFE05F0B6
:106F5000E8F9074B00220749204683F8F525FDF79D
:106F6000B5FC08B9FFF792FF10BD00BFEE1207088D
:106F7000B0A801200D1E0708054808B5FFF754FF0B
:106F8000044BB3F8F60510B1BDE808405BE608BD58
:106F900033600708B0A8012010B5074C02460B4625
:106FA0000649D4F8380946F089FFD4F83809FAF7C9
:106FB00089FDBDE81040DFE7B89701202D480108A2
:106FC0000FB407B504A951F8040B0191FFF73AFF7C
:106FD000FFF7D2FF03B05DF804EB04B0704770B563
:106FE000837916468EB0044603F00F02062A52D863
:106FF000DFE802F00415181A1D1F4B000D7813F07E
:10700000C0034AD0402B3ED12946204611F062FDF4
:1070100000285ED00EB0BDE87040FDF709BC91F9C4
:107020000050ECE70D88EAE7B1F90050E7E70D689A
:10703000E5E791ED000A03A8FAF7ACFA01462A4801
:10704000FDF7F6FBFEB1A37913F0C00F1BD120466C
:1070500011F091FC00EE100A03A8B8EEC00AFAF78E
:1070600099FA01462148FDF7E3FB204611F094FC14
:1070700000EE100A03A8B8EE400AFAF78BFA0146B0
:107080001A48FDF7D5FB0EB070BD17480EB0BDE82D
:107090007040FDF7CDBB0025B1E7042A29460CBF9F
:1070A00013481448FDF7C4FB002EECD0A37913F06D
:1070B000C00FE8D1204611F05EFC0190204611F08F
:1070C0006BFC019902460C480EB0BDE87040FDF71C
:1070D000AFBB03A9204611F071FB03AA294607485C
:1070E000FFF76EFFCFE700BFB6140708991807082F
:1070F000D8170708DB430708D867070804130708F1
:1071000013B50446019111F029FC019A014620466D
:1071100002B0BDE8104062E7004851E721130708BC
:107120002DE9F04F87B00346FCF74AFA064618B13E
:1071300007B0BDE8F04FEFE705AA474918463446C7
:1071400050F0BBFCB04605464FF0FF37DFF83091FA
:10715000DFF830A1DFF830B18DB97EB230461BF0D8
:10716000C1F810B14568002D5BD1B8F1000F36D1E0
:1071700039463A48F9F75AFE07B0BDE8F08F012EBC
:107180000ED0022E11D01EB92846FAF75DFB074635
:1071900005AA31490020013650F08FFC0546DBE797
:1071A0002846FAF751FB8046F2E74946284650F058
:1071B0002AFE20B92A49284650F025FE08B144F09D
:1071C00001045146284650F01EFE28B9594628466B
:1071D00050F019FE0028DBD044F00204D8E7002C60
:1071E0004FF00003304608BF03241A4619460293A5
:1071F000E4B2CDE900841BF052FA054610B93946D5
:107200001848B7E7424639461748F9F70FFE39469E
:107210001648F9F70BFE164B2946D3F8B80545F08A
:1072200053FD39461348F9F701FE5CB16979A14273
:1072300008D022461048F9F7F9FD2B68E1B228463C
:107240009B699847EB6A002BE1D00C48F9F7EEFDFB
:107250000023EB62DBE700BF90100708301307083C
:10726000B14707085813070877130708E213070800
:10727000B0A8012094130708AC130708CC13070823
:10728000C12107082D130708062807082DE9F34731
:107290004FF0000A4FF0FF35DFF8D09001AA5746B3
:1072A0005446D0462E46314950F007FC68B9BAF131
:1072B000040F50D03ADCBAF1020F13DC2B463246F1
:1072C0002B49012045F0E2FD0EE0BAF1040F09D888
:1072D000DFE80AF0030D12171C00FAF7B5FA0646AC
:1072E00003281BD9FFF718FF02B0BDE8F087FAF7B3
:1072F000ABFA05468F28F4E7FAF7A6FA80463F284E
:10730000EFE7FAF7A1FA04463F28EAE70378482BAB
:1073100003D0562BE6D1012700E0002701AA4946F9
:1073200000200AF1010A50F0C8FBBFE7BAF1050FCF
:10733000D8D1A40108F03F08902304F47C6403FB37
:1073400006550C4E44EA080406EB450544EA47346A
:10735000A5F8F845C8E7902303FB0652054B03EB5D
:107360004203B3F8F875C7F34037E2E79010070817
:10737000A8AE0120B0A8012013460A4601460148E4
:107380001EE600BF101407082DE9F04F85B0054632
:10739000FCF716F9044630B10021012005B0BDE824
:1073A000F04F45F0EBBC6FF0004287492846F9F7F3
:1073B000E7FE20B905B0BDE8F04F38F013BC6FF020
:1073C000004282492846F9F7DBFE28B9012005B0C2
:1073D000BDE8F04F38F06EBD6FF000427C492846A2
:1073E000F9F7CEFE034680BB7A4A82F8F00D1046CC
:1073F00092F9F71D92F8A254012D08D0033D052DF6
:1074000005D9002C00F0D18080F8F71DCDE092F86E
:10741000A3540133A52D13D101290ED16E4A80F852
:10742000F13D002380F8F01D82F8783A80F8F73DAE
:1074300005B0BDE8F04F38F087BD0139012449B2ED
:10744000782B02F11402D5D1DBE72846FAF7FCF9D4
:10745000614B834693F9783A03FA80F60093772ECE
:1074600000F2A7802846FDF7FDF90746002800F046
:107470008980FAF7E9F90124C5B23846FDF7F2F937
:107480000746002800F081800134FAF7DDF9019009
:10749000E4B23846FDF7E6F98046002877D001349B
:1074A000FAF7D2F90746E4B24046FDF7DBF9814628
:1074B00000286ED00134FAF7C7F90290E4B24846CA
:1074C000FDF7D0F98246002865D00134FAF7BCF9FF
:1074D0000FFA80F9E4B25046FDF7C4F9824600285D
:1074E0005BD00134FAF7B0F90FFA80F8E4B25046F5
:1074F000FDF7B8F9002852D00390FAF7A5F90399DF
:107500000FFA80FA0846FDF7ADF90346002857D078
:1075100004F0FD04FAF798F9042C46D1C3B2012D0A
:1075200002D9E91E052940D81BB1A52B01D0482B53
:107530003BD1284C0EB984F8F76D1421019AA52B84
:1075400001FB0646C6F89024029A86F8A254C6F8B3
:107550009474C6F89824A6F89C94A6F89E84A6F87D
:10756000A0A486F8A3340AD100981B4B01305844DC
:1075700083F8780A94F8F73D013384F8F73D05B0B5
:10758000BDE8F08F0446054677E7019081E707469E
:107590008AE7029093E781469DE78046A7E75FFA76
:1075A00088F382468046062CB9D005B0BDE8F04F7E
:1075B000B2E577222146094805B0BDE8F04FDBE689
:1075C0000134E4B2EFE700BF2D14070833140708B5
:1075D000E01F070820870120B0A801203814070801
:1075E00010B50D4C94F8F43573B194F8F5355BB1E2
:1075F0000A48FFF7E5FC0A48FFF7E2FC002384F89D
:10760000F43584F8F53510BD0648FFF70DFC04F09D
:1076100088FE0020FFF73AFCB0A8012041140708BB
:1076200078140708961407082DE9F04F01F020039D
:107630008FB081460F464B4C4FF0000800934A4BE9
:10764000D3F83809FAF73EFA94F806B00BF0300395
:107650004B454BD1204611F02BF9FAF78FF906462E
:10766000204611F047F9D6F808A005460AEB0006B7
:10767000204611F073F90BF00F02062A6AD8DFE8F2
:1076800002F0043E43474C505C001AF80520007895
:10769000111A4A424A41009B03B13ABB03A9204652
:1076A000019211F08BF87B0615D5019A9AB903A9BE
:1076B0002E48FDF7BDF82E4903A849F051FE0028D9
:1076C0004AD11AF80530202B46D131462948FDF71A
:1076D000AFF8FFF751FC03A92748FDF7A9F80022EE
:1076E00031462046FFF77BFCFFF746FC08F1010816
:1076F0000B34B8F5127FA2D10FB0BDE8F08F1AF9A4
:10770000052090F90000C3E73AF805200088BFE79C
:107710003AF90520B0F90000BAE75AF805200068E8
:10772000B6E796ED007AD0ED007AB4EE677AF1EE26
:1077300010FA0CBF01220022ADE70190204611F0A3
:107740002BF90199421C304650F026FBB0FA80F22A
:107750005209A0E700229EE7002231462046FFF7AB
:107760003EFCB6E7AF8F0608B89701209D140708C6
:10777000AA670708A81407089E140708F8B50C4C58
:107780002E250C4E0C4F2068FFF74EFB616811B19F
:107790003046FDF74DF8A16811B13846FDF748F8BD
:1077A000FFF7EAFB013D04F11004ECD1F8BD00BF86
:1077B0005C870608AD140708B314070808B5FFF77F
:1077C00033FBBDE80840FFF7D7BB10B504460348BC
:1077D000FFF72AFB2046BDE81040EFE7B914070881
:1077E00010B5F5F791FF134CD0B11348FFF7EDFF3B
:1077F0001248FFF719FBD4F83809FAF763F94FF488
:107800007A70FFF720FA0E4BD3F8B8051BF0BAF8E0
:1078100013F03CF802210120FEF706F8FFF758F9B3
:107820000848FFF701FBD4F83809BDE81040FAF723
:1078300049B900BFB8970120BE140708A012070875
:10784000B0A80120DE14070808B50A480024FFF795
:10785000B5FF094BD3F83809FAF734F9074B83F829
:10786000794AC3F8BC4A83F8C04A12F095FE204614
:10787000FFF70CFB0D150708B8970120B0A80120F1
:1078800010B505221849044650F064FA60B9174B48
:1078900093F8F42522B9012183F8F52583F8F4152E
:1078A0001348BDE8104089E703221249204650F0F2
:1078B00051FA98B90D4C94F8F4355BB194F8F5355C
:1078C00043B10D48FFF77CFB002384F8F43584F8BE
:1078D000F53510BD0948FFF771FFF5E70848BDE829
:1078E0001040FFF76DBB00BFD51D0708B0A80120F1
:1078F0003715070801200708411407084D15070828
:107900006115070810B504460648FFF78DFA2046B2
:10791000FFF78AFA044B93F8F42512B1012283F899
:10792000F52510BD94120708B0A801200CB48306F9
:1079300007B500D551B905A904980191FFF72CFBB3
:10794000012003B05DF804EB02B070470020F8E7B7
:10795000024B0146D3F83809FAF7C0B8B8970120AE
:1079600030B5264885B0FFF75FFAF5F77FFB20B901
:10797000234805B0BDE8304020E7F5F7CFFE08B951
:107980002048F6E7F5F7D4FE02680446037D8179C6
:107990005208407CE51D0C34029020790190E0886B
:1079A00000901948FCF744FF15F8010BFFF7D0FFD2
:1079B000A542F9D1154C1648FFF736FA6378022B29
:1079C00006D007D9032B10D11248FFF72DFA0CE08F
:1079D0001148FAE704F580541048FFF725FA94F8A7
:1079E000B431022B06D0032B06D005B0BDE83040E1
:1079F000FFF7C2BA0A48E8E70A48E6E77015070841
:107A00007A15070888150708971507081C2F012005
:107A1000C5150708D5150708DB150708E815070879
:107A2000EE150708071607080CB407B510F040005C
:107A300009D069B92320FFF78BFF05A904980191AC
:107A4000FFF7AAFA012003B05DF804EB02B070471B
:107A50000020F8E72DE9F04F074687B016460C46A0
:107A600015464FF0000B4FF019094FF46178DFF81D
:107A7000A4A0002E4BD0237828788342EB7844D101
:107A800061786A78914240D1A178AA7891423CD13C
:107A9000E178CA1A51425141CDE9041310F006FAB7
:107AA000059B0499524619FB03830393AB7819FB9A
:107AB000038302936B7801934379384600935B46C6
:107AC000FFF7B2FF049920780435049110F0EEF925
:107AD000E37852460499043419FB0383039314F8A2
:107AE000023C19FB0383029314F8033C019343798E
:107AF000384600935B460BF1010BFFF717FFBBF114
:107B0000280FB6D107B0BDE8F08F0021C4E7314699
:107B1000D9E700BF19160708F7B50646FBF750FD71
:107B2000054630B100222549012003B0BDE8F040F0
:107B300090E73046F9F788FE2728044636DC8700B0
:107B4000701C8DF80750FCF78DFE1C4D064668B181
:107B5000F9F77AFE002809DBC0B210F0B9F928B1B4
:107B6000037905F8243001238DF807303046FCF7FF
:107B700079FE064650B1F9F767FE0D2806D8EB19D5
:107B800058709DF8073001338DF80730B91C0DF19E
:107B9000070230462944FCF771FE9DF80730042B9C
:107BA00002D0002345F8243003B0F0BD2722294637
:107BB000034803B0BDE8F040FFF7DEBB8C7B01203B
:107BC000FE1607082DE9F04F804689B00C46154691
:107BD00002F1540B334EDFF8D490069294F904105E
:107BE00000230C2202FB03F02F4FC057884254D0D1
:107BF0000133072BF6D10C350C345D45EED109B0BD
:107C0000BDE8F08F95F904302A689942687995F8B3
:107C100006C095F808E095F807A03CD1216891428C
:107C200039D16179814236D1A179614533D1217A47
:107C3000714530D1E179A1EB0A077942794156F8D3
:107C40002A7056F82000049756F82E700791039773
:107C500056F82C70CDE9002002974A464046FFF7BF
:107C6000E3FE0799E279404694F9043056F8222061
:107C70000492227A56F822200392A27956F8222002
:107C80000292627956F822200192226800924A46B6
:107C9000FFF74CFEAFE70021D1E7069B002BB1D1E7
:107CA0001946DFE768850608847301202C1607084B
:107CB000F0B585B00346FBF783FC30B100224349A1
:107CC000012005B0BDE8F0407CE718465E1CF9F7DE
:107CD000BBFD044640B21AF08FFC054630B9214680
:107CE0003B4805B0BDE8F040FFF76AB9006801AB5A
:107CF000696803C3A86818603046FCF7B3FD044602
:107D0000002853D003782B2B05D02D2B43D0F9F727
:107D10009BFD019009E001342046F9F795FD012211
:107D2000019B02FA00F0034301930226002720463C
:107D3000FCF798FD044638B3F9F786FD254A002381
:107D4000114652F804EB5FFA83FC704504D001330E
:107D5000112BF6D14FF0000C51F82C30984213D172
:107D6000102200216046F8F737FA022F20D0032FA7
:107D700021D0012F14BF8DF809008DF80A000137BA
:107D80000136042FF6B2D2D1012E17D805B0BDE8C6
:107D9000F040FFF7C1B901342046F9F755FD012243
:107DA000019B02FA00F023EA0003BDE70126BDE7CC
:107DB0008DF80C00E3E78DF80B00E0E701AB03CB97
:107DC000286018686960A86005B0F0BD287F0120B0
:107DD00049160708688506082DE9F04F804689B0E6
:107DE00017460C46154600264FF0190A4FF46179E4
:107DF000DFF8B4B0002F54D06979A8780791A17842
:107E00002B7881426A7895F803C095F804E00693D0
:107E100045D12178994242D1617891423FD1E178B0
:107E200061453CD12179714539D1079963795B1A54
:107E300059425941069B1AFB029206911AFB039381
:107E400003925A46CDE90103079B4046009333460F
:107E5000CDE904CEFFF7E8FD069923795A4640465E
:107E600006340593063514F8033C049314F8053CD6
:107E70001AFB0393039314F8063C1AFB0393029333
:107E800014F8043C019314F8013C00933346013686
:107E9000FFF74CFD142EADD109B0BDE8F08F0021E5
:107EA000C8E73946D9E700BF5C1607082DE9F34754
:107EB0008246FBF785FB064630B100223B49012094
:107EC00002B0BDE8F04787E75046F9F7BDFC13283C
:107ED000054663DC364C06278DF80760474304F6F9
:107EE000C1290AF10100FCF7BDFC09EB07080646B1
:107EF00048B1F9F7A9FC03289FBFE31983F8C60A24
:107F000001238DF807303046FCF7ACFC064668B11B
:107F1000F9F79AFC0D2809D8062303FB054383F8DB
:107F2000C30A9DF8073001338DF807300DF10702C1
:107F300041463046FCF7A2FCFCF794FC064668B1CB
:107F4000F9F782FC3B2809D89DF807300622013357
:107F500002FB05428DF8073082F8C40A3046FCF770
:107F600081FC68B1F9F770FC0D2809D89DF807303D
:107F70000622013302FB05448DF8073084F8C50A58
:107F80009DF80730062B06D0002349F80730A8F8E3
:107F90000430FFF7C1F802B0BDE8F0871322314684
:107FA000044802B0BDE8F047FFF7E6B971B301201D
:107FB000B0A80120FE1607082DE9F04F07469046AD
:107FC0000C4615460026DFF80CA12DED088B97B066
:107FD00094ED008AB5EE408AF1EE10FA71D0D4ED3E
:107FE000019A94ED029AD4ED038AB8F1000F40D0C3
:107FF00095ED000A95ED01BAB4EE408AD5ED02AADE
:1080000095ED03AAF1EE10FA60D1F4EE4B9AF1EE81
:1080100010FA5BD1B4EE6A9AF1EE10FA56D1F4EE92
:108020004A8AF1EE10FA0CBF4FF001094FF0000937
:1080300012A8F9F7AFFAB0EE4B0A83460EA8F9F78B
:10804000A9FAB0EE6A0A05900AA8F9F7A3FAB0EE09
:108050004A0A049006A8F9F79DFA049A059B494636
:108060000390384602925246CDE900B33346FFF7FB
:10807000DBFCB0EE480A12A8F9F78CFAB0EE690AF8
:1080800081460EA8F9F786FAB0EE490A83460AA897
:10809000F9F780FAB0EE680A049006A8F9F77AFAC0
:1080A000049B0390524600213846CDF800901034CE
:1080B0001035CDE901B333460136FFF737FC0C2EFE
:1080C00086D117B0BDEC088BBDE8F08F4FF00009EA
:1080D000AEE700BF7A16070870B50546FBF770FAE1
:1080E000064628B100222D490120BDE8704063E713
:1080F00005222B492846F9F743F838B9274B0022C7
:10810000013043F8102B0C28FAD170BD2846F9F73E
:108110009BFB0B2804463AD82846FCF7A3FB0646EF
:1081200048B3F9F7A1FA1D4B012503EB041383EDC6
:10813000000A3046FCF796FB064638B1F9F794FA88
:10814000164B013503EB041383ED010A3046FCF7AF
:1081500089FB064638B1F9F787FA104B013503EB76
:10816000041383ED020A3046FCF77CFB28B9BDE816
:108170007040FEF7D1BF0546DBE7F9F775FA07480F
:10818000032D00EB041484ED030AABD0EFE7314676
:108190000B220448BDE87040FFF7EEB8ECB30120B5
:1081A0002D140708FE1607082DE9F043804685B018
:1081B0000D46164602270024DFF858903EB336F8E5
:1081C000242035F82430F05B93421ED1EB5B191A62
:1081D0004B424B4119462346CDE900204A464046D2
:1081E0000391FFF721FC0399EB5B4A4640460437B5
:1081F000019335F82430009323460134FFF796FBB2
:10820000042CDBD105B0BDE8F0830023E2E7314662
:10821000EAE700BF8E160708F8B50446FBF7D0F969
:10822000054628B100222B490120BDE8F840BBE7F4
:108230006FF0004228492046F8F7A2FFA8B9274B63
:108240004FF47A714FF4FA62A3F8FC1BA3F8FE2BEB
:10825000A3F8001CA3F8022CA3F8041CA3F8062C16
:10826000A3F8081CA3F80A2CF8BD2046F9F7ECFA8D
:108270000328074627D82046FCF7F4FA044670B1D5
:10828000F9F7E2FA012506462046FCF7EBFA10B1B1
:10829000F9F7DAFA2DB9BDE8F840FEF73DBF05461B
:1082A000F2E7A6F2EE2240F2DC539A42F3D8A0F2B3
:1082B000EE229A42EFD8094B03EB8703A3F8FC6B3D
:1082C000A3F8FE0BD0E7294603220548BDE8F84095
:1082D000FFF752B8ACB401202D140708B0A8012054
:1082E0009F1607082DE9F04F834691B091460C4642
:1082F00015460026DFF8F0A004F11508042209A8AD
:108300000BAF41464FF05CFD00238DF82830D4E9D7
:108310000232082B72F1000155D21A462E49384616
:10832000F8F79EFDB9F1000F54D02B780793079A08
:10833000237893424CD1D4E90202D5E902139A4240
:1083400008BF884244D1227D2B7D9A4240D104222D
:1083500005F1150140464FF0F1FB002838D12169A5
:108360002B69CB1A594259411C4B5246584605932A
:1083700000230493B5F912300393B5F9103002933A
:10838000174B0193079B079100933346FFF74CFB74
:10839000079909AB5246584620350593237D04932F
:1083A000B4F912300393B4F91030CDE9017314F825
:1083B000203B009333460136FFF7B8FA082E9BD1D5
:1083C00011B0BDE8F08F07493846F8F749FDA9E735
:1083D0000021C9E74946DCE7DB430708F62C07081C
:1083E000EF4B0708A7160708B21607082DE9F74F45
:1083F0000446FBF7E5F8074630B100226E4901203C
:1084000003B0BDE8F04F6DE76C496FF000422046C5
:10841000F8F7B6FE014638B94FF48072664803B0EB
:10842000BDE8F04F4FF0B4BB2046F9F70DFA054612
:1084300083B2072B00F2B8802046FCF713FA82467D
:1084400000284CD0F9F700FA01240FFA80F95046C1
:10845000FCF708FA68B14FF00008411E00F1100C5B
:10846000464611F8013F13F0DF0F3BD101270134DD
:10847000E4B2FCF7F7F9824600284CD00134F9F752
:10848000E3F90FFA80FBE4B25046FCF7EBF9034640
:10849000002842D001340190F9F7D6F9019B0FFA78
:1084A00080FAE4B21846FCF7DDF90346002836D01E
:1084B00001340190F9F7C8F9019B42B2E4B21846C1
:1084C0000192FCF7CFF9019A034650B30134E4B2AC
:1084D000032C28D803B0BDE8F04FFEF71DBE0446BC
:1084E0008146B4E76145C2D0A3F13002D2B2092A75
:1084F00005D9A3F16102052A07D8573BDAB2360144
:1085000046EA187642EA0818ABE7A3F14102052AC9
:10851000ADD8373BF2E78346B6E78246C2E702466C
:10852000CDE7274BD4E71FFA89F10229D2D80BF205
:10853000262189B2B1F5E16FCCD80AF2262189B2A1
:10854000B1F5E16FC6D8D4B2062CC3D81846019352
:1085500048F010FF0428BDD8002FBBD02DB2164A1A
:10856000019B680102EB451102F8009002EB4512F5
:10857000A1F810B0A1F812A015320C75114DC1E987
:108580000286591E033311F8010F445D04F0030401
:10859000022C08BF203802F8010B087808B1994274
:1085A000F1D103B0BDE8F08F07223946064803B089
:1085B000BDE8F04FFEF7E0BE907801202D140708CB
:1085C000F62C0708F96C0708D31607082DE9F047C1
:1085D000814686B090460D4617460026DFF868A013
:1085E000B8F1000F2DD03B782A789A42D7E9010CD8
:1085F00025D16A68824222D1AC68A4EB0C025442B5
:10860000544121460093524633460594CDE9010C6E
:108610004846FFF709FA0599AB68524648460C37B9
:1086200002936B68019315F80C3B009333460136B7
:10863000FFF77CF9082ED3D106B0BDE8F0870024FF
:10864000DFE74146E8E700BFE01607082DE9F843F9
:108650000446FAF7B5FF054628B100222F4901204C
:10866000BDE8F843B2E72E496FF000422046F8F724
:1086700087FD014628B960222848BDE8F8434FF03D
:1086800087BA2046F9F7E0F80646C3B2072B06D9A9
:10869000294607222348BDE8F843FEF76DBE204671
:1086A000FCF7E0F8074630B3F9F7CEF8051E4FF0B7
:1086B000010418BF01253846FCF7D4F80746E0B19D
:1086C0000134F9F7C1F88046E4B23846FCF7CAF83D
:1086D0000746A0B10134F9F7B7F88146E4B238464D
:1086E000FCF7C0F808B10134E4B2032C09D0BDE8AE
:1086F000F843FEF711BD0446DDE78046E5E7814615
:10870000EDE776B2084B0C2000FB063686F80C5CD1
:10871000C6F8108CC6F8149CBDE8F883BCB40120E0
:108720002D140708F5160708B0A801202DE9F04F11
:1087300091B007468846164600240DF12C0ADFF852
:10874000789004EB8405514608EB050358F80500C2
:108750001B79029002A88DF80C3044F05FFA4EB3FA
:1087600073197059052204A91B790DF1180B049097
:1087700002A88DF814304FF0E1F9B0FA80F55946AF
:1087800004A86D0944F04AFA23464A462946384669
:10879000CDF800B0FFF748F9234601344A46294690
:1087A0003846CDF800A0FFF7C1F8202CC9D111B090
:1087B000BDE8F08F3546EFE7041707082DE9F04FC5
:1087C00089B00546FAF7FCFE044630B1002268493C
:1087D000012009B0BDE8F04FA8E72846F9F734F8C2
:1087E0001F28074600F3BB802846A246FCF73AF84C
:1087F0005F4ABB0006462546A346039307EB870363
:10880000A046A146D118D4505A4B0C710293019442
:10881000029B05AA13F801CB96460293002330462B
:1088200016F8011B19B18C4501D00A2B0CD108AEEA
:108830008C4533444FF0000603F80C6C08D009B0A7
:10884000BDE8F04FFEF768BC01330EF8011BE6E708
:1088500009F1FF33461C032B03D8DFE803F02E4554
:108860006E7705A8F8F7F0FF019009F101095FFAAA
:1088700089F9B9F1050FCBD1039A05F00F003E4BF2
:1088800004F00F043A44019944EA081417469A1870
:1088900003F66C4340EA01104FEA281882F86DBCD9
:1088A0001F4482F86C0C82F86EACFC7087F8048070
:1088B00009B0BDE8F04F28F06DBF05A8F8F7C4FF78
:1088C0000546D2E74E2B14D0452B14D0532B14D091
:1088D000572B14D0552B14D0442B05D1052301213F
:1088E00001FA03F348EA030812F8013B002BE9D12F
:1088F000BBE70023F3E70123F1E70223EFE70323BC
:10890000EDE70423EBE7DFF878C0002319461CF8F5
:10891000013B834204D0072901F10103F6D15946F6
:10892000DFF860C000231CF801EB70450AD101207C
:1089300000FA03F34AEA030A8B4612F8010B0028F7
:10894000E1D192E70133072BEDD1F5E705A8F8F760
:108950007BFF10280446B4BF0446002485E71F228D
:108960002146064809B0BDE8F04FFEF705BD00BF3F
:108970001CB501203C8A0608B0A80120FE16070895
:10898000418A0608498A06082DE9F047814686B0E3
:1089900090460D4616460027DFF860A0B8F1000F9C
:1089A0002AD033882A889A4224D16C887188621A26
:1089B00054425441F2782146484605940292B278D6
:1089C000CDE900323B465246FFF72EF80599EB7889
:1089D0005246484604360293AB78019335F8043B7F
:1089E00000933B460137FEF7A1FF102FD6D106B00A
:1089F000BDE8F0870024DDE74146E8E70E170708E9
:108A00002DE9F8430546FAF7DBFD044628B10022BC
:108A100025490120BDE8F843B6E72846F8F714FFDA
:108A20000F28064630DC28362846FBF71BFF1F4F71
:108A30000546DFF884804FEA86092846F8F704FFE8
:108A400037F8023B984226DC012C08EB090311D0D1
:108A5000022C12D0A3F86C0C28462C214FF065F99B
:108A6000054668B1013501230134A3B1032CE4D1DB
:108A7000BDE8F88383F86E0CEEE783F86F0CEBE744
:108A8000A21E53425341EFE721460F220848BDE89A
:108A9000F843FEF771BC074B002243F82620BDE8DF
:108AA000F843FEF739BB00BFBCB50120508A060869
:108AB000FE1607081CB50120B0A801202DE9F04FD3
:108AC000144685B00646894600274FF0060B284A13
:108AD0000BFB07F54FF00008E03519F805A0002C56
:108AE00042D0635DAAEB0300414241413046CDE9EB
:108AF00000833B460391FEF797FF03991C4A3B46D0
:108B000030460135CDE9008A08F10108FEF70EFF75
:108B1000174AB8F1060FE0D10137062FD8D14FF42C
:108B20008275134FA5F5827819F805A0F4B1635D3D
:108B30003046AAEB0302514251413A46CDE9008347
:108B400006230391FEF770FF039906233A46304649
:108B50000135CDE9008AFEF7E9FE40F20D139D4292
:108B6000E0D105B0BDE8F08F2146C8E72146ECE72B
:108B7000201707082DE9F043804687B017460C46BA
:108B800015460026DFF88C90002F40D0B5F9003054
:108B9000B4F90010B5F902209942B5F9040095F92D
:108BA00006C032D1B4F9021091422ED1B4F90410AA
:108BB00081422AD194F90610A1EB0C0EDEF10001DE
:108BC00041EB0E010591CDE90032CDE9020C3346AF
:108BD0004A464046FEF728FF059994F906304A4672
:108BE000404608350393B4F904300293B4F90230D7
:108BF000019334F9083B009333460136FEF796FEA5
:108C0000102EC1D107B0BDE8F0830021DAE7394664
:108C1000E3E700BF341707087FB50546FAF7D0FC35
:108C200000285BD000222E49012004B0BDE870402E
:108C3000A0E72D2B03D0A3F13002092A49D8042C38
:108C400004DD04B0BDE87040FEF766BA2846F8F7C8
:108C5000FBFD04AB621C03EB440424F80C0C15F878
:108C6000013F303B092BFAD914462B78002BE0D179
:108C7000052CE6D1BDF80430BDF904600F2BE0D817
:108C8000BDF90610A1F5FA7292B2B2F5FA6FD8D812
:108C9000BDF90820A2F5FA7080B2B0F5FA6FD0D80D
:108CA000BDF90A008142CCDC8242CADB9142C8DCB9
:108CB000BDF90C5005F17D04A4B2FA2CC1D8084BC3
:108CC00023F8361003EBC6035A8098809D7104B0D8
:108CD00070BD202BB5D101352246C5E70446C4E757
:108CE000D47401202DE9F04F80468FB017460C4612
:108CF00015460026DFF8A8B0A3882068ADF82C3010
:108D00002378B4F902900893637894F905A0069348
:108D100023790A900793B9F1000F3AD0002F3DD084
:108D20002868BDF828100C9080B2AB8881422A7860
:108D3000ADF8343095F801C0B5F9023095F804E08B
:108D40002AD14B4528D1BDF82C10BDF83400081AA3
:108D500041424141009240465A460991CDE901C342
:108D6000CDE903EA3346FEF75FFE0999079B5A46B1
:108D70004046CDF810A006340635CDE90293069B97
:108D80000193089B009333460136FEF7CFFD202E5A
:108D9000B2D10FB0BDE8F08F0021DBE73946E5E73F
:108DA00049170708F0B589B0044648F0E3FA10F017
:108DB000FF0205D12C49012009B0BDE8F04091E740
:108DC00005222A492046F8F7DBF930B91521264853
:108DD00009B0BDE8F04047F049B9204601AA24494E
:108DE00002AD4EF06AFE00244FF0FF33204E079391
:108DF00078B1062C02D1FEF78FF933E0F8F724FDA5
:108E000001AA45F8040B3146002001344EF055FE0E
:108E1000EEE7042CEFDD029E1F2EECD8039D0F2DF4
:108E2000E9D8049C252CE6D8059800F57A73B3F5AB
:108E3000FA6FE0D80699FF29DDD8079A531C402B1A
:108E4000D9D80C4B062707FB0633A3F87C0D83F813
:108E50007A5D094883F87B4D83F87E1D83F87F2D6A
:108E6000FFF7A0FF09B0F0BD2AB601202D140708B6
:108E700090100708B0A80120F62C07082DE9F04F44
:108E800007469BB093460C4615460026DFF804A122
:108E90000E930E9B5A1C01D0B3426FD1A6460DF122
:108EA000400C94F8048094F81390BEE80F00ACE8EE
:108EB0000F00DEF800300890CCF80030237B0992D8
:108EC0000A93237C0B9394F911300C93A37C0D939C
:108ED000BBF1000F5CD0AE460DF1540CBEE80F00A4
:108EE000ACE80F00DEF80030149ACCF8003023F024
:108EF0007F4322F07F420F9095F804E09A42A868E1
:108F000095F80CC0E97C41D1F0453FD1089B0F9A00
:108F100093423BD10A9B634538D1099B834235D1AB
:108F2000A9EB010359425941099B52463846CDF8F5
:108F30001C9006930A9B0F910593089BCDE9038330
:108F40000D9B02930C9B01930B9B00933346FEF702
:108F50006BFD0F99099B52463846CDF81C9006933D
:108F60000A9B0593089BCDE903830D9B02930C9B01
:108F700001930B9B00933346FEF7D8FC0136143463
:108F80001435402E85D11BB0BDE8F08F0021CBE712
:108F90005946DFE7601707082DE9F0418AB004461B
:108FA0000D4648F0E7F910F0FF0211D13F4991F862
:108FB000F40548B94FF0FF33024601F63C61012049
:108FC0000AB0BDE8F04159E76B1C6CD02B46F4E7C2
:108FD000052237492046F8F7D3F838B94FF47E71A7
:108FE00034480AB0BDE8F04147F040B8204601AD32
:108FF0000024314E6A4630494EF05FFD78B1092CAD
:1090000002D1FEF789F84EE0F8F71EFC6A4645F8F3
:10901000040B3146002001344EF04FFDEEE7092CE1
:10902000EFD101993F29ECD8DDF808E0BEF1010F3E
:10903000E7D8DDF80CC00CF10103402BE1D8049F08
:10904000332FDED8059E072EDBD8069D1B4A05F57B
:10905000742303F510739342D3D8079C072CD0D800
:10906000089800F5742303F510739342C9D8099A40
:10907000FF2AC6D80D4B4FF0140808FB013309B284
:10908000C3F8440E83F84CEE0D4883F84DCE83F8B8
:109090004E7E83F8406EC3F83C5E83F8484E83F8FA
:1090A0004F2EFFF779FF0AB0BDE8F081B0A801208C
:1090B0002D140708ECB601209010070880841E00CC
:1090C000F62C07084FF0FF3166E72DE9F04F164602
:1090D000154687B007460C464FF0000B194AD4F8E6
:1090E0000880D4E9009A56B3AB689845D5E90001E9
:1090F00023D1814521D1AAEB0103594259415B4655
:109100003846CDF800800591CDE9019AFEF78CFC38
:1091100005990C4A5B460BF1010B3846CDF80080EF
:109120000C340C35CDE9019AFEF700FCBBF1080FB9
:10913000044AD4D107B0BDE8F08F0021DFE7314603
:10914000E8E700BF8117070870B586B0044648F00D
:1091500011F910F0FF0205D12149012006B0BDE848
:109160007040B2E705221F492046F8F709F838B9E0
:1091700040F2FF311A4806B0BDE8704046F076BFB5
:10918000204602AD0024184E01AA17494EF095FC66
:1091900078B1042C02D1FDF7BFFF1FE0F8F754FBB4
:1091A00001AA45F8040B3146002001344EF085FC3D
:1091B000EEE7042CEFD1029A072AECD80B4B0C21D6
:1091C0000B4801FB0233039AC3F84C22049AC3F8FC
:1091D0004422059AC3F84822FFF7B6FF06B070BDD7
:1091E000ECBB01202D14070890100708A8B9012036
:1091F000F62C07082DE9F04F8046A1B017460C4623
:1092000015460026DFF8F8B0A6460DF1480C94F894
:109210000C9094F818A0BEE80F00ACE80F0023688B
:109220000C9323790A93A3680B93238A0D93638A83
:109230000E93A38A9EE807000F93E38A8CE8070049
:109240001093002F5AD0AE460DF1640CBEE80F000B
:10925000ACE80F002B7E9EE8070053458CE8070022
:109260004AD12B790A9A934246D12B680C9A9A429A
:1092700042D12B7B4B453FD1AB680B9A9A423BD1F5
:10928000169A824238D117991E9BCB1A59425941DE
:10929000109B5A464046119108930F9B07930E9BD3
:1092A00006930D9B05930B9BCDE903930C9B0293B7
:1092B0000A9BCDE900A33346FEF7B6FB1199109B3C
:1092C0005A4640461C3408931C350F9B07930E9B4F
:1092D00006930D9B05930B9BCDE903930C9B029387
:1092E0000A9BCDE900A333460136FEF71FFB042E8F
:1092F0008AD121B0BDE8F08F0021C9E73946DEE709
:10930000921707082DE9F0438DB0044648F032F873
:1093100010F0FF0205D13E4901200DB0BDE8F04339
:1093200068E705223B492046F7F72AFF38B94FF492
:109330007E7137480DB0BDE8F04346F097BE204639
:1093400002AD0024344E01AA33494EF0B6FB78B189
:109350000A2C02D1FDF7E0FE57E0F8F775FA01AAF2
:1093600045F8040B3146002001344EF0A6FBEEE731
:109370000A2CEFD1DDF80880B8F1030FEAD8DDF848
:109380000CE0BEF1010FE5D8DDF810C0BCF1070F0D
:10939000E0D8059F214B07F5742202F510729A421E
:1093A000D8D8069E072ED5D8079D05F5742202F55C
:1093B00010729A42CED8089CB4F5004FCAD20998D0
:1093C000B0F5004FC6D20A99B1F5004FC2D20B9A40
:1093D000B2F5004FBED2124B4FF01C0909FB083307
:1093E000A3F8B60283F8BCE20E4883F8A8C2C3F81B
:1093F000A47283F8B062C3F8AC52A3F8B442A3F8E5
:10940000B812A3F8BA22FFF77DFF0DB0BDE8F083D4
:109410004CBC01202D1407089010070880841E0002
:10942000A8B90120F62C07080FB407B504A951F814
:10943000040B0191FDF7B0FD03B05DF804EB04B03F
:109440007047F7B58479054614F0C00303D0402B6C
:1094500018D003B0F0BD04F00F040FF09DFA062CF5
:1094600005D10146164803B0BDE8F040DCE70190A5
:1094700028460FF080FA019A0146124803B0BDE871
:10948000F040D1E70024104E104F0FF013FB0546BB
:109490000F48FDF7C9FC2B79A34204D803B0BDE8FF
:1094A000F040FDF769BD14B13046FDF7BDFC2B68F7
:1094B000384653F824100134FBF7BAF9EBE700BF44
:1094C000B4170708C4170708EB1707089918070807
:1094D000DB1707082DE9F0478CB0074610F8013B71
:1094E000202BFAD000251F4CDFF880802E46DFF8B5
:1094F0008090DFF880A001A920460FF05FF939467F
:1095000001A84EF080FCE0B101A94046FBF790F9BC
:10951000494601A847F024FFF0B920460FF01EFA93
:10952000114B0146007820280CBF50461846FBF727
:109530007FF90136FDF720FD2046FFF782FFFDF79A
:109540001BFD01350B34B5F5127FD4D10EB943F0B4
:10955000FFFB0CB0BDE8F08700212046FDF7D0FDF1
:10956000E7E700BFAF8F0608B6140708A214070884
:10957000AA670708A81407082DE9F04F2DED028B04
:109580008DB0067805460130202EFAD0284647F0E7
:10959000F1FE044618B101281FD12A2E1DD1894D94
:1095A0000026894F8948FEF709F9284601A90FF0DE
:1095B00005F9013601A93846FBF73AF92846214654
:1095C0000B35FDF79DFDFDF7D7FCB6F5127FECD10D
:1095D0000DB0BDEC028BBDE8F08F3D2128464EF06A
:1095E000A4FB002800F0E7800346984613F8012DFD
:1095F000202AFAD0A8EB05080130074610F8013BF5
:10960000202BFAD06F4E4FF000095FFA88F8B3466E
:1096100001A930460FF0D2F801A847F0ABFE01A92E
:10962000024682462846F7F7ABFD044648BBC245D2
:1096300027D10B2303FB09B999F8063003F00F0873
:10964000B8F1060F32D1384647F094FE8442054601
:1096500020D35F4901A847F083FE20B15D4901A8EE
:1096600047F07EFEF8B93B78222B1CD17B1913F80A
:10967000013C222B17D1AA1E791C30460FF036FA76
:10968000A6E709F101090B36B9F5127FC0D143F005
:109690005FFB9DE73B5DA3F16102192A9CBF203B64
:1096A0003B550134CFE72A463946E6E713F0C003BD
:1096B0000AD0402B4DD04848FEF724F93046FFF73A
:1096C000C0FEFDF759FC83E73B78002BF3D04349FC
:1096D00038464EF088FB0446384647F04BFE84423D
:1096E000E9D13846F7F7C0FF3046B0EE408A0FF0B8
:1096F00042F907EE900AF8EEE77AF4EEC87AF1EE56
:1097000010FAD8D830460FF047F907EE900AF8EE75
:10971000677AF4EEC87AF1EE10FACCDBB8F1050FF7
:109720000CD118EE104A30460FF018F9B8F1050FB9
:1097300032D8DFE808F030303A3A3C3EB8F1040F56
:10974000384603D1F8F766F80446ECE7F8F77CF8FA
:10975000FAE7304625460FF0ADF9A246814690F86B
:1097600004B02346AB4500D91BB1BAF1000FA2D01B
:10977000D9E7D9F800306FF00042394653F8250098
:10978000F7F7FEFC002805BF2C46012300234FF00D
:10979000010A0135E6E7047001A91148FBF748F812
:1097A00000213046FDF7ACFC12E70480F4E70460CA
:1097B000F2E70460F0E728460DB0BDEC028BBDE88F
:1097C000F04F87E6AF8F0608A2140708ED170708C9
:1097D000AA670708FF170708231807080A180708C9
:1097E0001818070870B586B00346F9F7E9FE044675
:1097F00038B100221949012006B0BDE87040FFF7DA
:109800005DB903AD164E02AA154918464EF055F93A
:1098100080B1032C03D1FDF77FFC06B070BDF8F7D3
:1098200013F802AA45F8040B3146002001344EF02B
:1098300044F9EDE7032CEED1059BDDE903451A461B
:1098400001932946E0B228F0D5F80028E3D0019B27
:109850002A4621460348FFF7E7FDDEE71CB5012055
:10986000901007082017070808B50346F9F7A8FE67
:1098700040B10C4B00220C48A3F8F625BDE8084087
:10988000FDF79CBF1846F7F7DFFF014630B1054BE7
:10989000A3F8F6050548BDE80840C5E5BDE8084061
